:020000040800F2
:100000000020001089000308C548020805C3000845
:10001000C3480208C1480208BF48020800000000A7
:10002000000000000000000000000000BD480208C1
:10003000BB48020800000000B9480208C9DB0008FC
:10004000F1000308F1000308F1000308F1000308C0
:10005000F1000308F10003082517010851180108F1
:1000600015180108D91701089D170108E51E000899
:10007000D51E0008C51E0008B51E0008A51E0008F4
:10008000911E00087D1E0008F1000308F10003081E
:10009000E1490208F1000308F100030861170108B3
:1000A00019D3000849D3000809D3000871D3000808
:1000B00039D3000829D30008F1000308F100030830
:1000C000F1000308F1000308F1000308F100030840
:1000D000F1000308F104010875040108F90301089F
:1000E000E9160108F1000308A9480208F100030815
:1000F000F1000308F1000308F1000308F100030810
:10010000000000000000000000000000F1000308F3
:10011000F1000308F1000308793401085D34010897
:10012000691E0008551E0008411E00082D1E00080B
:10013000191E0008F1000308000000000000000084
:10014000F1000308F1000308F100030800000000BB
:10015000000000000000000000000000000000009F
:100160000000000000000000F1000308F100030897
:10017000F100030800000000000000000000000083
:0801800000000000F10003087B
:10018800002870B51EDB0928044620DD012303EB97
:1001980083035B00B0FBF3F2092AF8D87BB10E4E5B
:1001A800B4FBF3F00928CCBF57223022A6FB03E5A5
:1001B800024403FB1044EB0801F8012BF0D10023A3
:1001C8000B7070BD2D230B7040420131DBE73030DE
:1001D80001F8010BF3E700BFCDCCCCCC884230B49A
:1001E8004FF001042ED301FB04F4B0FBF4F58D426B
:1001F800F9D284B1AAB901E0B0FBF4F5092DCCBF5E
:10020800572230222A4404FB150003F8012BB4FBC3
:10021800F1F4002CF0D100221A7030BC7047B0FB0A
:10022800F4F5092DCCBF372230222A4404FB1500EF
:1002380003F8012BB4FBF1F4002CF0D100221A7062
:1002480030BC70470546002AEBD1D7E703685A1C33
:1002580002601970704700BF2DE9F047089C2578A7
:10026800002B804689460CBF4FF0200A4FF0300A19
:10027800661C35B3002A29DD334601E0024698B1F1
:1002880013F8011B501E0029F8D1971E60B13D4696
:10029800013D51464046C8476B1C002BF8DC2578C9
:1002A80027EAE770013055B1041B29464046C84784
:1002B800301916F8015B002DF7D1BDE8F087BDE8CD
:1002C800F087002A04DC2846BDE8F0870020EBE729
:1002D800571EDCE783684268D0ED037A00EB8301A0
:1002E8000133934281ED040A836004BF00238360D5
:1002F80000EB830393ED047A036870EE277A9A4241
:10030800C0ED037A77EEC77AC0ED037A0CDA0133D1
:1003180007EE103AF8EEC76AB7EE007A87EEA60A3B
:10032800036030EE070A704707EE102AB8EEC77A66
:1003380087EE870A704700BF90ED057A90ED004A76
:10034800D0ED066AD0ED014AD0ED047A90ED035A5B
:10035800D0ED025AA4EE007AB0EE406AB0EE470A39
:10036800B0EE667AA6EE247A67EEC07AA0EE457AF9
:10037800E6EE257A80ED057AC0ED067A704700BF73
:10038800D0ED057A90ED013AD0ED003AD0ED064A6D
:1003980090ED024A90ED077A90ED035A90ED086AC5
:1003A800D0ED045AC0ED067AF0EE406A27EE830AD3
:1003B800C0ED056AA3EEA60A80ED087AA4EE240A29
:1003C800A5EE470AA5EEC60A80ED070A704700BFEA
:1003D800D0ED007A90ED017A30EE670AE7EE007A08
:1003E800B0EE670AC0ED007A704700BF704700BFE3
:1003F8000A44914214D030B40139551E41F2210209
:1004080011F8014F082380EA042004044CBF82EA53
:1004180040004000013B80B2F7D18D42F0D130BCA2
:10042800704700BF012380F84530704790F82030AE
:1004380033B1012B03D14FF40063838270477047B7
:100448004FF480638382704770B40468037B22682A
:10045800022101FA03F31A4213D042690A495C20C7
:1004680000FB02124FF6FE7650685289C568006894
:10047800296831402960C168D24392B20A40C260FB
:10048800636070BC704700BF645A002030B40A4BE8
:100498001D7875B1094B002003EBC5051A689988CA
:1004A8005062D4682143D160083323F8040CAB426E
:1004B800F4D130BC704700BF445D0020485D002087
:1004C80010B40268047B11680223A340194209D0C2
:1004D8000649406800240C7001684FF6FE742140FC
:1004E800016053605DF8044B704700BF3E4F002029
:1004F800014B186810F0A6B8EC19002010B490E869
:100508000600047B40690223A3404B6013685DF832
:10051800044B4FF6FE710B40136010F023B8F8B58A
:10052800174D2B78A52B28D16B78BE2B25D102220D
:1005380029464FF6FF70FFF75BFF124FAC1C22886D
:100548004AB1A618BE4218D2052A16D92146FFF785
:100558004FFF3446F3E721460222FFF749FF022204
:10056800A118FFF745FF0634074B641B1C8041F6B2
:100578000F53C31A58425841F8BD0020F8BD00BFB8
:1005880000F0030800000408663500202DE9F04F4C
:10059800DFF848914C4F8BB00326A7EB09071822C8
:1005A800002104A830F051FF484BCDF81090059772
:1005B8001A69120604D5464A5A6002F188325A600E
:1005C80001228DF824203422DA60424B424C1B88E9
:1005D800ADF800300222694604A811F0A3FA0222FD
:1005E80069464FF6FF70FFF703FFDFF8F4A0804677
:1005F8004FF0000B544536D30AAC002524F8245D8F
:100608000222214604A811F08DFA02222146404612
:10061800FFF7EEFE40BAC043ADF80800022202A977
:1006280004A811F07FFA079860B106ABC0F1040284
:100638002946184430F009FF069904A811F018FA61
:10064800079508909DF82430089A23B11F490B6933
:1006580043F080030B61013E2DD0002A9FD1FFF7A4
:100668005EFF50B32CE065888DF80DB0C5F30B051F
:10067800AB1DADF808302388C3F30B02ADF80A2090
:100688001B0B062202A904A88DF80C3011F04AFAB7
:10069800062202A94046FFF7ABFE616880462A465B
:1006A80004A811F03FFA616840462A46FFF7A0FE09
:1006B800143480469EE7002AD1D005200BF05EFE58
:1006C8000BB0BDE8F08F00BF000004080020024016
:1006D8002301674530150308C070030800F00308BC
:1006E800207503080378202B024600F10100F9D099
:1006F800092BF7D02D2B2CD02B2B03BF5378B7EE1B
:10070800000A0246B7EE000AA3F13001C8B2092870
:100718009FED467A10D8F2EE046A07EE901AF8EECA
:10072800E77A12F8013FE7EE267AA3F13001C8B262
:100738000928B0EE677AF0D92E2B4CD003F0DF03EE
:10074800452B0BD0F7EE007A67EE276A20EE260AD3
:1007580070475378BFEE000A0246D5E710B45178C7
:100768002D2959D02B290ABF9178501C901C0024A0
:10077800A1F13003092B53D8002303EB830301EBCA
:10078800430310F8011FA1F13002092AA3F1300335
:10079800F3D9B3F59A7F28BF4FF49A73072B42D940
:1007A800DFED236A1A46F7EE007A083A072A67EE61
:1007B800A67AFAD803F007032BB1F2EE046A013BDC
:1007C80067EEA67AFBD124B3C7EE276A5DF8044B1F
:1007D80020EE260A70475378A3F13001C8B20928E1
:1007E80002F10102AAD8F2EE046AF0EE665A07EEA8
:1007F800901AF8EEE77A12F8013F87EEA66AA3F19D
:100808003001C8B2092866EEA56A37EE067AEED935
:1008180094E767EE276AD9E7901C91780124A7E747
:10082800F7EE007ACFE7F7EE007AC5E700000000A0
:1008380020BCBE4CB5EEC00ADFED317AF1EE10FAFD
:10084800CCBF30EE270A30EE670ADFED2E7A20EEB5
:10085800270A30B5FDEEC07A87B017EE904A0546F4
:1008680084EAE470002303A9A0EBE47001930093E9
:1008780002932DF0C5FB002CACBF20232D2303A829
:100888008DF800302EF07EFD012803A924D002281F
:100898002DD0032805BF3023684668468DF80130FF
:1008A80030F0DBFD68462EF06DFD0338C4B22246F9
:1008B8006946284630F008FE00232B5528462EF0BE
:1008C80061FD2E22431C2A540DEB0401E81830F078
:1008D800E1FD284607B030BD302368468DF8013069
:1008E8008DF802308DF8033030F0B7FDDAE73023A9
:1008F80068468DF801308DF8023030F0AEFDD1E752
:100908006F12033A00007A442DE9F0410646154675
:100918000846B6FBF2F43CB905FB1464124B1B5DA8
:1009280000F8013BBDE8F081B4FBF2F767B90E4B64
:1009380005FB174705FB1464DA5D00F8012B1B5D06
:1009480000F8013BBDE8F081B7FBF2F8B8F1000F01
:1009580002D04046FFF7D8FF05FB1878024B13F882
:10096800082000F8012BE3E76C4203082DE9F04763
:1009780014461D46064600234FF47A72204629463F
:100988002FF0AAF9DFF848814B4A4C4F88FB003119
:100998000144C31782FB002EC3EB611188FB0128B9
:1009A80087FB00278644464AC3EBEE2EC1EB011CA9
:1009B80082FB0E29A0EB8C0C0744424A86F806C03D
:1009C800C3EB27474FEAEE7C08EB010ACCEBA90CF6
:1009D80082FB07824FEAE1780CEB4C0CC8EB6A18F3
:1009E800AEEBCC0EC8EB0818DFF8E8C086F804E0D8
:1009F800A1EB880171718CFB0010F917C1EBE212B1
:100A080040F2B55101FB1272C3EBE050B2F5896FA9
:100A18004FEA80073FDA40F2DA239A4243DCB2F524
:100A2800B77FB4BF4FF0000C4FF0010C4FEA4C08F1
:100A3800254B08EB0C0103EBC1031FFA8CFE588B06
:100A4800224908EB0C0301EBC30116310B2301E02B
:100A580031F8020D82421BDA013BF9D11A4BC4442A
:100A680003EBCC0C0123BCF80400B37007F2B27797
:100A78000132121ABE44F270A6F800E02046294658
:100A88004FF47A7200232FF027F93281BDE8F087FE
:100A98000133DBB2E9E74FF0030EF44640F296501B
:100AA8004FF00608CCE74FF0020EF44640F229401A
:100AB8004FF00408C4E700BFC5B3A29107452EC292
:100AC800ABAAAA2A73B06D163015030834150308AB
:100AD80089888888792D0311104B2DE93048D3E98E
:100AE800004554EA05020BD1034601220020187183
:100AF800587198719A70DA7018801881BDE830883A
:100B0800074B1A6814EB020B45F1000C5A46634672
:100B1800FFF72CFF0120BDE8308800BFB016002089
:100B28004C470020F0B402888578164FC3780479C2
:100B38004179A2F2B27202F0030606EB4606013DC5
:100B480005EB860507EB4505013BAE8885790089ED
:100B580040F2B557920807FB0232931903EB43039F
:100B680004EBC303C3EB031301EB8303C3EB0313CE
:100B780005EB830300214FF47A72C2FB0301F0BC3A
:100B8800704700BF30150308FAB170B48E180446D8
:100B980003E0101A14D1B14214D014F8012BA2F1B9
:100BA8004103192B11F8013BA3F1410598BF2032ED
:100BB800192D03F12000ECD9D01A01D1002BEAD16C
:100BC80070BC7047002070BC70471046704700BF6B
:100BD8004FF0FF32FFF7D8BFA0F16103192B98BF80
:100BE80020387047A0F14103192B98BF2030704777
:100BF800202805D0093804288CBF00200120704720
:100C080001207047613819288CBF002001207047E7
:100C1800413819288CBF0020012070473038092836
:100C28008CBF002001207047A0F13003092B07D9A1
:100C380020F02000413819288CBF0020012070477F
:100C48000120704730B402681146531C036011F844
:100C5800024B0160D31C517803609378151D056021
:100C68001B0443EA0123D078234343EA006030BCE5
:100C7800704700BF0368591C1A46016012F8021B2E
:100C88000260587841EA0020704700BF03685A1C88
:100C980002601878704700BF38B5044600681546EA
:100CA8002FF0D8FA22682A44226038BD036810B4AD
:100CB8000A0A5C1C04601A7003685A1C02601970E6
:100CC8005DF8044B704700BF03685A1C026010B4FB
:100CD800197003680A0A5C1C04601A7003680A0C1D
:100CE8005C1C04601A700368090E5A1C02601970B3
:100CF8005DF8044B704700BF03685A1C0260197006
:100D08000368090A5A1C0260197070472DE9F047F8
:100D1800002488B080460F461E46A14605AD531CE8
:100D28000393117839B3252933D1931CCDF810904A
:100D38000393507830284ED04FF0000AA0F13003CA
:100D4800DBB2092B42D96C2819D0642800F09380B3
:100D580024D825281CD063D9582876D063281BD1DD
:100D680031784046B847039A531C039311780436E8
:100D780001340029D7D1204608B0BDE8F087039B8D
:100D88005A1C03921B78642B7CD02AD8252B54D16B
:100D9800252140460134B847039AC0E7732833D069
:100DA80044D975284FD106F1040E30682B4600222D
:100DB8000A217646FFF712FA049A009553463946F7
:100DC8004046FFF749FA039A0444A8E704AA03A98E
:100DD8002DF05EF8B7E7D31C039390784FF0010A23
:100DE800ACE7732B10D05BD9752B3AD0782B96D102
:100DF800A3F15802B2FA82F2306852092B46102148
:100E08000436FFF7EBF9D7E73368049A00933946BD
:100E180000234046FFF720FA04360444039A7EE78D
:100E28000028B9D1204608B0BDE8F0876E28B3D1B4
:100E3800039A336804361C6071E72AD9582BD7D037
:100E4800632B8DD06BE77828A6D1A0F15802B2FAAF
:100E580082F2306852092B461021FFF7BFF9043699
:100E6800AAE706F1040E30682B4600220A217646CE
:100E7800FFF7B4F9A0E7331D306829461E46FFF78F
:100E88007FF999E7331D306829461E46FFF778F940
:100E980092E7002B7FF443AF204608B0BDE8F08707
:100EA8006E2BC6D03BE700BF0EB400B584B005ABCF
:100EB800019053F8042B0649039301A8FFF726FF76
:100EC800019B00221A7004B05DF804EB03B0704770
:100ED800550200080FB430B583B006AB0A490B4879
:100EE80053F8042B096800680193FFF70FFF084CBB
:100EF800054620680FF096FB0028FAD0284603B074
:100F0800BDE8304004B070476C25002070250020F3
:100F1800EC190020DFED2B7AB4EEE70AF1EE10FAB7
:100F28004ADDDFED296A9FED297A01E0B0EE670A14
:100F3800B4EEC70AF1EE10FA70EE667AF6DC9FEDB1
:100F4800247AF4EEC77AF1EE10FA38D5DFED1E6A8E
:100F58009FED207A01E0F0EE407AF4EEC77AF1EEE8
:100F680010FA37EEA60AF6D4DFED1B7AB4EEE70ADC
:100F7800F1EE10FA14DDDFED137A37EEC00A60EEF9
:100F8800006A9FED166A9FED167ADFED167AA6EED7
:100F9800867A20EE266AE6EE877AA6EE270A70475A
:100FA800DFED117AB4EEE70AF1EE10FA44BFDFED97
:100FB800087A37EEC00AE2E7F0EE407ABFE7B0EE13
:100FC800670AD1E7DB0F4940DB0FC940E4CB164184
:100FD800DB0F49C0E4CB16C1DB0FC93F92E741B92B
:100FE8009730083C15A82ABEDB0FC9BF09B909E02C
:100FF800194690FBF1F301FB13030846002BF7D1C8
:10100800084670470146FBE707EE901AF8EE677A44
:101018009FED837A27EE800A20EE070AFDEEC07A5C
:1010280017EE903A2033402B00F28C80DFED7D7A6A
:10103800B4EEE70AF1EE10FA40F3E880B0EE407A39
:101048009FED796ADFED796A01E0B0EE677AB4EE78
:10105800E67AF1EE10FA77EE467AF6DC9FED747ACE
:10106800F4EEC77AF1EE10FA40F1CD809FED6E6A8A
:10107800DFED706A01E0F0EE477AF4EEE67AF1EE21
:1010880010FA37EE867AF6D4DFED6B7AB4EEE77AAB
:10109800F1EE10FA51DCDFED697AB4EEE77AF1EEA1
:1010A80010FA44BFDFED627A37EEC77A27EE076A97
:1010B800DFED635ADFED637ADFED636A9FED635A14
:1010C800E6EE257A67EE065AE6EE276AF7EE007A2C
:1010D800A5EEA67AF0EE675AE7EE055AE7EE457AEE
:1010E80087EEA55ADFED547A30EE277AFDEEC76A0F
:1010F80016EE903A2033402B29D99FED557AF6EE1B
:10110800006AB7EE006AF7EE004AC4EEA57A00233B
:10111800836143610362C36180ED045A67EEA66A86
:1011280027EE866A27EE877AC0ED006AC0ED026A6C
:1011380080ED016A80ED037A7047DFED3A7A37EE89
:10114800C77AB3E7B7EE005AF0EE455ACAE7B4EEED
:10115800E70AF1EE10FA5FDD9FED336ADFED336ADF
:1011680001E0B0EE677AB4EEE67AF1EE10FA77EEC7
:10117800467AF6DC9FED2E7AF4EEC77AF1EE10FA95
:1011880047D59FED296ADFED2B6A01E0F0EE477A3B
:10119800F4EEE67AF1EE10FA37EE867AF6D4DFED61
:1011A800267AB4EEE77AF1EE10FA27DCDFED237A3F
:1011B800B4EEE77AF1EE10FA44BFDFED1D7A37EEB0
:1011C800C77A27EE076ADFED1E4ADFED1E6ADFEDFC
:1011D8001E7AE6EE246A67EE064AE6EE267AB7EE4F
:1011E800006AA4EEA77AF6EE006A36EE476AF8EED1
:1011F800007A27EE277A66EE266A84E7DFED097A19
:1012080037EEC77ADDE7B0EE677A3DE7F0EE407A71
:1012180024E7B0EE677AC2E7F0EE477AAAE700BFA4
:1012280027D4D236DB0F4940DB0FC940E4CB164147
:10123800DB0F49C0E4CB16C1DB0FC93FDB0FC9BFC9
:1012480092E741B99730083C15A82ABEF304353F08
:101258000000008070B406688E4217D90139751EE7
:10126800002311F8014F0822634013F0800F4FEA62
:10127800430318BF83F0D503013ADBB2F5D18D42A1
:10128800EFD1721C0260337070BC70470023F8E71E
:1012980010B44C09012250F8243001F01F0102FA61
:1012A80001F10B4340F824305DF8044B704700BF50
:1012B8004B0901F01F0150F82320012303FA01F123
:1012C800114214BF18460020704700BF074A084B58
:1012D80010781B78074A834296BFC31AC3F180036C
:1012E8000020126818441044704700BFB44C002016
:1012F800314C0020F43A0020064A074B10781B783E
:1013080083428ABFC3F18003C01AC018C0F17F00AE
:10131800704700BFB44C0020314C002008B540F2A3
:10132800E93300E09BB10289013B12F0020F9BB246
:10133800F8D0017340F2E93300E043B10289013B80
:1013480012F0010F9BB2F8D0007BC0B208BD10F0BC
:10135800EFFAC0B208BD00BF38B504460D4600BF5D
:10136800806810F059F929466068FFF7D7FFA06830
:1013780010F058F900BF38BD38B500231C4620FAD4
:1013880003F2C3F11F0102F0010201338A40202B4E
:1013980044EA0204F3D1104D286810F03DF9210EFB
:1013A8000E48FFF7BBFFC4F307410C48FFF7B6FF31
:1013B800C4F307210948FFF7B1FFE1B20748FFF777
:1013C800ADFF02200CF004FB286810F02BF9022076
:1013D800BDE838400CF0FCBAA425002000300140DC
:1013E800F8B584894FF6FF764FF47A742BB311B3AE
:1013F8000F78013101E0B44217D00589013CAD07EF
:10140800A4B2F8D507734FF47A7402E0BCB2B442C0
:101418000BD00589ED0704F1FF37F7D5057BEDB251
:101428000AB115700132013BE0E710F081FA003093
:1014380018BF0120F8BDFF27DFE70120F8BD00BF76
:1014480030B5134C237883B01BB90120237003B047
:1014580030BD1049052200230D688DF804208DF851
:10146800053000BFA86810F0D7F86A4601A9022322
:101478006868FFF7B5FFA86810F0D4F800BF9DF8BA
:10148800013003F0010383F00100237003B030BD85
:10149800A54700206047002070B5064C0646256821
:1014A80003E023685B1BB34203D8FFF7C9FF00289A
:1014B800F7D070BD4C4700202DE9F04F89B0B2F14C
:1014C800000A02900491039340F3C5800B46002262
:1014D80001EB8A0153F8040B8B420244FAD1039BB7
:1014E8000592002B00F0AF80059B002B7CD05E4B53
:1014F800059A1B68DFF8889100920099DAB25118B2
:10150800B1F5807F8CBFC2F58072009A0192574A6C
:1015180092689A4240F28280554A117800220692D7
:101528008DF81C2002228DF81820002960D01A0E90
:101538008DF819200DF11A021C0C190A93701470F9
:1015480051700620FFF7A8FF0621D9F80000FFF721
:1015580003FF484A0123137000BFD9F80030986888
:1015680010F05AF8424BD9F800201B785068002B2D
:1015780006A90CBF042305230022FFF731FF00242E
:10158800049D029E019FA34629684FEA8408002211
:101598000B46013471B1B9422DD2D9F80000316837
:1015A8004068FFF71DFF2A68336813443360BF1A89
:1015B800C5F800B0A24505F1040506F10406E3D11B
:1015C800D9F80030986810F02DF800BF264B019923
:1015D80000981B68421A0092234A0B441360039A2E
:1015E8004AB3009A002A88D1059809B0BDE8F08F5F
:1015F8000DF11902A0E7029CD9F8003054F8081040
:10160800586800223B46FFF7EBFE54F808202B6889
:101618003A44DF1B44F808202F60D1E70598009C66
:101628001549164A001B0590059800230B70137086
:1016380009B0BDE8F08F059B009A9B1A05930598A1
:1016480009B0BDE8F08FFFF7FBFE00287FF44CAF30
:10165800039B0593C8E7039C1CB9FFF7F1FE0594AB
:10166800C2E700230593BFE7F43A00209C06002058
:10167800A4470020A5470020B44C0020314C00208E
:101688006047002070B5104D104E2B7831788B4292
:1016980084B016D00E4A03921A4402928CBF0C46AC
:1016A800CA1A04A98CBFC3F180020024012341F89F
:1016B800102D02A802220194FFF7FEFE00233370CA
:1016C8002B7004B070BD00BF314C0020B44C00201A
:1016D800344C002070B5194C194D2378297899425B
:1016E80084B027D0174A03921A44029234BF0E4698
:1016F800CA1A04A934BFC3F180020026002341F8A6
:10170800102D02A802220196FFF7D6FE237818446E
:10171800C0B203062B7848BF80F080008342207057
:1017280002D0002004B070BD002301202B7023706C
:1017380004B070BD012004B070BD00BF314C002062
:10174800B44C0020344C002010B50C4C45F2082055
:10175800FFF7A2FE20680621FFF7FEFD084B206870
:101768000122C7211A70FFF7F7FD06480649074A04
:10177800002303700B70136010BD00BF604700208A
:10178800A5470020B44C0020314C0020F43A00203A
:10179800F0B51F4C83B0277800234FF0030E009359
:1017A8000E4615468DF804308DF800E06FB3030E31
:1017B8008DF801300DF10203010C020A98701970BE
:1017C80006205A70FFF768FEE8B100BF114F3B686A
:1017D80098680FF021FF23783A68002B14BF05237F
:1017E8000423694650680022FFF7FAFD3B68324639
:1017F800002158682B46FFF7F3FD3B6898680FF007
:1018080011FF00BF284603B0F0BD0DF10103D3E777
:10181800A447002060470020F0B5124B9D6885B0B2
:101828000DB905B0F0BDED0A14D0002704AE7C193F
:101838006410E00210226946FFF7AAFF0F2809DDAD
:101848006B4653F8042B01320AD1B342F9D125462D
:10185800AF42ECDBFFF716FF034BED021D60E0E73C
:10186800671CF5E79C060020F43A0020F0B55B4BB6
:101878005B4A97B01968914200AF00F0A3805949BC
:10188800594A00234FF47000C1F888003B607B6020
:10189800136843F48033136003E03B68B3F5A04F4B
:1018A80009D0136803F400337B603B6801333B6065
:1018B8007B68002BF1D04C4B1B6813F4003318BF26
:1018C80001237B607B68012B52D0464C464B474A2C
:1018D800E260474A596A11605A6A42F080725A6255
:1018E8005A6942F4FC025A610025032207F10801F3
:1018F800012341F6FF764FF09040FD60BE603A73D9
:10190800BB7327F0ABFA4FF6FF7307F108013948AC
:10191800BB6027F0A3FA07F108013748374E27F0D4
:101928009DFA07F10801364827F098FA07F10801EF
:10193800344827F093FA07F10801334827F08EFA64
:1019480007F1080027F0E4FABB683049304AA1FBE8
:10195800031330499B0CF0204FF0070E5C370B60E7
:10196800566084F823009560C2F800E0BD46F0BDDB
:10197800294A1D4B122111605A685A605A685A60E8
:101988005A6842F480625A605A6822F47C125A609B
:101998005A6842F4E8125A601A6842F080721A6073
:1019A8001A689201FCD559680F4A21F00301596061
:1019B800596841F002015960536803F00C03082B81
:1019C800FAD182E700221A6062B6144B1B6883F3CF
:1019D8000888134B1B689847FEE700BFFC9F002050
:1019E800EFBEADDE00ED00E0001002400005FA0594
:1019F800405E002000040048000800483F1901002C
:101A0800000C0048001000480014004883DE1B4307
:101A180010E000E0504700200020024000D8FF1FDF
:101A280004D8FF1F70B50F4C0F4DC0EBC00004EB7E
:101A38008004686926693043686182B09209667BD0
:101A4800A1600025012101A863618DF804608DF86B
:101A580005208DF806508DF8071027F0C9F902B057
:101A680070BD00BF4C05002000100240074BC0EBC2
:101A7800C00030B403EB8000054C056963692B4353
:101A880063610176427630BC704700BF4C05002088
:101A9800001002402DE9F04F5E4C54F8204083B00E
:101AA800002C71D0A66D984691465B4B72682265F2
:101AB800A160236004F15E014FF4807304F5AF72F6
:101AC8006161A261E36023610746307E23F08CFBED
:101AD800F068A8B1514B00215A68904203F11C03E9
:101AE80000F0928001310C29F6D100207A1CD2B284
:101AF8000C21FFF7BBFF236DF26862632433E364B4
:101B0800B068D8B1454B00215A68904203F11C03D4
:101B180078D001310C29F7D100257A1CD2B20B21DB
:101B28002846FFF7A3FF2346F27E3D492846FFF7E4
:101B380079FF236DB268A2632833A36494F85D002B
:101B48000FF018F9054694F85C000FF013F918F037
:101B5800080F824696F819B01AD0CDB118F0110FB7
:101B68004FF00B0307F1010714BF4E213E21EF711F
:101B78005A46AB7128460FF0C1F918F0010F45D04D
:101B8800636B5BB3A36B4BB3204603B0BDE8F08F28
:101B980018F0010F0CBF4FF02E084FF04E0819F047
:101BA800020F09D045B10B227B1CAA71EB712846A4
:101BB8005A4641460FF0A2F919F0010FE0D0BAF1E8
:101BC800000FDDD001370C238AF807705A464146CA
:101BD8008AF8063050460FF091F9D1E7337FB27E8C
:101BE8008DF804209B090021012201A88DF80530F9
:101BF8008DF806108DF8072027F0FAF8204603B074
:101C0800BDE8F08FCDB288E7C8B26FE728460FF07D
:101C180003FDB5E778250020941503084C0500203E
:101C28000505000800B97047F0B595B0054623F0E2
:101C3800BBFD6E4EC368026832600446002B00F09C
:101C4800C38028460FF096F8694B186018B129220E
:101C580000238271C371227A664D2E210FF04EF94E
:101C680030680BF0F9FC23F0BFFA3068624A038849
:101C780023F001031B041B0C038014A91E232B80D3
:101C880001270F230025138021F84C7D2D23029373
:101C9800ADF80C50ADF80650ADF80E5023F032FDFB
:101CA800E379ADF8145060229907ADF816500695FF
:101CB800ADF81C50ADF81E50ADF82050ADF82250CC
:101CC800049200F1838013F0010F14BF0222002256
:101CD8004FF48073ADF81470ADF81C20ADF82030C7
:101CE800002304AA6179306806930BF00FF9306875
:101CF800617923F0E7FC3068436C43F400434364A4
:101D080003889BB243F080030380E3799B0768D57F
:101D18006179026A04238B4022EA03020262026AA2
:101D2800134303623268354F13889BB243F00103B3
:101D38001380207C00222921FFF798FE3049207C5F
:101D480000236022FFF76EFEE068386026F0BCFFD3
:101D5800386803684FF6FE721340036026F0B4FF3C
:101D680009A826F083FF33686279264938680A9102
:101D780034331344099380221023002509A940F223
:101D88002A3E0E920B934FF400724FF400530D95B8
:101D98001095139511950F921293ADF830E026F037
:101DA80073FF627933680C2A98BF1749D86898BFBF
:101DB80031F812503A6815490543DD60136801206F
:101DC80043F002031360087015B0F0BD13F0010F63
:101DD80014BF08222A460423ADF81E20ADF8163099
:101DE8007EE70122617926F07FFE9BE79430002090
:101DF800601600208A3000208830002090300020B3
:101E0800C904000810500020203F03088C3000202F
:101E18000348D0F83C3113B100F59A701847704761
:101E28004C0500200348D0F8203113B100F58C7020
:101E3800184770474C0500200348D0F804310BB10F
:101E4800FC301847704700BF4C0500200348D0F805
:101E5800E8300BB1E0301847704700BF4C05002050
:101E68000348D0F8CC300BB1C4301847704700BFD6
:101E78004C0500200348D0F8B0300BB1A830184703
:101E8800704700BF4C0500200348D0F894300BB1D0
:101E98008C301847704700BF4C0500200248836FFC
:101EA8000BB17030184770474C0500200248C36DCD
:101EB8000BB15430184770474C0500200248036C9A
:101EC8000BB13830184770474C0500200248436A68
:101ED8000BB11C30184770474C0500200248836836
:101EE80003B11847704700BF4C050020F8B5574CA0
:101EF8000601A7190546387A23F076F93B7A03F0EC
:101F08001F015B090122022B02FA01F278D0032B90
:101F180071D0012B67D0A319013518790EF02AFF6B
:101F2800EDB2074610B11223C5718371A319587910
:101F38000EF020FF10B11323C5718371A31998798E
:101F48000EF018FF10B11423C5718371A5190E2165
:101F5800EA7938460EF0D2FF68790EF00BFFEA797D
:101F68000E210EF0CBFFA8790EF004FFEA790E21BE
:101F78000EF0C4FFA359364A934251D0354A9342D2
:101F880059D0354A934240D03444227B002A2FD17D
:101F9800012002249A8822F480521204120C9A809A
:101FA800998889B241F4805199801A8802F4415283
:101FB80042F44572024322431A809A8822F47062DE
:101FC8001204120C42F4E0629A809A8B22F40062A6
:101FD8001204120C07219A8319821A8892B242F0CD
:101FE80040021A80F8BD1D4B996A0A439A6292E72B
:101FF80000200446CEE7194B19690A431A618AE79B
:10200800164BD9680A43DA6085E702F5EA321169A6
:1020180041F400411161116921F400411161B3E7F4
:1020280002F56042D16841F48051D160D16821F451
:102038008051D160A8E702F5EC32116941F4804182
:102048001161116921F4804111619DE774470020F5
:102058000030014000380040003C004000100240C1
:10206800F0B53E4C059D00EB800004EB80046468ED
:10207800002C71D03A4E49004FF42040CFB2706026
:10208800A169090454D46068DFF8E0E047F49031AE
:1020980000EA0E0001434FF420406160706003E0E5
:1020A800411E002848D00846A1698907F8D54FF491
:1020B8002040A262706003E0421E00283CD0104617
:1020C800A2695206F8D5274A6168DFF8A0E0706077
:1020D80042EA0342174301EA0E0217436760C3B19D
:1020E800013BDBB201332B44A0694FF4204210F0CE
:1020F800040002F1FF3207D1511C26D0A06910F06C
:10210800040002F1FF32F7D0626A05F8012B9D4204
:10211800EAD14FF42040706002E0431E60B11846D7
:10212800A3699B06F9D520237060E3610120F0BD07
:10213800411E08B10846A3E70B4A138801339BB236
:102148004FF0FF3113807160F0BD074972600B8852
:1021580001339BB20B80F0BD2046F0BDEC46002059
:10216800601600200024000264350020009800FC5E
:10217800F0B5037C012B85B0044663D0022B67D1F0
:10218800836913B11A689B881385606940F2E93343
:1021980001E0002B6CD00289013B12F0020F9BB2C8
:1021A800F7D0C323037340F2E93301E0002B5FD07B
:1021B8000289013B12F0010F9BB2F7D0037B6069E3
:1021C8004FF0060E838902AE4FF47A734FF6FF7113
:1021D800FF2703E0013B9BB28B423CD00289950765
:1021E800F8D507734FF47A7302E0ABB28B4232D062
:1021F8000289D20703F1FF35F7D5027BD2B20EB1BF
:1022080032700136BEF1010EE8D1A36913B11A6824
:102218009B8893619DF80C009DF808609DF8091053
:102228009DF80A509DF80B209DF80D3041EA0621D3
:1022380043EA002342EA0522012021876287A38717
:1022480005B0F0BD90F91400431C01D0022805DD4B
:10225800002005B0F0BD0FF06BFBD6E702AB617D47
:10226800009343220623FFF7FBFE0028D2D1EFE7B5
:102278000FF05EFBA3E700BFF0B5037A012B85B032
:10228800044663D0022B67D1036913B11A689B888F
:102298001385E06840F2E93301E0002B6CD0028935
:1022A800013B12F0020F9BB2F7D0BB23037340F23D
:1022B800E93301E0002B5FD00289013B12F0010FE6
:1022C8009BB2F7D0037BE0684FF0060E838902AE1D
:1022D8004FF47A734FF6FF71FF2703E0013B9BB27F
:1022E8008B423CD002899507F8D507734FF47A736F
:1022F80002E0ABB28B4232D00289D20703F1FF353C
:10230800F7D5027BD2B20EB132700136BEF1010EA2
:10231800E8D1236913B11A689B8893619DF80C0072
:102328009DF808609DF809109DF80A509DF80B204B
:102338009DF80D3041EA062143EA002342EA0522CE
:102348000120E1822283638305B0F0BD90F90C007F
:10235800431C01D0022805DD002005B0F0BD0FF0B8
:10236800E7FAD6E702AB617B00933B220623FFF72F
:1023780077FE0028D2D1EFE70FF0DAFAA3E700BF23
:10238800B0F1FF3F56D0022854DCF0B4324C00EBD9
:10239800800004EB80004468002C5BD02F4E49007D
:1023A8004FF42040CDB27060A169090444D460683C
:1023B8002B4F45F08071384041F4903101434FF480
:1023C80020406160706003E0411E002838D0084654
:1023D800A1698F07F8D54FF42040A262706002E02F
:1023E800421E68B31046A2691106F9D562681C49F5
:1023F80045F0007545F480350A4015434FF42040F8
:102408006560706002E0421ED0B11046A269920772
:10241800F9D54FF42040A362706002E0431E78B102
:102428001846A3699B06F9D520237060E361012053
:10243800F0BC704700207047411E08B10846B3E75A
:10244800084A138801339BB24FF0FF311380716043
:10245800F0BC70472046FBE7EC46002060160020E1
:10246800009800FC643500202DE9F04F87B090F803
:1024780055300190002B40F0E483019A137C012B26
:1024880000F07B84022B44D1936913B11A689B88AE
:102498001385019B586940F2E93302E0002B00F0F4
:1024A800E2840289013B12F0020F9BB2F6D06B2343
:1024B800037340F2E93302E0002B00F0D484028970
:1024C800013B12F0010F9BB2F6D0037B019B5869C8
:1024D80040F2E93302E0002B00F0C1840289013B9D
:1024E80012F0020F9BB2F6D08023037340F2E93357
:1024F80002E0002B00F0B3840289013B12F0010FC7
:102508009BB2F6D0037B019B9B6913B11A689B8829
:1025180093616423A94CAA4DDFF8ACA2A948DFF85F
:10252800ACC24FF010084FF47A779E46DAF80430C0
:10253800C3F30803002B40F04E82EFF31183002B06
:1025480040F049822168826800BF23689942F9D126
:102558002E6807FB06F39B1AB3FBF6F307FB013162
:1025680001260091DAF80430C3F30803002B40F089
:102578001582EFF31183002B40F0108223688168E5
:1025880000BF22689342F9D1D5F800B007FB0BF2DF
:10259800521AB2FBFBF207FB0323009A9B1AB3F50E
:1025A8007A7FDFD3BEF1010EC0D1019A137C012BD3
:1025B80051D0022B58D1936913B11A689B8813859F
:1025C800019B586940F2E93302E0002B00F0608477
:1025D8000289013B12F0020F9BB2F6D06B23037302
:1025E80040F2E93302E0002B00F052840289013BFB
:1025F80012F0010F9BB2F6D0037B019B586940F2A1
:10260800E93302E0002B00F032840289013B12F02A
:10261800020F9BB2F6D00323037340F2E93302E0C2
:10262800002B00F024840289013B12F0010F9BB2B9
:10263800F6D0037B01988269002A00F01F84136892
:1026480092889A61017C90F85070012900F0DF812E
:10265800022955D114E0164603236B22717D96F9A1
:102668001400FFF78DFE337C0199012B91F850700F
:1026780000F0CD81022B43D18A6912B11368928888
:102688001A85019B40F2E932586902E0002A00F0FD
:1026980019840389013A13F0020F92B2F6D0192374
:1026A800037340F2E93202E0002A00F00B84038948
:1026B800013A13F0010F92B2F6D0037B019B40F26E
:1026C800E932586902E0002A00F0F9830389013AE7
:1026D80013F0020F92B2F6D0077340F2E93302E02A
:1026E800002B00F0EC830289013B12F0010F9BB232
:1026F800F6D0037B019B9B6913B11A689B88936191
:102708000F23DFF8C4A02F48DFF8C0C04FF010082F
:102718004FF47A779E46DAF80430C3F30803002BA7
:1027280040F07382EFF31183002B40F06E82216832
:10273800826800BF23689942F9D12E6807FB06F327
:102748009B1AB3FBF6F307FB013101260091DAF877
:102758000430C3F30803002B40F03A82EFF31183EF
:10276800002B40F035822368816800BF22689342BD
:10277800F9D1D5F800B007FB0BF2521AB2FBFBF205
:1027880007FB0323009A9B1AB3F57A7FDFD3BEF1C8
:10279800010EC0D101990A7C91F84E40012A00F03F
:1027A8009F81022A40F0A5818B6913B11A689B8822
:1027B8001385019B40F2E93258690CE04C47002030
:1027C8005047002010E000E000ED00E048470020FE
:1027D800002A00F071830389013A13F0020F92B2C4
:1027E800F6D01A23037340F2E93202E0002A00F01F
:1027F80063830389013A13F0010F92B2F6D0037B89
:10280800019B40F2E932586902E0002A00F0448353
:102818000389013A13F0020F92B2F6D0047340F222
:10282800E93302E0002B00F037830289013B12F004
:10283800010F9BB2F6D0037B01988269002A00F051
:102848003283136891889961027C012A00F09F8283
:10285800022A00F05981012A00F0E280022A40F0A1
:10286800E880019B9A691AB1136891881985019BC0
:10287800586940F2E93302E0002B00F0ED8202894A
:10288800013B12F0020F9BB2F6D01C23037340F2F7
:10289800E93302E0002B00F0DF820289013B12F0ED
:1028A800010F9BB2F6D0037B019B586940F2E933D4
:1028B80002E0002B00F0C0820289013B12F0020FF7
:1028C8009BB2F6D01823037340F2E93302E0002BE1
:1028D80000F0B2820289013B12F0010F9BB2F6D0E0
:1028E800037B01988269002A00F0AD821368918801
:1028F8009961027C012A00F05481022A00F0A48028
:10290800012A00F05A81022A45D1019B9A6912B125
:10291800136892881A85019B586940F2E93302E0EE
:10292800002B00F086820289013B12F0020F9BB255
:10293800F6D03823037340F2E93302E0002B00F0AD
:1029480078820289013B12F0010F9BB2F6D0037B1B
:10295800019B586940F2E93302E0002B00F06682DF
:102968000289013B12F0020F9BB2F6D001230373D8
:1029780040F2E93302E0002B00F058820289013B63
:1029880012F0010F9BB2F6D0037B019B9B6913B138
:102998001A689B88936107B0BDE8F08FEFF311893F
:1029A80088F3128881680368DB0344BFCCF80060B1
:1029B80081682368DCF800205FFA89F989F31188B7
:1029C800D5F800901A4407FB09F35B1AB3FBF9F337
:1029D80007FB0233E1E5EFF3118288F3128886687A
:1029E8000368D90303D50123CCF80030866823682F
:1029F800DCF80010D2B282F311882A68194407FB68
:102A080002F39B1BB3FBF2F307FB0131A8E5019826
:102A18003B46417D90F914001922FFF7B1FC6FE69F
:102A2800019C1C221823617D94F91400FFF7A8FC6F
:102A3800227C012A00F0B580022A7FF461AF019B55
:102A48009A691AB1136891881985019B586940F2EF
:102A5800E93302E0002B00F0E6810289013B12F025
:102A6800020F9BB2F6D03723037340F2E93302E03A
:102A7800002B00F0D8810289013B12F0010F9BB2B4
:102A8800F6D0037B019B586940F2E93302E0002B42
:102A980000F0B8810289013B12F0020F9BB2F6D018
:102AA8000223037340F2E93302E0002B00F0AA810D
:102AB8000289013B12F0010F9BB2F6D00199037B0A
:102AC8008A69002A00F0A581136892889A61097CB6
:102AD800012972D002293FF41DAF07B0BDE8F08F7D
:102AE8002346019C1A22617D94F91400FFF748FCE3
:102AF800227C012A00F04B81022A7FF4ACAE019BB4
:102B08009A691AB1136891881985019B586940F22E
:102B1800E93302E0002B00F072810289013B12F0D8
:102B2800020F9BB2F6D01B23037340F2E93302E095
:102B3800002B00F064810289013B12F0010F9BB267
:102B4800F6D0037B019B586940F2E93302E0002B81
:102B580000F045810289013B12F0020F9BB2F6D0CA
:102B68001823037340F2E93302E0002B00F03781A9
:102B78000289013B12F0010F9BB2F6D0037B01984A
:102B88008269002A00F03281136891889961027C79
:102B9800012A3FF445AF022A3FF468AE012A7FF4C8
:102BA8004BAF019C37220223617D94F91400FFF793
:102BB800E7FB227C012A7FF4A6AE01980123417D20
:102BC80090F914003822FFF7DBFB07B0BDE8F08F5F
:102BD800EFF3118988F3128881680368DB0344BF27
:102BE800CCF8006081682368DCF800205FFA89F976
:102BF80089F31188D5F800901A4407FB09F35B1A8A
:102C0800B3FBF9F307FB0233BCE5EFF3118288F35A
:102C1800128886680368D90303D50123CCF80030ED
:102C280086682368DCF80010D2B282F311882A681B
:102C3800194407FB02F39B1BB3FBF2F307FB0131BB
:102C480083E51D09013D052D03F00F0300F2C28045
:102C5800A34A32F8150040FA03F2D40740F1BA80CB
:102C6800012404FA03F3013B18402DF085F89D4B2D
:102C7800DFF88C825F5D074418EBC70500F0AA8077
:102C880020220023AA71EB7158F83700964A00F108
:102C980038439B0AD25C02F01F035209022A04FA45
:102CA80003F300F01881032A00F01081A24200F01B
:102CB8008C80AB88049304A90024059426F0CEF8F0
:102CC800AB88019E894AF260B3FA83F2C2F11F020F
:102CD800511C3FD0D1B201F0FC0303F1804303F54E
:102CE800803301F00301D3F808E088004FF00F0C9F
:102CF80058F83710DFF80C820CFA00F72EEA0707AD
:102D080006F10C0E48F822E09F60D3F808C0784F0F
:102D1800DFF8F4E1C1F38721814041EA0C014FF06B
:102D28000109996009FA02FCB918CEF800C0082315
:102D380004A8049291F88C808DF815308DF81690BF
:102D48008DF8144023F0C4F96A4A12F80830F02BC1
:102D580027DCAB88B3FA83F3C3F11F03581C3FF495
:102D68008CAB012202FA03F363490A681343019A00
:102D78000B60137C012B7FF485AB10468023417DCB
:102D880090F914006B22FFF7FBFAFFF7C2BB019C16
:102D98001B221823617D94F91400FFF7F1FA227CB5
:102DA80059E507EB0803F02193F89C308DF80C30B7
:102DB80003A803238DF80E408DF80F9002F8081031
:102DC8008DF80D3026F014F8C3E74C4A51690B43CF
:102DD80053616EE7019A454BD3600123C4E70EF0B7
:102DE800A7FD01988269002A7FF4CEAE027C012AF1
:102DF80003463FF415AE022A3FF43AAD19E60EF049
:102E080097FD9FE60EF094FD01998A69002A7FF4E8
:102E18005BAE0B7C012B3FF4D0AE022B3FF47BADB5
:102E280007B0BDE8F08F0EF083FD2BE60EF080FDB5
:102E3800ABE50EF07DFD8BE50EF07AFD0198826919
:102E4800002A7FF453AD027C012A03463FF4A9AE61
:102E5800022A3FF4FBAD53E50EF06AFD24E50EF0BF
:102E680067FDFFF750BB0EF063FDFFF72FBB0EF0B9
:102E78005FFD01988269002A7FF4E1AB037C90F83A
:102E88005070012B3FF4C3AD022B3FF4FAAB37E48B
:102E98000EF04EFDFFF7B1BB0EF04AFD01988269B6
:102EA800002A7FF4CEAC027C012A03463FF46FAFC0
:102EB800022A3FF42BAECEE40EF03AFDA0E40EF069
:102EC80037FD17E40EF034FDFFF7F8BB0B4AD16964
:102ED8000B43D361EDE6094A91690B439361E8E638
:102EE800A43B0308B03B0308D43A03082D040008A8
:102EF800301503083C1D002000040140001002406A
:102F0800CC490020FC1C0020140401401749184B30
:102F1800184A194810B4D1F8884044F47004C1F82C
:102F280088401C6844F001041C605C6822405A60B8
:102F38001A6822F0847222F480321A601A6822F425
:102F480080221A605A6822F4FE025A60DA6A22F075
:102F58000F02DA621A6B002410404FF00062186307
:102F68009C608A605DF8044B704700BF00ED00E08C
:102F7800001002400CC07FF8CCFC00FF2DE9F04F98
:102F880095B0B0F908500D81EDB2442D00AF0C4654
:102F9800904600F01684064632D9812D00F05D83F4
:102FA80000F28680542D00F0B38040F2BD806E2D73
:102FB80000F0D583802D40F0B9806A4B1D780B3D19
:102FC80015F0FF0514D0DFF8C4E100220A262168B5
:102FD800BEF80030481C20600E702168FF2B02F1FB
:102FE8000102A8BFFF23481CAA4220600B70EEDB39
:102FF80001252B46284654376381BD46BDE8F08F2E
:10300800052D00F0CC831FD8022D79D040F204831F
:10301800032D00F09B83042D40F088805249204600
:103028002A46FDF739FE00212046FDF765FE226895
:103038000021531C0125236028462B465437117064
:103048006381BD46BDE8F08F242D57D040F29A82A7
:10305800282D00F03D83382D68D10A68434B01259F
:10306800511C2160157022680521501920601170CB
:1030780022680A2150192060117022680021501915
:103088002060117022681978501920601170226828
:103098005978501920601170226899785319236063
:1030A8002B461170284654376381BD46BDE8F08F22
:1030B800A02D11D040F28582B82D00F04583FE2D59
:1030C80034D12B4D05F1080635F8021B2046FDF7D3
:1030D80013FEB542F8D18BE7264B08461968FDF771
:1030E800F3FD254B20461968FDF7EEFD234B1968C3
:1030F80020460125FDF7E8FD2B467BE7204BF6E748
:103108000422204920460125FDF7C6FD2B46C9E7C4
:103118000B6800215A1C2260197022680125531976
:1031280023602B461170BDE7522D80D021462846DA
:103138000EF066FD034600287FF45AAF742D00F0A8
:103148007E82772D24D13268716891421EBF531C4C
:10315800336011780C4A08BF1946204615F0A0FEC6
:1031680046E700BFDE4C002076540020DF2E00200A
:10317800344D0020ACF7FF1FB0F7FF1FB4F7FF1F57
:103188006430002094420308697E0108941D0020E1
:10319800F52D01F0AD82472D00F04083292D3268CE
:1031A80001F06682392D01F05082212D01F02D8227
:1031B80070680B3D811AEF2D00F28E840FF2040E19
:1031C8005EF825F091400008E13A0008E13A00086D
:1031D800E13A0008E13A0008E13A0008E13A00085B
:1031E800E13A0008E13A0008E13A0008E13A00084B
:1031F800E13A0008E13A0008E13A0008E13A00083B
:10320800E13A0008E13A0008E13A0008E13A00082A
:10321800E13A0008E13A0008E13A0008E13A00081A
:10322800E13A00081D400008E13A0008FB3F0008A9
:10323800E13A0008D13F0008E13A0008E13A000805
:10324800E13A000897410008E13A000821410008E6
:10325800E13A0008EF400008E13A0008C9400008D8
:10326800E13A0008BF3F0008E13A0008673F00085C
:10327800E13A0008153F0008E13A0008E13A000881
:10328800E13A0008E13A0008F92F0008E13A00089D
:103298009B3E0008E13A0008E13A0008174400089C
:1032A800E13A0008BD430008E13A0008E13A0008A5
:1032B800E13A0008E13A0008B1430008E13A0008A1
:1032C800E13A0008E13A000871430008E13A0008D1
:1032D80023430008E13A0008E13A0008E342000805
:1032E800E13A0008E13A0008E13A0008E13A00084A
:1032F800E13A0008E13A0008E13A0008754200089E
:10330800E13A0008BF410008E13A0008DF4400083C
:10331800E13A000831440008E13A0008D1450008C4
:103328007D3E0008613E0008E13A0008E13A0008E5
:10333800E13A0008E13A0008E13A0008E13A0008F9
:10334800E13A0008E13A0008E13A0008E13A0008E9
:10335800E13A0008E13A0008E13A0008E13A0008D9
:10336800E13A0008E13A0008E13A0008E13A0008C9
:10337800E13A0008E13A0008E13A0008E13A0008B9
:10338800E13A0008E13A0008E13A0008E13A0008A9
:10339800E13A0008E13A0008E13A0008E13A000899
:1033A800E13A0008E13A0008E13A0008E13A000889
:1033B800E13A0008E13A0008E13A0008E13A000879
:1033C800E13A0008E13A0008E13A0008E13A000869
:1033D800E13A0008E13A0008E13A0008E13A000859
:1033E800E13A0008E13A0008E13A0008E13A000849
:1033F800E13A0008E13A0008E13A0008E13A000839
:10340800E13A0008E13A0008E13A0008E13A000828
:10341800E13A0008E13A0008E13A0008E13A000818
:10342800E13A0008E13A0008E13A0008E13A000808
:10343800E13A0008E13A0008E13A0008E13A0008F8
:10344800E13A0008E13A0008E13A0008E13A0008E8
:10345800E13A0008E13A0008E13A0008E13A0008D8
:10346800E13A0008E13A0008E13A0008E13A0008C8
:10347800E13A0008373E0008E13A00081B3E000820
:10348800F13D0008E13A0008E13A0008E13A000895
:10349800E13A0008E13A0008E13A0008E13A000898
:1034A800E13A0008E13A0008E13A0008E13A000888
:1034B800E13A0008E13A0008773D0008E13A0008DF
:1034C8003F3D0008E13A00089D3C0008833C0008A5
:1034D800D53D0008E13A0008693C0008E13A0008D7
:1034E800413C0008E13A0008E13B0008E13A0008E5
:1034F800893B0008E13A0008E13A00082D3B000842
:10350800FF3A0008EB3A0008B93B0008C33A000844
:10351800993A0008E13A0008E13A0008E13A00085F
:10352800E13A0008E13A0008E13A0008E13A000807
:10353800E13A0008E13A0008E13A0008E13A0008F7
:10354800E13A0008E13A0008E13A0008E13A0008E7
:10355800E13A0008793A0008E13A0008E13A00083F
:10356800213A0008E13A0008E13A0008E13A000887
:10357800BD390008E13A0008E13A0008E13A0008DC
:10358800A3390008202D7FF4D1AD0B68914D591C4B
:103598006A7821601A7023682A78591C21601A7089
:1035A8002368AA78591C21601A7029892046FDF7DA
:1035B800A3FB23686A79591C21601A702268A979CB
:1035C80037E5822D7FF4B2AD0B68834A834D1178BD
:1035D800804A581C2060197011892046FDF78CFB21
:1035E8007F4B22681B88FF2B02F10101A8BFFF2334
:1035F80021601370A96881F3100189B22046FDF794
:103608007BFB296801F30F0189B22046FDF774FBA3
:10361800744B226819780CE5012D7FF487AD0B688F
:103628000022591C21601A7023685A1C22601D70E0
:1036380022682521531C23602B46117032E532681D
:10364800716891421EBF531C33601178664A08BFE7
:103658001946204615F024FCCAE4644B1E780A3E3D
:1036680016F0FF063FF4C4AC614BDFF8A8811E4496
:1036780003F101090A2314E0502B00F0B987002553
:1036880029462268501C206020461370FDF734FB41
:1036980029462046FDF730FBB1453FF4A9AC19F89F
:1036A800013B0A2BE8D1534A9568116805EB85055B
:1036B8004FF6FF726D009542A8BF15469142A8BF0C
:1036C800114625EAE57521EAE171ADB289B2D8E77C
:1036D8000B68DFF84491484E591C022221601A7089
:1036E80023684FF006085A1C226083F8008023687C
:1036F8000A22591C21601A70236801255A19226070
:103708001D70B9F800102046FDF7F6FAB9F8021056
:103718002046FDF7F1FA23685A19226083F80080E1
:1037280023685022591921601A70236800225919F8
:1037380021601A7031882046FDF7DEFA718820462C
:10374800FDF7DAFA2B46ADE42C4BD0E40B685A1C93
:103758000A601D700B685A1C0A601D7067E4204BD4
:103768000A681B881D4DFF2BA8BFFF23511C216031
:103778001370A96881F3100189B22046FDF7BCFADD
:103788001F4B20461988FDF7B7FA296801F30F0186
:1037980089B220460125FDF7AFFA2B4682E40B22B9
:1037A80018492046FDF778FA082217492046FDF700
:1037B80073FA0125072215492046FDF76DFA2B46B5
:1037C80070E4002A3FF414AC114B136001252B461A
:1037D80068E400BF14450020564D002054430020E3
:1037E800404D0020134F0020197F0108DE4C0020B7
:1037F800D4150308501D0020841D00201837002010
:10380800104F00209C420308A8420308B442030852
:10381800DD1B0108881D0020B83A00207268356851
:103828007B623046551BFDF70DFA052D38627B6A21
:1038380000F2DD878026B346012594E80600521A77
:10384800103AB242B8BF1FFA82FBC14A396A92687D
:103858003A61521A9345396A7B622046FA6088BFFA
:103868001FFA82FBFDF730FA7B6A002B00F09D8778
:10387800002D40F016872368C7F800D05D71C0B0EE
:103888000533C7F808D0FB61BBF1000F01F0608079
:103898003B6A3A69934281F05780AA463E6A7D6244
:1038A8007C6080255446FB681C1BA94BB4F5807FBF
:1038B80028BF4FF480749B6832199A4288BF9C1BBA
:1038C800FDF7E0FE2246BC6830462146FDF760FF62
:1038D800F969B86104EB000C0B787B61644530D260
:1038E800DFF890920CF1FF3C04F1FF3E1EF8013F17
:1038F80009EB830219F823405688FCB100234FF4E2
:10390800004204F1FF3816424FEA520202D008780A
:10391800284308706D0806D10AF1010A4D701FFA94
:103928008AFA01318025D34505D8E645C0F0668678
:10393800984500F3638601339C42E4D1E645D5D12E
:10394800F9617B6ABA6913449BB2DA457B6206D295
:103958007B6A3A6A1C46D6183B699E42A3D37C68A8
:10396800802D1CBF0AF101031FFA83FA0AF1020134
:1039780089B22046FDF7C0F92368796A01255A19EA
:10398800226020461D70FDF7B7F923685344236071
:103998002B46D7F800D0FFF785BB6E4B1B78DB07AB
:1039A80000F19A80012508F0DFFC08F0B9FE2B46EB
:1039B800FFF778BB3046FDF75DF93368B8851A46DE
:1039C800591C316012F8021B326087F82E105A78A1
:1039D80087F82F20DA1C32609A7887F830201A1D71
:1039E8003260DA7887F831205A1D32601B7987F8FF
:1039F800323007F12C000023BB86FDF793F8564AB6
:103A0800564B1268801A4FF0010561F10001C3E9B5
:103A180004012B46FFF746BB531C336013780F2B6A
:103A28005AD8911C3160C3EBC3034D495078C85430
:103A3800D01C30600B4491785970111D3160D178D9
:103A48009970511D31601179D970911D316051798A
:103A58001971D11D31609179597102F108013160F4
:103A6800D2799A7101251FF0A5FB2B46FFF71ABBE7
:103A78003046FDF7FFF8DFF80081A8F80E00304661
:103A8800FDF7F8F80125A8F80C002B46FFF70ABB4C
:103A98003046FDF7EFF8DFF8E480A8F8100030466C
:103AA800FDF7E8F8A8F812003046FDF7E3F801251D
:103AB800A8F814002B46FFF7F5BA1346511C3160DD
:103AC80013F8020B3360D31C51783360927826F0D8
:103AD80033FD00287FF48CAA4FF0FF352B46FFF703
:103AE800E1BA204B204918684E2201252CF0B2FB80
:103AF8002B46FFF7D7BA1146531C33601B4B11F8FE
:103B0800020B1870316051785970D11C316092786D
:103B18009A703046FDF7AEF8154B0125D8802B4634
:103B2800FFF7C0BA3046FDF7A5F8DFF84480A8F8DB
:103B380000003046FDF79EF8A8F802003046FDF771
:103B480099F80125A8F804002B46FFF7ABBA00BF87
:103B58009C060020C04C00204C470020A0160020E6
:103B68002C3600207C450020341F0308C03A002072
:103B780064280020D8150308C83A00203C5A0020C1
:103B8800DFF8749399F80030002B3FF431AADFF87E
:103B98006C8300253046FDF76DF811F0DFFD99F8CC
:103BA8000030A8EC010A01359D42F3DBFFF720BA8B
:103BB8001346511C3160C24913F8020B0870336078
:103BC800C04953788B70D31C3360BF4B92789A707E
:103BD80001252B46FFF766BA0D297FF47DAF531CEC
:103BE80033601578072D3FF677AFDFF8149330462A
:103BF8004FF00C08FDF73EF808FB05F809EB08053F
:103C0800A8803046FDF736F8E8803046FDF732F8F0
:103C1800336828811A46591C316012F8021BA972B0
:103C280032605B78EB723046FDF70CF8012549F8F5
:103C380008002B46FFF736BA531C33601078060687
:103C480000F17786A14B1B78DD073FF5D1A9032842
:103C580028BF0020012508F06BFB2B46FFF722BA8E
:103C68009A4B1B78D8073FF5C3A9012509F042F9FB
:103C780008F056FD2B46FFF715BA944B1B78D90769
:103C88003FF5B6A9924B4FF4C87201251A802B460E
:103C9800FFF708BA09297FF71FAFDFF868821346D4
:103CA800511CD8F80050316013F8021B297033609A
:103CB8005378AB70D31C33609378642B02F1040102
:103CC800A8BF64236B713160D378642B02F10501BE
:103CD800A8BF6423AB7131601379EB71931D336016
:103CE8005379642B02F10701A8BF64232B7231605A
:103CF8009379EB7002F108033360D3792B71304666
:103D0800FCF7B8FF726833686881D11A00290CDDA6
:103D1800591CD8F800003160521A002A19784172EB
:103D280003DD9A1C32605B78437001252AF05CFD44
:103D38002B46FFF7B7B9674B1868D31C01462132E9
:103D48009D1E356013F8035C0D705D1E356013F819
:103D5800025C4D70336013F8015C8D70033393423D
:103D680001F10301ECD111F0C9FBFFF741B9C1F32F
:103D78004705122D3FF6B0AEC5B107F1500307F164
:103D88002A0903EB450AC846AAF1260A3046FCF779
:103D980071FF28F8020FC245F8D14F4B39F8022FAE
:103DA80023F8022FC145F9D1112D09D84B4A6B00D0
:103DB800023B13440021223223F8021F9342FBD115
:103DC800474A01231D461370FFF76CB93F4B1B7818
:103DD800DA073FF50DA9434A1378012543F0040398
:103DE80013702B46FFF75EB9531C3F4833600178C8
:103DF8001378002940F0D185042202703B4A9B00C9
:103E0800138009F099FD3A4B012598612B46FFF77D
:103E180049B9DFF8F48000233046C8F80030FCF7D1
:103E280011FF0125C8F800002B46FFF73BB91346E0
:103E3800511C316013F8025B3360D31C5078336037
:103E48009178002D00F0D085012D7FF4D1A80FF0D6
:103E58001DFB2B46FFF726B9531C33601378002B44
:103E680000F0A0854FF4004001250EF0DBFE2B4644
:103E7800FFF718B9154B1B7813F001017FF42CAE2E
:103E8800531C3360107801250FF042FA2B46FFF7D8
:103E980009B91346511C3160164913F8025B8D703D
:103EA800336055784D7083423FF4A2A8D31C336029
:103EB8000F4B92781A7201252B46FFF7F3B800BF13
:103EC800A0550020C83A0020D83A0020C04C002055
:103ED800E26A00207C45002046320020483200205B
:103EE8006C32002020390020D23C0020104F0020E6
:103EF800A0160020E83A0020DE4C002040380020C0
:103F08006C35002080450020183700200723B1FBBE
:103F1800F3F3C3EBC305491B7FF4DEADDBB203F15A
:103F2800FF395FFA89F9002B3FF462A8DFF808A38C
:103F380009F101090D46531C336092F90010BE4B7C
:103F48004FF0000893F902208A4203F1080300F0B9
:103F58007B8408F10108B8F1060FF3D1BCE5531CC6
:103F6800336013780E2B3FF6B7AD911C316055784E
:103F7800032D3FF6B1ADB148062101FB03F143180B
:103F880002F1030E5D71C6F800E095784554111DE5
:103F98003160D1785970511D316011799970911D36
:103FA80031605179D970D11D316092791A7101252A
:103FB8002B46FFF777B8531C3360A14B12785A751C
:103FC80001252B46FFF76EB83046FCF753FEDFF8A5
:103FD8009082C8F800003046FCF74CFEC8F8040090
:103FE8003046FCF747FE0125C8F808002B46FFF7C6
:103FF80059B8DFF870820023C8F800303046FCF763
:1040080021FED8F8003001250343C8F800302B46BC
:10401800FFF748B8511C316015783B62132D3FF605
:104028005BAD911C316050787A6214F073FF002800
:104038003FF452AD7A6A8349007801F82500D01C14
:10404800306001EB850590786870101D3060D0787D
:10405800A870501D30601279EA7001F150003B6A77
:1040680002E00431884207D00A78002AF9D18D7815
:10407800CA789542F5D20123734A83F001030125DA
:1040880013702B46FFF70EB8704810294FF0000246
:104098000B4628BF1023026042608260C26002742F
:1040A800002B3EF4A5AF3268411E13440132326042
:1040B80012F8010C01F8010F9A42F7D1FEF798BFE8
:1040C800531C336015781F2D3FF606AD05297FF484
:1040D80003AD3046FCF7B6FD5D4B43F8250026F0EE
:1040E8009DFAFEF785BF5A4D05F140083046FCF7AA
:1040F800C1FD3368A5F88000591C1A46316012F8D2
:10410800021B85F8821032605B7885F883300435AD
:10411800A845EBD1FEF76CBF531C494D33601378AB
:104128002B723046FCF7A6FDA8833046FCF7A2FDAB
:1041380028833046FCF79EFD32686883531C336041
:104148001278EA747268D31A032B00F30684336872
:10415800D11A05290EDD5A1C32601B78EB723046E5
:10416800FCF770FD3368E8605A1C32601B782B74CA
:1041780033687268D21A002A7EF73AAF5A1C326046
:104188001B7885F8213001252B46FEF78BBF531C81
:104198003360304915780D70C01A00287EF728AFB3
:1041A800931C33605378003318BF012301254B70EB
:1041B8002B46FEF777BF1346511C3160DFF8A88005
:1041C80013F8021B88F802103360234953780B70E8
:1041D800D31C3360214D93782B71131D3360D37832
:1041E800092BA8BF09233046AB70FCF743FD3368A1
:1041F80072682880D11A012905DD3046FCF73AFD9E
:1042080033687268E8819A4207D05A1C32601B787A
:10421800003318BF012388F8073008F0E3F9336842
:1042280072689A423EF4E4AE5A1C32601B78EB7016
:1042380001252B46FEF736BFC4480020243700204E
:1042480098480020D43300208B140020A43A002082
:104258008C4D00200C3B0020BC3A00203C5A00202A
:10426800A825002064300020A0550020C84B1B68FA
:10427800002B3EF4BDAE16F0A1FEFF283EF4B8AE0A
:104288003046FCF7F7FC3F2840F2B483DFF8288378
:10429800002588F8005033687268A8F80400D21A1C
:1042A800012A7EF7A5AE1A46591C316012F8021B86
:1042B80088F8021007F15000326000225D7800F89B
:1042C800242D16F04DFE97F82C30AB423EF490AEFC
:1042D800284616F069FEFEF78BBEAE4B1B78012B05
:1042E8003EF686AE531C11463360DFF8D08211F8D3
:1042F800023B88F80230D31CC01A3160012892F8BA
:1043080001E0336040F385833046FCF7B3FC0125B8
:10431800A8F800002B46FEF7C5BE531C336092F880
:104328000080B8F1110F3FF6D7AB931C33609A4D5C
:10433800537805F818303046FCF79CFC40F6CA0361
:104348009842A8BF184640F2EE23984205EB480170
:10435800B8BF18460125A0F2EE222B46192092FB81
:10436800F0F24A70FEF79EBE1346511C8B4D316029
:1043780013F8021B2971336053786B713046FCF7D0
:1043880079FC336828805A1C32601B78AB71304640
:10439800FCF770FC336868805A1C32601B78EB713C
:1043A80001252B46FEF77EBE0125FDF7CDF92B46EC
:1043B800FEF778BE531C3360794B1278DFF8008221
:1043C8001A700023C8F800303046FCF73BFC33680D
:1043D800D8F800207349744D10435A1CC8F80000DF
:1043E80032601B780B723046FCF744FC286030467C
:1043F800FCF740FC68603046FCF73CFCA86030469F
:10440800FCF738FC3046FCF735FCFEF7F1BD674B8E
:1044180002F108010132326012F8010C03F8010FB1
:104428009142F7D1FEF7E4BD3046FCF723FC304655
:10443800FCF720FC3046FCF71DFC3046FCF726FC58
:1044480033685B4D1946581C2A68306011F8020B16
:1044580082F82C003160597882F83610D91C316006
:104468009B7882F837303046FCF710FC3046FCF772
:104478000DFC3046FCF70AFC3046D5F80080FCF706
:10448800F9FBA8F83A003046D5F80080FCF7F2FBB3
:1044980033687268A8F83800D11A01290ADD591C56
:1044A8002A6831601B7882F82E303046FCF7EEFB24
:1044B80033687268D31A032B0BDD3046D5F80080B9
:1044C800FCF7D8FBA8F8320030462E68FCF7D2FB80
:1044D800B086286847E4531C3360354DDFF8E48024
:1044E800137888F805303046D5F80090FCF7C2FB01
:1044F800A9F820003046D5F80090FCF7BBFB72689D
:104508003368A9F81E00D11A072919DD3046FCF7CF
:10451800B1FBA8F80A003046FCF7ACFBA8F80C0081
:104528003046D5F80090FCF7A5FBA9F822003046E4
:10453800D5F80090FCF79EFB33687268A9F8240050
:10454800D11A03290BDD3046FCF794FBA8F80E00BE
:104558003046FCF78FFB33687268A8F81000D21A4F
:10456800002A05DD591C2A6831601B7882F826303C
:1045780008F038F828F036F80E4B1B68002B00F0CE
:104588001A822868012510F029FC2B46FEF78ABDFF
:10459800C44C002012300020E03400207C28002089
:1045A8000C3B002098480020A825002097480020B0
:1045B8007C450020F03A0020C84C00201430002030
:1045C80064300020A05500201346511C3160BE49BC
:1045D80013F8020BC8703360BC4953784B71D31C75
:1045E8003360BB4B9278DA7001252B46FEF75ABD33
:1045F800D8F80850D8F80010FFF758B8FB697C685D
:104608001A463B7D1370FFF7ABB91346511C316056
:10461800B04D13F8021B6970336053782B70D31CAC
:1046280033609378AB703046FCF724FB33682881FD
:10463800591C1A46316012F8021B697132605B78A6
:10464800AB7101252B46FEF72DBD531C3360137843
:104658000A2B00F0DF803046FCF718FB3046FCF7E9
:1046680015FB01253046FCF711FB2B46FEF71ABD5A
:10467800531C336013780A2B00F0C680502B7FF44C
:10468800BEAE3046FCF7F6FADFF86482A8F8000000
:104698003046FCF7EFFA0125A8F802002B46FEF792
:1046A80001BD8D4B3A6A9B68D4F800905A449A42EF
:1046B80040F2BF803A6AA3EB0208FCF7E3FF4246E8
:1046C8004946386AFDF764F8236803442360002DDF
:1046D8003EF48EACB042BEF68BAC002100E02368FD
:1046E80001305A1CB04222601970F8D1FEF780BC24
:1046F800336872689A4240F0D680784BFF221A706D
:104708004FF0000A764D12F04FFB514620227548B3
:1047180085F800A02CF099FE87F82CA097F82C308B
:10472800072B00F20481DFF8CC916E4E524697F8C1
:104738002C3003EB430309EBC3035B7CE3B197F82D
:104748002C3003EB430309EBC30320215B699BB1C6
:1047580097F82C3003EB430309EBC303586946F879
:1047680022000CF09DFD2B7856F823000CF05AFF20
:104778002A780132D2B22A7097F82C300133DBB292
:1047880087F82C3097F82C30072BD0D92368591C80
:1047980021601A70B8F1000F3EF42AAC524BC8F8E9
:1047A800003001252B46FEF77DBC002D7FF479AF44
:1047B80059462046FCF7A0FA23685A1C22601D704F
:1047C800454B26689D683B6A0BEB0302AA4200F240
:1047D800FD80FCF757FF5A463146386AFCF7D8FF88
:1047E80023680125034423602B46FEF75BBC304653
:1047F800FCF740FA326871687B6A9142834648D177
:1048080006461D46FFF719B83046FCF733FADFF8BD
:10481800E8803BE7931C3360344B51781970D11C06
:10482800316091785970111D3160D2789A70FEF715
:10483800DFBBFCF727FF5A464946386AFCF7A8FF52
:1048480023680344236045E70AEBC80B30468BF81E
:104858000210FCF70FFA33682AF838001A46591C78
:10486800316012F8021B8BF8031032605A788BF80B
:104878000420DA1C32609A788BF806201A1D326000
:104888000135DB788BF80530A9457FF454ABFEF78A
:10489800AFBB511C316012781D46131C064618BF69
:1048A8000123FEF7CABF5A1C194632600B4811F89B
:1048B800022B027031605B784370042A1ED9FF2AEC
:1048C8007EF4B5AB1CE700BFC83A00204054002076
:1048D800D83A0020144500209C060020A01600208D
:1048E8009B5500205C55002069BF0208DF2E002080
:1048F800841D00207C590020B83A00204B490978D3
:10490800994205D8022A7EF492ABFF2B7EF48FAB36
:10491800236801255A1922601D70B8F1000F3EF472
:1049280067AB434BC8F800302B46FEF7BBBB52467B
:104938002CE700F07F00032828BF002001250EF097
:10494800C1FD2B46FEF7AEBB7D62AA46FFF70EB847
:10495800DA46C7F824B0FFF709B83046FCF78AF9F9
:10496800A8843046FCF786F933687268E884D11A5F
:1049780003297FF7EDAB1A46591C316012F8021B68
:10498800A97732605B7885F820303046FCF772F9F9
:10499800336872686884FFF7DBBB04297EF428ABB0
:1049A800FFF72CBA234A1368012523F40043136048
:1049B8002B46FEF777BB20482049214A214B03604C
:1049C80001250B6013602B46FEF76CBB3B6AED1AA2
:1049D800FCF758FE2A463146386AFCF7D9FE2368A8
:1049E80003442360FEF704BB012510F015FC2B4699
:1049F800FEF758BBC50800F0070301350133EDB2D7
:104A0800DFF848802846194688F8013024F0F8FC79
:104A18003FE40D4B91781A88012512FB0EF22B46C4
:104A280092FBF1F2A8F80020FEF73CBBDE4C002018
:104A3800F51B010874450020A0260020F42600205C
:104A48005C270020F50300082E390020C84C002000
:104A58002DE9F04F2DED0E8BDFF8F4B097B0DBF8B1
:104A68000420079058469047002800F08E82BBF833
:104A7800A87000218BF85110002F6DD1BBF93A00B6
:104A8800DBF82450DBF82810BBF93860DBF820404D
:104A9800BBF93C20DFF8BCA0401B521ACBF8300011
:104AA8009BF85210CBF83420341B0BF12C00CBF8B8
:104AB8002C401CF0E5FFDAF80020910041F17987DD
:104AC800DBED0C5A1F4CDBED0B7A1F4994ED406A65
:104AD800D4ED416A94ED427AD4F80C2109681B4B55
:104AE8000593B8EEE58ADBED0D5AF8EEE77AF8EEB5
:104AF800E58A013277EE867A38EE268A78EE878A5A
:104B08008A42C4ED407A84ED418AC4ED428AC4F8F1
:104B18000C2101F04A8393F800E0BEF1140F02F073
:104B28009B870023D4F814510693062D01F297842D
:104B3800DFE815F00416161728152917020CC616F3
:104B48008A1500BFC8160020443D0020304D0020C3
:104B5800B45500203C580020DE4BDF481A68089303
:104B68004FF47A76B6FBF2F2C2EB421602EB8602FB
:104B7800D600DA4BDFF8C88344780593B6B2B7425B
:104B88001D78B8F9060003F08980DBF87C30BBF9A2
:104B98003810DBF8602003F1010E07EE901A0A4482
:104BA800BEF1010FCBF87CE0CBF86020F8EEE77A95
:104BB80003F08180DBED1B5ADBED1D6A07EE10EA7E
:104BC80037EEE56AB8EEC75A012F86EE057A37EE5A
:104BD800257A77EEC77A8BED1C7AE7EE866A8BED3D
:104BE8001B7AF0EE667ACBED1E6ACBED1D6A03F0F8
:104BF8000384DBF89030BBF93A10DBF8642003F14A
:104C0800010E07EE901A0A44BEF1010FCBF890E0AE
:104C1800CBF86420F8EEE77A03F06880DBED205AE1
:104C2800DBED226A07EE10EA37EEE56AB8EEC75AFE
:104C3800012F86EE057A37EE257A77EEC77A8BED67
:104C4800217AE7EE866A8BED207AF0EE667ACBED74
:104C5800236ACBED226A03F0A783DBF8A430BBF903
:104C68003C10DBF8682003F1010E07EE901A0A44A5
:104C7800BEF1010FCBF8A4E0CBF86820F8EEE77A94
:104C880003F04F80DBED255ADBED276A07EE10EACB
:104C980037EEE56AB8EEC75A012F86EE057A37EE89
:104CA800257A77EEC77A8BED267AE6EE276A8BEDC2
:104CB800257AF0EE667ACBED286ACBED276A03F009
:104CC8006683874CA8F80600BBF8A820059B013A24
:104CD8001D78ABF8A82008990022072D4A608A6041
:104CE800CA6040F0598108F027FE059BDFF8508222
:104CF8001D78079BC01A94F82831A8F8000009937A
:104D0800002B40F04F81744A5279002A01F07A81D1
:104D1800744A1278013AD2B2072D84F8282102F099
:104D28001A8200230A93704BD4F83421D3F800A0D8
:104D3800684B0893079B9FED6D6AD4ED4C9A6C49BC
:104D4800C4F834319A1A07EE902AF8EE677AB7EE6B
:104D5800007AC6EE278A0025664BDFF8E891DFF86F
:104D6800E881654F06932E46D1ED006A94ED4BDA43
:104D78009FED629ADFED62AA9FED62CA9FED62AA7B
:104D8800DFED62BA9FED62BA77EE69CA6CEEA6CA29
:104D9800F4EEC7CAF1EE10FA88BFF0EE47CA5D4BD1
:104DA80099ED008A2B44D3ED007AF5EE407AF1EEC6
:104DB80010FA17D0584B2B4493ED007A78EE476AD7
:104DC800B0EEE66AF4EEC67AF1EE10FA08D5F5EE22
:104DD800C06AF1EE10FACCBF37EE878A37EE678AE1
:104DE80083ED008A4D4B1A88930739D0022E37D0AD
:104DF8009AF82E104A4B07EE901A2B4493ED007A3E
:104E08004B42F8EEE76A07EE903A26EE877AF8EE1C
:104E1800E77AB4EEE77AF1EE10FA0AD407EE901AC0
:104E2800F8EE677AF4EEC77AF1EE10FA88BFF0EE82
:104E3800477A3C4B3C4903EB460331F91600B3F97A
:104E48000C30C31A07EE103AB8EEC77AD007E7EE6F
:104E5800497A41F17380354B93ED008A27EE888AB1
:104E6800089B94F868212B4493ED01EA78EE4EDA1A
:104E7800002A00F0F7802E4BD4F86C2107991B68A4
:104E88008A1A9A4240F3EE809AF84830022B02F0D0
:104E9800A181022E04F04584264B1B68990700F176
:104EA8009780254B87ED00CA1B689342C0F2CA80E1
:104EB800F7EE007AF4EEE79AF1EE10FA40F1D280BC
:104EC80008991E4BD1ED017A93ED007AF0EEE77A5E
:104ED8003CE000BF2C580020A0550020304D002099
:104EE800C8160020BC3A00207C45002000247449E4
:104EF800B0270020B4380020C0380020CDCCCC3DED
:104F0800AE47813F000000000000C8420000344363
:104F1800610BB63BA42700200C1800207845002020
:104F280018180020C83A0020284500208C270020A7
:104F3800B827002024450020B4270020C0270020DF
:104F4800344D002000180020CC380020F4EEC77A39
:104F5800F1EE10FA40F18680D1ED027AF0EEE77AB0
:104F6800B4EEE77AF1EE10FA7CDDD1ED037AF0EEDB
:104F7800E77AB4EEE77AF1EE10FA73DD0F4B1B68AF
:104F88009B075FD50E490F4B43E00F4B0F4C1D7825
:104F98000593072D3FF4A7AE94F828310993002B09
:104FA8003FF4B1AE013B84F82831012D01F0A8820D
:104FB80017B0BDEC0E8BBDE8F08F00BF2445002074
:104FC80028450020C83A0020304D0020C81600208F
:104FD800D34BD449DFF8C8E331F916C09EED008AF7
:104FE800DFF8C0E387ED00CA03EB460028EE098A24
:104FF800B0F90C00A0EB0C0007EE900AF8EEE77A87
:10500800DEF8000027EE888A904278EE4EDABFF686
:105018004FAFB3F90C20B1F900E0C348AEEB020E74
:1050280000688EEAEE72A2EBEE7282421ADAB3F9E7
:105038000E30B1F90220D21A82EAE273A3EBE273CE
:1050480098420FDDB94B1A88002384F86831002A8A
:1050580043F06A85B64AB74B1178186881F00101A8
:105068000CF0E6FAB44B2B4493ED000A069B2DEEA8
:10507800000A022E20EE2D0AA3EC010A069304F082
:105088000D83AE4BD7ED006A93ED007AAC4BD3EDB0
:10509800007AAC4B93ED006AAB4B67EE277A2B4452
:1050A80027EEAC7AD3ED007A67EE277AF0EE665AEF
:1050B800EDEEA75AB1EE467AB4EEE57AF1EE10FAC3
:1050C80008DCB4EEE56AF1EE10FA8CBFB0EE657A52
:1050D800B0EE467A94ED4C6AF7EE007AB4EEE76AE1
:1050E800F1EE10FAACBF0123002343B1F0EEE66AFB
:1050F800F0EEC77AF4EEE67AF1EE10FA01D587ED14
:10510800007A022E04F0AC82904A914B52F82600A5
:105118001B68B0EE4E0A98478E4A8F4B52F826000D
:105128001B6898479AF8373023B18C4B1B88002BA3
:1051380000F06B87B0EE4C8A894B38EE400A2B445E
:1051480093ED008A83ED000A9AF8483030EE480A59
:1051580020EE288A002B33D0824B1B7813F00103F2
:1051680000F0B886F7EE007AF4EEE79AF1EE10FA5E
:1051780094F86831C1F2E684002B00F0EB87D4F88C
:105188006C31079AD31A784A12689A4218DD774B1D
:10519800D3ED007AF0EEEDDAF4EEE7DAF1EE10FA9C
:1051A80042F12980614B1A88002384F86831002A6B
:1051B80000F09C866E494A6912B10A6813604B7404
:1051C8006C4B94F878212B4493ED000A2DEE000ADD
:1051D80020EE088A88ED008A32B9069B87ED00CA5E
:1051E80003ED01CA88ED00CA0136032E09F104094E
:1051F80008F1040807F1040705F104057FF4CFADB1
:10520800059B1A78072A01F0B384012A01F09087D8
:105218000023069394F88021002A41F07E81DFF86C
:1052280088A1554BDAF800201968D60491F82C00AB
:1052380000F10687DFF87491504AB9F81A3092EDF8
:10524800006A4F4A4F4DD2ED005AD5ED036A4E4AD7
:1052580084ED646A07EE103A4C4B92ED005AD3ED98
:10526800007AD3ED013AD3ED024A84ED626AB8EED2
:10527800C77A35EEC64A012236EEC77A84ED614A0E
:10528800C4ED655A84F89821C7EE055A0A8D534231
:1052980006EE103A3E4BDFED3F6A93ED005A3E4B67
:1052A80093ED004AB7EE007AF4EEC75A35EE045A89
:1052B800F1EE10FA88BFF0EE475A35EE275AB8EEED
:1052C800C66AF4EEE65AF1EE10FA07EE902AB4EE4A
:1052D800C65AB8BFF0EE665AF1EE10FAC4ED685A35
:1052E800B8EE677A01F10483B4EEC75AF1EE10FA0A
:1052F80088BFB0EE475A264BDFED286AD3ED017A16
:10530800254B93ED014A77EE847A25EE265A77EEFF
:10531800A37AB4EEE76AF1EE10FA52DC48E000BF77
:10532800C83A002028450020BC2700202447002038
:105338002647002028470020602700209C260020C0
:1053480000000020D42700206C270020A42600207D
:10535800A0260020F8260020F4260020784500200A
:1053680038180020C04C0020B8270020C42700208F
:105378002C470020782700207C4500203C3900205D
:10538800943A0020584D00206C280020C038002096
:10539800B438002000000000CC3800206F12833A97
:1053A8008C270020B42700203C5800209848002073
:1053B800B4EEE77AF1EE10FA8CBFB0EE676AB0EEA1
:1053C800476AEC4B4A8DD3ED027A9FEDEB7A534254
:1053D80004EE103A74EEA77AB8EEC44A26EE076ACD
:1053E800F4EEC47AF1EE10FA0AD407EE102AB8EEF9
:1053F800474AB4EEE74AF1EE10FA88BFB0EE674AC2
:10540800DE4ADFEDDD7A527824EE274A0AB9B1EE9A
:10541800444A002841F0D085B7EE003AD84E327899
:10542800002A02F04B86D749DFEDD77AD1ED024A40
:10543800D1ED016A91ED037A66EE244AE5EE264A3B
:10544800E4EE074A63EE244AF4EEE74AF1EE10FA76
:10545800B4BFF0EE673AF0EE643A98BFF0EE647AC3
:10546800012ACDED0E4A02F04E8691ED067AD1ED75
:10547800052AD1ED076A26EE077AA5EE227AA4EE70
:10548800267A23EE077AB4EEE77AF1EE10FAB4EE54
:10549800E37A8CBFF0EE676AF0EE476AF1EE10FA35
:1054A80088BFF0EE676AB4BFF0EE637AF0EE477A31
:1054B800022A8DED0F7A00F0DE8091ED0A7AD1EDA7
:1054C800092AD1ED0B3A26EE077AA5EE227AA4EE48
:1054D800237A23EE077AB4EEE67AF1EE10FAB4EE08
:1054E800E77A8CBFF0EE663AF0EE473AF1EE10FA42
:1054F80098BFF0EE636AA8BFF0EE477A032A8DEDF5
:10550800107A00F0B88091ED0E7AD1ED0D2AD1ED28
:105518000F3A26EE077AA5EE227AA4EE237A23EE36
:10552800077AB4EEE67AF1EE10FAB4EEE77A8CBFB9
:10553800F0EE663AF0EE473AF1EE10FA98BFF0EE68
:10554800636AA8BFF0EE477A042A8DED117A00F05D
:105558009280D1ED123AD1ED112A91ED137A66EECF
:10556800233AE5EE223AE4EE073A63EE233AF4EE04
:10557800E63AF1EE10FAF4EEE73A8CBFB0EE667A4E
:10558800B0EE637AF1EE10FA98BFF0EE476AA8BF62
:10559800F0EE637A052ACDED123A6CD0D1ED163AC9
:1055A800D1ED152A91ED177A66EE233AE5EE223A07
:1055B800E4EE073A63EE233AF4EEE63AF1EE10FA37
:1055C800F4EEE73A8CBFB0EE667AB0EE637AF1EEAD
:1055D80010FA98BFF0EE476AA8BFF0EE637A062A81
:1055E800CDED133A47D0D1ED1A3AD1ED192A91ED04
:1055F8001B7A66EE233AE5EE223AE4EE073A63EECA
:10560800233AF4EEE63AF1EE10FAF4EEE73A8CBFFC
:10561800B0EE667AB0EE637AF1EE10FA98BFF0EE6B
:10562800476AA8BFF0EE637A072ACDED143A22D074
:1056380091ED1E7AD1ED1D2AD1ED1F3A26EE077A9B
:10564800A5EE227AA3EE847A27EE037AB4EEE67A00
:10565800F1EE10FAB4EEE77A8CBFB0EE666AB0EEFF
:10566800476AF1EE10FA8DED157A98BFF0EE466AAA
:10567800A8BFF0EE477A77EEE67AF7EE006AF4EE26
:10568800E67AF1EE10FAC4ED4C7A43F3D78586EE4C
:10569800A77A022ADDED0F7A67EE244A67EE877A49
:1056A800CDED0E4ACDED0F7A2DD0DDED107A67EEF7
:1056B800877A032ACDED107A25D0DDED117A67EED1
:1056C800877A042ACDED117A1DD0DDED127A67EEC6
:1056D800877A052ACDED127A15D0DDED137A67EEBB
:1056E800877A062ACDED137A0DD0DDED147A67EEB0
:1056F800877A072ACDED147A05D0DDED157A27EEE5
:10570800877A8DED157A2149096811F080530A933B
:1057180001F0CB81F6EE005AC4ED685A002A02F077
:105728009D8494F998311A4994ED656AC87894ED86
:10573800645ADAF80010DFF868E0164FDEED004A28
:10574800B7F906E0B9F81A700B9707EE103A124B42
:10575800D4ED616A1D78114BD4ED627A1B780893F9
:10576800BDEEC66A01F4805316EE10CABDEEC56AD6
:105778000D9317E0B43800206F12833A0C3B0020D9
:10578800DE4C0020DC270020000000001839002033
:10579800184F0020D2690020C04C0020605A002019
:1057A800D827002001F4800301F01007B8EEC77A6B
:1057B8000C9305F0010816EE101A002840F06487D3
:1057C800002F41F0D582D34D9DED0E5A95ED006A1C
:1057D800D14825EE866AA5EE076AB0EE675AA6EEAE
:1057E800265ABDEEC56A16EE10EA16EE107AE645A0
:1057F800A8BF67467145C8BF0F4606EE107AB8EED7
:10580800C66A012A80ED006A00F0DC8095ED046A22
:105818009DED0F5A25EE866AA5EE076AB0EE675A27
:10582800A6EE265ABDEEC56A16EE10EA16EE107AF6
:10583800E645A8BF67467145C8BF0F4606EE107A11
:10584800B8EEC66A022A80ED016A00F0BB8095EDC9
:10585800086A9DED105A25EE866AA5EE076AB0EE35
:10586800675AA6EE265ABDEEC56A16EE10EA16EE7F
:10587800107AE645A8BF67467145C8BF0F4606EED1
:10588800107AB8EEC66A032A80ED026A00F09A80A0
:1058980095ED0C6A9DED115A25EE866AA5EE076A0C
:1058A800B0EE675AA6EE265ABDEEC56A16EE10EAA5
:1058B80016EE107AE645A8BF67467145C8BF0F4681
:1058C80006EE107AB8EEC66A042A80ED036A79D02B
:1058D80095ED106A9DED125A25EE866AA5EE076AC7
:1058E800B0EE675AA6EE265ABDEEC56A16EE10EA65
:1058F80016EE107AE645A8BF67467145C8BF0F4641
:1059080006EE107AB8EEC66A052A80ED046A59D008
:1059180095ED146A9DED135A25EE866AA5EE076A81
:10592800B0EE675AA6EE265ABDEEC56A16EE10EA24
:1059380016EE107AE645A8BF67467145C8BF0F4600
:1059480006EE107AB8EEC66A062A80ED056A39D0E6
:1059580095ED186A9DED145A25EE866AA5EE076A3C
:10596800B0EE675AA6EE265ABDEEC56A16EE10EAE4
:1059780016EE107AE645A8BF67467145C8BF0F46C0
:1059880006EE107AB8EEC66A072A80ED066A19D0C4
:1059980095ED1C6A9DED155A65EE865AE7EE055A97
:1059A800E6EEA57AFDEEE77A17EE905AAC45A8BF69
:1059B800AC46A942D8BF614607EE901AF8EEE77ADE
:1059C800C0ED077AB8F1000F00F06C87534A1268EF
:1059D800002A40F07487524A127892B1307868B140
:1059E8004D4FDFF85C810025E8B2D8F80030B7ECFD
:1059F800010A9847307801358542F5DB494A126833
:105A08009047059B1A78072A01F0A1800026DAF84A
:105A18000020530500F1D187434B1B78BBB1434AA3
:105A2800B9F81A30B2F906209A4210DC404B1B78BC
:105A3800012B01F09583192B01F092830E2B06D0D0
:105A4800082B04D03B4D0023AB60C4F8403194F8D8
:105A5800AA5125B1384B1B889F0741F02F8394F832
:105A6800B021002A40F0488799F81E70002F00F0F6
:105A78002984022F01F0D582032F41F0CE8299F8B4
:105A88002030C3EB431103EB8101C90089B299F8B7
:105A98001F300233DBB2002A00F05585002900F0E0
:105AA800528526480768B1FBF7F10FB2A4F8E071F8
:105AB800002B03F0438007EE907AF8EEE77AF7EED2
:105AC800006A86EEA77A1B4D012BD4ED7D6AD5EDD1
:105AD800007A77EEE67A67EE877AC4ED797A3BD07A
:105AE800D5ED017AD4ED7E6A77EEE67A022B67EE81
:105AF800877AC4ED7A7A2FD0D5ED027AD4ED7F6A11
:105B080077EEE67A032B67EE877AC4ED7B7A23D0AB
:105B180018E000BFDC270020E8380020A44200205D
:105B2800885D00205C5A00208B140020D269002078
:105B38000C3B0020584D002078450020F03A00200A
:105B4800545A0020D5ED037AD4ED806A77EEE67AD0
:105B580067EE877AC4ED7C7A05990978092903F0FC
:105B6800ED81002F40F3B4839BB394ED7D7AD4ED9F
:105B7800797A77EE877A012BC4ED7D7AC5ED007AC4
:105B880021D094ED7E7AD4ED7A7A77EE877A022B5B
:105B9800C4ED7E7AC5ED017A15D094ED7F7AD4ED07
:105BA8007B7A77EE877A032BC4ED7F7AC5ED027A8C
:105BB80009D0D4ED807A94ED7C7A77EE877AC4EDBB
:105BC800807AC5ED037A013B022BB8BF0223DBB212
:105BD8000993099B002A18BF02239E46C84BDFED94
:105BE800C96A1A68059B91781878137807EE903A75
:105BF800F8EEE77AB0EE007A67EEA67AF4EEC77AA6
:105C0800F1EE10FA40F35F86DFEDBF6A37EEC77A30
:105C1800B0EE676AA7EE266AF0EE466A95ED007A5E
:105C28009FEDBA6A27EE066AF0EEC65A84ED546A0A
:105C3800C4ED575A99B107EE101AB8EEC75A9FED3E
:105C4800B17A66EE064A25EE075AB7EE007A37EEC5
:105C5800457A64EEA54AA4EE857A26EE076A9FED9A
:105C6800AC7A537926EE877A27EE067ACBB1DFED48
:105C7800A56A9FEDA86A65EEA65A06EE903AF8EE78
:105C8800E66A65EEA65AF4EEC65AF1EE10FA01F38A
:105C98008981B7EE006A76EE655AC6EE256A27EE68
:105CA800267A0C289FED9C8ADFED9C6A00F02487F9
:105CB800B4EEC87AF1EE10FA98BFB0EE478AB4EEA7
:105CC800E68AF1EE10FAB8BFB0EE668A84ED4E8A25
:105CD800BEF1000F00F0DD80B0EE007AF4EEC77A76
:105CE800F1EE10FA05DD37EEC77ADFED876AE7EEE9
:105CF800267A95ED017ADFED856A27EE267AF0EEB1
:105D0800C75A84ED557AC4ED585A99B106EE901ADF
:105D18009FED7C6AF8EEE66A27EE075A66EE866A19
:105D2800B7EE006A36EE666A25EE255AA5EE266AB3
:105D380027EE067ADFED766A937967EEA67A67EE44
:105D4800877AABB107EE103AB8EEC77A9FED6D6A65
:105D5800DFED706A27EE257A27EE067AB4EEE67A4A
:105D6800F1EE10FA41F31081DFED6D6A67EEA67A65
:105D78000C2800F0A186DFED686A9FED687AF4EEE2
:105D8800E67AF1EE10FA88BFF0EE667AF4EEC77A9A
:105D9800F1EE10FAB8BFF0EE477ABEF1010FC4ED8C
:105DA8004F7A76DD5378DFED576A07EE903AF8EED2
:105DB800E77AB0EE007A67EEA67A537AF4EEC77AFD
:105DC800F1EE10FA05DD37EEC77ADFED4F6AE7EE40
:105DD800267A95ED027ADFED4D6A27EE267AF0EE07
:105DE800C75A84ED567AC4ED595A9BB106EE903ADB
:105DF8009FED446AF8EEE66A27EE075A66EE866A71
:105E0800B7EE006A36EE666A25EE255AA5EE266AD2
:105E180027EE067ADFED3E6AD37967EEA67A67EE5B
:105E2800877AFBB107EE103AB8EEC77A9FED356A6C
:105E3800DFED386A27EE257A27EE067AB4EEE67AA1
:105E4800F1EE10FA01F39C80B5EEC07AF1EE10FA8B
:105E580002F1FE82B7EE006A36EE477AC6EE076AAE
:105E680067EEA67A0C2800F06586DFED2B6A9FEDB9
:105E78002B7AF4EEE67AF1EE10FA88BFF0EE667A45
:105E8800F4EEC77AF1EE10FAB8BFF0EE477AC4ED37
:105E9800507A092800F0FC8599F82150002D40F02F
:105EA800B185002384F8B0311E4B1B7823B91E4DF1
:105EB800AA78002A41F0C180059B1D78072D7FF440
:105EC80074A807F039FD194B059A801B1578D880FE
:105ED800FFF76BB894F86821002A3FF471A9144AB7
:105EE80084F868311288002A7FF464A9114A124B99
:105EF8001178186881F001010BF09AFBFFF760B97F
:105F0800804500200AD7233CD7A368416F12033B82
:105F180000004843A4707D3F00C0F94400C0F9C4A4
:105F28000000C8425554002014300020344D002091
:105F380024470020264700202847002094ED577A60
:105F4800B1F90000D4ED586AB1F902E0E24AF4EE82
:105F5800C76A80EAE0738EEAEE71A3EBE073F1EEB4
:105F680010FAA1EBEE71B8BFF0EE476A8B42B8BFEA
:105F78000B4607EE103A1378B8EEC77A27EE097A7F
:105F8800002B40F0B880D54B93ED006AB4EEEA6A76
:105F9800F1EE10FA41F14C80F7EE005A75EEC65A50
:105FA8003BEEC77A65EE8B5ACD4BA7EE256A93ED8B
:105FB800007A26EE076AB5EEC06AF1EE10FA40F2F2
:105FC8007085CAEE065AB7EE007AB0EE476AA6EEBA
:105FD800E56AF0EE466AF4EEC76AF1EE10FA88BF99
:105FE800F0EE476AF5EEC06AF1EE10FAB8BFF0EECF
:105FF8004C6ABC4B93ED007A67EE877AA7EEA68AC7
:10600800FEF72EBF0122FEF787BEB74BB74A2B44D7
:1060180093ED007AD2ED007AB54B67EE277AF7EE6A
:10602800006AF4EEE67AF1EE10FA93ED007A88BF92
:10603800F0EE667A67EE877A27EE888AFFF77CB8F3
:10604800AC4BDFF8EC921A78D5075CBFB9F818208A
:10605800A4F88C21A84AA94D1288D5ED037A07EE39
:10606800102AB8EEC77AF4EEC77AF1EE10FA41F2C8
:10607800C587A34D2B8807EE103AB8EEC77AF4EE21
:10608800C77AF1EE10FAC1F277809E4A9E4D92EDE2
:10609800006AD5ED006A94F99821C4ED646A76EE39
:1060A800665A012AC4ED626AC4ED615A84ED656AD4
:1060B80001F0EE85079BC4F89C31002537EEC77ABE
:1060C800FCEEE77A914E84ED687A17EE902AA4F8F0
:1060D8008C21012296ED005A84F898218C4A954229
:1060E80041F279878B4BD3ED007AD3ED013AD3EDAA
:1060F800024AFFF7C9B87A4B93ED005AB5EEC05A79
:10610800F1EE10FA40F3CD84834BD3ED004AF5EE5F
:10611800C04AF1EE10FA40F3C48434EEC77A66EE52
:10612800CA5A87EE246AC5EE856AB7EE007AB4EEDD
:10613800C76AF1EE10FA88BFB0EE476AB5EEC06ADA
:10614800F1EE10FA76EE876AB8BFB0EE4C6A66EEEA
:10615800266A40E7714AD2ED007AB0EEC87AB4EE0A
:10616800E77AF1EE10FA7FF72BA86D4AD2ED007AA4
:10617800B0EEED7AB4EEE77AF1EE10FA7FF720A8E8
:10618800684AD9ED007A92ED007AF0EEE77AF4EEFB
:10619800C77AF1EE10FA7FF513A801220799C4F81F
:1061A8006C1184F86821FEF7EEBF07EE102A197803
:1061B800DFF88081C4F80C71B8EEC77AF7EE006A90
:1061C800132986EE879AB8F90400B4F810619BED9C
:1061D800070A01F0E984544A544992ED001AD2EDB5
:1061E800053A92ED122A92ED173AD2ED091AD2ED3C
:1061F8000E4A92ED016A92ED064A92ED0A7AD2EDC4
:106208000F5AD2ED132AD2ED186A92ED045AD2ED44
:10621800030A67EE897A69EE288A29EE088AE1EE90
:10622800273A01EB86070025A2EE283AC4F8005168
:10623800C4F80451E1EE884AA6EE274AE7EE085A68
:1062480092ED167A92ED0D6A92ED021AD2ED0C1AC1
:10625800C7ED003AE2EEA86A25EE635A27EE437AC4
:1062680092ED0B2AD2ED152AC7ED204AA0EEE34A9B
:1062780026EE646AD2ED143A82ED054AA1EE275A59
:10628800F0EE477AE1EEE45AA2EE086AE2EEC36A5B
:10629800E3EEA87A82ED065AC2ED0E5A82ED0F6A35
:1062A80087ED403AC2ED176AC2ED187AC4F8085172
:1062B800721C02F01F02A4F81021A8F80400059B24
:1062C800FEF729BCA4F8E071002A3FF4EDAD0B4DB0
:1062D8004FF0020E82E400BF98270020A02700207C
:1062E80094270020902700202418002088270020C9
:1062F80084270020C04C002070280020584D002022
:1063080072280020943A00205C2800207828002079
:106318008FD00300C03800209C270020C827002009
:10632800C4270020CC270020D43F0020683D00204F
:1063380098480020344D0020BC4A1178D4F81871D0
:10634800BB4B9FEDBC7AFE009A1982ED007A0029BA
:1063580079D0B948B0EE476AF0EE476A0022F0EC0F
:10636800017A013267EEA77A05EE902AB4EEE77A51
:10637800F1EE10FAF8EEE55AB8BFB0EE677A8A4245
:1063880076EEA76AA7EEA56AE9D1F5EEC06A9A1972
:10639800F1EE10FA82ED007A55DDC6EE265AA74ACC
:1063A800A7490988F7EE007A75EEE75AD2ED007A28
:1063B80065EEA77AFDEEE77A17EE902A812A42F376
:1063C80053808A42A8BF0A4607EE902AF8EEE77A79
:1063D8009C4AF01902EB800292ED057AD2ED003A60
:1063E80092ED066A92ED014AD2ED046AD2ED034AB3
:1063F80092ED025AA3EEA77AA4EE276A66EEC76A60
:10640800A7EE646ABDEEC77AE5EE276A17EE100AB2
:10641800812882ED056AC2ED066A42F32280814234
:10642800A8BF014607EE901AF8EEE77AFCEEE77A85
:10643800CDED087ABDF8202099198A801FB9BEF1E0
:10644800130F02F0E786BEF1150F41F0ED801E44F0
:10645800DFF81082B28828F81720D4F814517A4A45
:10646800013582FB05325119EA17C2EBA102C2EBD2
:10647800C202AD1AC4F814517448D4F81C11079B11
:10648800734D02682D78C4F81C31591A0A44026009
:10649800002D64D107EE901A6E4EDFF8E0916E4F32
:1064A800B8EEE78A06F5F07506F51378F6EC017A8A
:1064B8009BED070ADBF80832F8EEE77A284627EE64
:1064C800800A9847A5F1E000DBF828319847A5F144
:1064D8007000DBF898319847D6F8EC00DBF8AC3060
:1064E8009847D7ED007AA9EC010AE0EE087A24353E
:1064F800A845E7EC017AD9D1059B1D78FEF749BD7F
:10650800564B574A19681288564BC96919805A80E0
:1065180017B0BDEC0E8BBDE8F08F534B534E1A7875
:1065280012F0010F327840F03983002A00F03E85DE
:1065380092004F494F48DFF848A1DFF8489129F009
:1065480089FEFFF743BAB4F8E071013F3FB2002F6C
:10655800A4F8E0717FF7B8AE474DFFF705BB07EE2B
:10656800901A3C4D454BDFF8FC80DFF8EC90069420
:10657800F8EEE78A05F5B8760027CDF824801C46A2
:10658800059BDBED077A1B78172B00F0A08195EDB2
:10659800007AB8EEC78A082B28EE278A07D1B0EE12
:1065A800480A089329F096FF089BA8F80000DAF833
:1065B800002092000BD5002F03F01381B0EE480A9B
:1065C800DBF8083206F170009847B0EE408AB0EE6A
:1065D800480ADBF82831A6F170009847DBF89831B3
:1065E80030469847059B1B78032BB0EE408A00F095
:1065F8007A81D5F8F000DBF8AC30B0EE480A98475D
:10660800D9ED007AA4EC010AE0EE287A0137032FCD
:1066180006F1240608F1020805F10405E9EC017AFF
:10662800AED1059B069C1D78FEF7B3BC4A3D002001
:106638004040002000000000C81600204C3D00200B
:10664800483D0020683F002093244992602600209E
:10665800403D0020E0550020642600206C460020C4
:1066680068350020344D0020C04C0020DE4C00204E
:1066780040380020E8380020584D002030580020CD
:106688003C58002098480020002F00F09186B8F16F
:10669800000F42F0A982089BCD4D002B42F0F680F6
:1066A80095ED006A9DED0E5ACA4825EE866AFDEE04
:1066B800E44AA5EE076AB0EE675AA6EE265A14EE2B
:1066C800901ABDEEC56A16EE10EA16EE107AE64587
:1066D800A8BF67467145C8BF0F4606EE107AB8EEE8
:1066E800C66A012A80ED006A00F0DF8095ED046A31
:1066F8009DED0F5A25EE866AA5EE076AB0EE675A39
:10670800A6EE265ABDEEC56A16EE10EA16EE107A07
:10671800E645A8BF67468E45B8BF0F4606EE107A15
:10672800B8EEC66A022A80ED016A00F0BE8095EDD7
:10673800086A9DED105A25EE866AA5EE076AB0EE46
:10674800675AA6EE265ABDEEC56A16EE10EA16EE90
:10675800107AE645A8BF67468E45B8BF0F4606EED5
:10676800107AB8EEC66A032A80ED026A00F09D80AE
:1067780095ED0C6A9DED115A25EE866AA5EE076A1D
:10678800B0EE675AA6EE265ABDEEC56A16EE10EAB6
:1067980016EE107AE645A8BF67468E45B8BF0F4685
:1067A80006EE107AB8EEC66A042A80ED036A7CD039
:1067B80095ED106A9DED125A25EE866AA5EE076AD8
:1067C800B0EE675AA6EE265ABDEEC56A16EE10EA76
:1067D80016EE107AE645A8BF67468E45B8BF0F4645
:1067E80006EE107AB8EEC66A052A80ED046A5CD017
:1067F80095ED146A9DED135A25EE866AA5EE076A93
:10680800B0EE675AA6EE265ABDEEC56A16EE10EA35
:1068180016EE107AE645A8BF67468E45B8BF0F4604
:1068280006EE107AB8EEC66A062A80ED056A3CD0F4
:1068380095ED186A9DED145A25EE866AA5EE076A4D
:10684800B0EE675AA6EE265ABDEEC56A16EE10EAF5
:1068580016EE107AE645A8BF67468E45B8BF0F46C4
:1068680006EE107AB8EEC66A072A80ED066A1CD0D2
:1068780095ED1C6A9DED155A65EE865AE7EE055AA8
:10688800E6EEA57AFDEEE77A17EE905AAC45A8BF7A
:10689800AC46A942D8BF614607EE901AF8EEE77AEF
:1068A800C0ED077A002A3FF491A892004A49494866
:1068B80029F0D0FC494A1268002A3FF48CA81CF041
:1068C800ADF8FFF788B8F0EE676AFFF7A7B995ED5E
:1068D800007A0BEB4702B8EEC78A128FA8F800209F
:1068E80028EE278A63E629F0F5FDA8F8000080E67F
:1068F800B0EE465AFEF7FFBC39493A4BD1F8EC10D6
:106908001B6844F620608142A8BF0146B1F57A7F32
:10691800B8BF4FF47A7189B213F0100FA4F8B2110E
:10692800DAF8003000F02384DB0441F1A1852E4B16
:10693800D3F800E0BEF832707F082C4D2C48D4F80C
:10694800B431D5ED037AA0FB01018809642191FBDC
:10695800F0F11429BDEEE77A04EB4305A8BF142132
:1069680001338B42C4F8B43117EE10CAA4BF002318
:10697800C4F8B43104EB4303A5F8B8C1B3F9B8318E
:1069880007EE103AB8EEC77A77EEC77AFDEEE77AE7
:10699800CDED067ABDF9181081EAE173A3EBE17336
:1069A800BB4201F32D8713494FF07E530B60FFF76D
:1069B8005BB8114B0593114C5EE5DBF80830002BF2
:1069C8003FF42AA80E49A1F14C009847FFF724B8D4
:1069D800DC270020E838002040380020A4420020AE
:1069E80020010020183900207C450020584D002047
:1069F800D34D621000000020304D0020C816002042
:106A0800005600201E21CE48FAF752FC00283FF419
:106A180048AACC4B1B8858063FF543AA94F8043281
:106A2800AB4242F01C82C84BD4ED827AD3ED016AA6
:106A380094ED505ADFEDC55A9FEDC56A27EEC57A29
:106A480068EE277AA8EE267AE5EE267AB4EEE57A9D
:106A5800F1EE10FA88BFB0EE657AB4EEC67AF1EEC0
:106A680010FAF4EEE57AB8BFB0EE467AF1EE10FA15
:106A780088BFF0EE657AF4EEC67AF1EE10FAB8BF88
:106A8800F0EE467A84ED4E7AC4ED507AFFF709BAF3
:106A9800FDEEC87AAF4A17EE903A9780D380FFF799
:106AA800FBB9DFEDAD6AFFF7A4BADAF800104902C6
:106AB8003EF530AEFEF732BE9FEDA47ADFEDA46A54
:106AC800A449F4EEC77AF1EE10FA98BFB0EE677AEF
:106AD800FDEEE77AB4EEE67AF1EE10FA17EE903AA8
:106AE800B8BFB0EE667ABEF1010F84ED4F7A4B80E5
:106AF8003FF758A9FFF7D0B9B4EEC87AF1EE10FA0B
:106B080098BFB0EE478ABDEEC77AB4EEE68ADFF8E2
:106B180044C2F1EE10FA17EE103AB8BFB0EE668A2A
:106B280084ED4E8AACF80030BEF1000F7FF4D4A893
:106B3800FFF7B2B9BDEEE77A864B17EE102A9A80B6
:106B4800FFF793B9002B3EF43BABFEF718BB06F0FA
:106B5800F3FE059B7F491A78069B072AA0EB0300E2
:106B680088807EF453AF06F0E7FE0646FEF74FBF77
:106B780006F0E2FE059BDFF8DC811A780A9B012A01
:106B8800A0EB0300A8F8020000F0D482072A7EF4E4
:106B98003FAB06F0D1FE0690FEF73CBB002A00F0A2
:106BA8000582D4ED583A94ED574AD4ED627A6B4990
:106BB80094ED617A91ED005AD4ED555A94ED546AEA
:106BC800674D6848F4EEC43AF3EE046AF1EE10FA41
:106BD80077EEA64A00F11E8395ED026A26EE656AF5
:106BE800B0EE674AA6EE074AB4EEE44A34EE666AA7
:106BF800F1EE10FA48BFB0EE456A012A80ED006A4E
:106C080000F0D48195ED066A26EE656AB0EE674A13
:106C1800A6EE074AB4EEE44A34EE666AF1EE10FADC
:106C280048BFB0EE456A022A80ED016A00F0BE81D5
:106C380095ED0A6A26EE656AB0EE674AA6EE074A3F
:106C4800B4EEE44A34EE666AF1EE10FA48BFB0EEEC
:106C5800456A032A80ED026A00F0A88195ED0E6A64
:106C680026EE656AB0EE674AA6EE074AB4EEE44A35
:106C780034EE666AF1EE10FA48BFB0EE456A042AAF
:106C880080ED036A00F0928195ED126A26EE656A3E
:106C9800B0EE674AA6EE074AB4EEE44A34EE666AF6
:106CA800F1EE10FA48BFB0EE456A052A80ED046A95
:106CB80000F07C8195ED166A26EE656AB0EE674AAB
:106CC800A6EE074AB4EEE44A74EE666AF1EE10FAEC
:106CD80048BFF0EE456A062AC0ED056A00F06681F5
:106CE800D5ED1A6A66EEE56AB0EE674AA6EE874AFF
:106CF800B3EE046AB4EEE44A74EE466AF1EE10FAB2
:106D080048BFF0EE456A072AC0ED066A00F04E81DA
:106D1800D5ED1E6ADFF850A0DFF8509066EEE55A10
:106D2800E5EE877AF4EEE74A77EEC67AF1EE10FAE6
:106D3800C8BFF0EE457AC0ED077AFEF747BE00BF40
:106D480018390020784500200000002000C0F944D0
:106D580000C0F9C4344D002000000000D8270020EE
:106D6800DC270020E83800203C5800209848002004
:106D7800B8F1000F41F00282DB4D9DED0E5A95ED02
:106D8800006ADA4825EE866AA5EE076AB0EE675A09
:106D9800A6EE265ABDEEC56A16EE10EA16EE107A71
:106DA800E645A8BF67467145C8BF0F4606EE107A8C
:106DB800B8EEC66A012A80ED006A3FF476AD95ED1B
:106DC800046A9DED0F5A25EE866AA5EE076AB0EEB5
:106DD800675AA6EE265ABDEEC56A16EE10EA16EEFA
:106DE800107AE645A8BF67467145C8BF0F4606EE4C
:106DF800107AB8EEC66A022A80ED016A3FF455ADF2
:106E080095ED086A9DED105A25EE866AA5EE076A8B
:106E1800B0EE675AA6EE265ABDEEC56A16EE10EA1F
:106E280016EE107AE645A8BF67467145C8BF0F46FB
:106E380006EE107AB8EEC66A032A80ED026A3FF4BD
:106E480034AD95ED0C6A9DED115A25EE866AA5EED6
:106E5800076AB0EE675AA6EE265ABDEEC56A16EE68
:106E680010EA16EE107AE645A8BF67467145C8BF16
:106E78000F4606EE107AB8EEC66A042A80ED036A59
:106E88003FF413AD95ED106A9DED125A25EE866A12
:106E9800A5EE076AB0EE675AA6EE265ABDEEC56A99
:106EA80016EE10EA16EE107AE645A8BF6746714559
:106EB800C8BF0F4606EE107AB8EEC66A052A80EDFE
:106EC800046A3FF4F2AC95ED146A9DED135A25EE71
:106ED800866AA5EE076AB0EE675AA6EE265ABDEE98
:106EE800C56A16EE10EA16EE107AE645A8BF6746A0
:106EF8007145C8BF0F4606EE107AB8EEC66A062A74
:106F080080ED056A3FF4D1AC95ED186A9DED145AF1
:106F180025EE866AA5EE076AB0EE675AA6EE265AEF
:106F2800BDEEC56A16EE10EA16EE107AE645A8BF61
:106F380067467145C8BF0F4606EE107AB8EEC66AB6
:106F4800072A80ED066A3FF4B0AC95ED1C6A9DED0A
:106F5800155A65EE865AE7EE055AE6EEA57AFDEE75
:106F6800E77A17EE905AAC45A8BFAC46A942C8BF0D
:106F78008C4607EE90CAF8EEE77AC0ED077A91E4FE
:106F8800DFED5B6AFEF76CBFB5EEC07AF1EE10FA82
:106F980001F15A82B7EE006A36EE477AC6EE076A02
:106FA800FEF7E4BEDFED526AFEF779BEDFF878A19E
:106FB800DFF87891FEF70ABD4E494A79002A3EF477
:106FC8002BAA4D4A1278002A3EF426AA0B784B4980
:106FD800DFED4B4A07EE903A0B88B8EE677A07EE7A
:106FE800902A06EE903AF8EEE77AF8EE666A67EECF
:106FF800277AB7EE007A87EEA63AB4EEE43AF1EED5
:1070080010FA88BFB0EE643AB4EEC73AF1EE10FA5F
:10701800B8BFB0EE473AFEF701BA3A4B5988FEF7C7
:1070280036BDB4F8B21101F57A7189B2FEF72FBDF9
:10703800354B93ED006AFEF7BEBF344F3B78013BFA
:107048000D2B24D8DFE813F0F506BB07E606CB06C0
:1070580023002300A4078F0734070E0067075B0788
:10706800860702072A4B1B78002B02F0F5801A20AE
:107078000FF06AF9002842F0EF80264B1B78002BAE
:1070880042F0EA8009233B7018F0BEFAAA78012A78
:1070980000F063852B79012B01F05985022B7EF4D2
:1070A8000BAF3B78012B7EF407AF1A4B1B78002BF4
:1070B8007EF402AF19F0F0F9FEF7FEBE164B9FED15
:1070C800177AD3ED087AF4EEC77AF1EE10FA00F2E7
:1070D800F9849FED137A134DD5ED037A77EE877A0D
:1070E800C5ED037AFEF7BBBCDC270020E83800209A
:1070F8000000C84214450020564D0020404D002095
:10710800713DAA3FA054002094270020123000208F
:107118000E3B00200F3B0020382600208FC2753C14
:1071280000000000584D00203C58002098480020DE
:10713800DFF8708206F000FC9049D4F87C210968D9
:107148000690821A511AC4F87C01A8F80420A8F8FD
:107158000610FEF75FB806F0EFFB0A90FDF7E3BDF7
:10716800874B9B7B002B3EF46DACFEF770BCDD00BB
:107178003FF5DAABFEF778BCB4F88C51954240F293
:10718800028594F8A451002D40F06E877D4A7E4E0A
:1071980092ED007AD6ED007A94F99821C4ED647ADC
:1071A80077EE676A012AC4ED627AC4ED616A84EDFC
:1071B800657A02F03D80079BC4F89C31734A9FEDC5
:1071C800747A92ED005A84ED687A012284F8982145
:1071D800FEF784BF6F4B1B88002B40F0E8856E4A92
:1071E8006E4B117818680AF023FAD4F86C21079BC3
:1071F8009A1AFDF74EBE6A4BD9ED007A93ED007AE4
:10720800F0EEE77AF4EEC77AF1EE10FA7DF7D8AF30
:10721800FDF7C8BFD5ED015A65EEC65AB0EE674A0C
:10722800A5EE874AB4EEE44A74EE665AF1EE10FA17
:1072380048BFF0EE455A012AC0ED005A3FF4B6AEF9
:10724800D5ED055A65EEC65AB0EE674AA5EE874AEF
:10725800B4EEE44A74EE665AF1EE10FA48BFF0EE66
:10726800455A022AC0ED015A3FF4A0AED5ED095A9D
:1072780065EEC65AB0EE674AA5EE874AB4EEE44A10
:1072880074EE665AF1EE10FA48BFF0EE455A032A3A
:10729800C0ED025A3FF48AAED5ED0D5A65EEC65AD6
:1072A800B0EE674AA5EE874AB4EEE44A74EE665A31
:1072B800F1EE10FA48BFF0EE455A042AC0ED035A21
:1072C8003FF474AED5ED115A65EEC65AB0EE674A72
:1072D800A5EE874AB4EEE44A74EE665AF1EE10FA67
:1072E80048BFF0EE455A052AC0ED045A3FF45EAE99
:1072F800D5ED155A65EEC65AB0EE674AA5EE874A2F
:10730800B4EEE44A74EE666AF1EE10FA48BFF0EEA5
:10731800456A062AC0ED056A3FF448AED5ED196AFC
:1073280066EEC66AB0EE674AA6EE874AF3EE045ADE
:10733800B4EEE44A74EE656AF1EE10FA48BFF0EE76
:10734800456A072AC0ED066A3FF430AED5ED1D6ADE
:10735800DFF854A0DFF8549026EEC66AE6EE077A06
:10736800F4EEE47A77EEE57AF1EE10FAB8BFF0EED3
:10737800457AC0ED077AFEF729BB00BFF03A002036
:10738800FC480020943A00205C280020782800203F
:10739800000000002447002026470020284700203E
:1073A800CC270020344D00203C580020984800206D
:1073B800089BD94D002B41F08D8095ED006A9DED1D
:1073C8000E5AD64825EE866AFDEEE44AA5EE076A0F
:1073D800B0EE675AA6EE265A14EE901ABDEEC56AAC
:1073E80016EE10EA16EE107AE645A8BF6746714514
:1073F800C8BF0F4606EE107AB8EEC66A012A80EDBD
:10740800006A3EF4DFAA95ED046A9DED0F5A25EE59
:10741800866AA5EE076AB0EE675AA6EE265ABDEE52
:10742800C56A16EE10EA16EE107AE645A8BF67465A
:107438008E45B8BF0F4606EE107AB8EEC66A022A25
:1074480080ED016A3EF4BEAA95ED086A9DED105ADA
:1074580025EE866AA5EE076AB0EE675AA6EE265AAA
:10746800BDEEC56A16EE10EA16EE107AE645A8BF1C
:1074780067468E45B8BF0F4606EE107AB8EEC66A64
:10748800032A80ED026A3EF49DAA95ED0C6A9DEDF3
:10749800115A25EE866AA5EE076AB0EE675AA6EE7F
:1074A800265ABDEEC56A16EE10EA16EE107AE645C3
:1074B800A8BF67468E45B8BF0F4606EE107AB8EEED
:1074C800C66A042A80ED036A3EF47CAA95ED106A28
:1074D8009DED125A25EE866AA5EE076AB0EE675A48
:1074E800A6EE265ABDEEC56A16EE10EA16EE107A1A
:1074F800E645A8BF67468E45B8BF0F4606EE107A28
:10750800B8EEC66A052A80ED046A3EF45BAA95EDDA
:10751800146A9DED135A25EE866AA5EE076AB0EE49
:10752800675AA6EE265ABDEEC56A16EE10EA16EEA2
:10753800107AE645A8BF67468E45B8BF0F4606EEE7
:10754800107AB8EEC66A062A80ED056A3EF43AAAB1
:1075580095ED186A9DED145A25EE866AA5EE076A20
:10756800B0EE675AA6EE265ABDEEC56A16EE10EAC8
:1075780016EE107AE645A8BF67468E45B8BF0F4697
:10758800FEF7FEB9664ED4ED017A94ED006A3188B3
:10759800726977EEA77AF0EE006AB0EE677AA6EE27
:1075A800267A4E1E04EBC601D6EE267A083910322A
:1075B800F6EE003A27EE237A67EEA37A84ED207A76
:1075C800C4ED217A574C274604F1800091ED027AE8
:1075D80091ED036AD7ED036AD7ED027A52ED014ABD
:1075E80012ED025A37EE674A76EEC65A77EE277AD8
:1075F800E4EE845A013EA1F10801E5EE047A07F1B0
:10760800080702F1080236EE267A00F10800E4EED7
:10761800877AE5EE475A67EEA37A25EEA37AC0ED9E
:10762800007A80ED017AD1D1BEF1140F7EF417AF44
:1076380006F082F9069BDFF80081C01AA8F802005C
:10764800D4F81451FEF70BBFD4F81831B4F810C1B0
:10765800354ACCF120095FFA89F90CEB431702EBA4
:1076680087075FEA990201F0F285013216012F4877
:107678002F4907EB060807F1100212ED024A12ED36
:10768800035A12ED016A12ED047A50ED024A50EDE8
:10769800035A50ED016A50ED047A64EE244A65EE0F
:1076A800255A66EE266A67EE277A1032904541ED34
:1076B800024A41ED035A41ED016A41ED047A00F1B5
:1076C800100001F11001D8D11A48A6F110010F4499
:1076D80000EB0108214419F0030209D0B7EC017A44
:1076E800F8EC017A67EE277A013AE1EC017AF5D1F4
:1076F800BCF1000F41F03180BEF1140F7EF4AFAE43
:1077080006F01AF9069BDFF83080D4F81451C01A35
:10771800A8F80200FEF7A3BEDC270020E838002006
:10772800503D0020C8160020683D0020F83E00208B
:10773800D8160020E83E0020344D0020D04E318875
:1077480073684FEA51094FEA89005FEAD10C04EBEC
:10775800000204EB810500F0A18000F110010CF19A
:10776800010CC84F02EB0C1C2944103203F1100E17
:1077780005F1100050ED032A50ED043A17ED043AD4
:1077880017ED032A50ED026A10ED016A17ED021A8F
:1077980057ED010A11ED044A11ED035A52ED044A5E
:1077A80052ED035A12ED027A52ED017A51ED021AA6
:1077B80011ED010A73EE238A32EE228A47ED048A1C
:1077C80007ED038A71EE268A30EE868A47ED028A33
:1077D80007ED018A74EE848A35EE858A42ED048AC3
:1077E80002ED038A77EE218A37EE808A42ED028A1B
:1077F80002ED018A73EE633A75EE655A1EED035A7F
:1078080032EE623A74EE644A25EE638A1EED044A4B
:1078180023EE052A64EE652AA3EE048A1032944505
:1078280024EE843AA3EE842A07F110070EF1100E15
:10783800A5EE853A00F1100001F11001E4EE852A69
:1078480000ED078A00ED082A01ED073A41ED082A04
:107858005EED055A1EED065A71EE666A30EEC66A8E
:1078680031EEC77A70EE677A26EE253A65EEE63A8B
:1078780025EE674A67EE054AE6EE053AA6EE853A32
:10788800A7EE254AE7EEA54A00ED063A40ED053A8F
:1078980001ED064A41ED054A7FF46CAF1FFA89F9FC
:1078A8001A46494678481EF085FC726849462846BB
:1078B8001EF080FC059B1A78142A7FF4C1AEB7E647
:1078C800D4F8185171497248724BEA0011441544B2
:1078D8008A88196800EE102A643AC82AA8BFC82204
:1078E800782AB8BF782207EE902AB8EEC07AF8EE68
:1078F800E77A00EB850577EE670A77EE876A67EE29
:10790800877A20EEA67AB8EE400AC7EE870A28469C
:10791800D5F81490D5F81880EF692E6A1FF01AF977
:10792800059BC5F8149093F800E0C5F81880BEF1DF
:10793800140FEF612E6201F0A484D4F81821564B7D
:10794800D4F81451013283FB0213A3EBE27303EB67
:107958004303D31A0135C4F81831C4F8145175E635
:10796800474E4948B268B18927F0ACFC059B93F8AB
:1079780000E0BEF1140F01F09184D4F814510135E0
:10798800C4F81451FFE5454E31785FEA910C01F0D7
:10799800AC85434F0CF101094FEA491907EB090877
:1079A80007F12002A7F1700012ED076A52ED056A8F
:1079B80012ED037A52ED017A52ED025A12ED084A9D
:1079C80052ED064A12ED045A26EE066A66EEA66ADB
:1079D80027EE077A67EEA77AA4EE046A203290456C
:1079E800E4EEA46A00F11000A5EE057AE5EEA57AAA
:1079F800F1EEC65AB1EEE66AF1EEC76AB1EEE77A81
:107A080040ED085A00ED076A40ED066A00ED057A78
:107A1800CAD1A9F120023A4404EB0C1711F0030073
:107A280018BF08320FD052ED017A12ED027A67EED4
:107A3800A77A0138E7EE077A02F10802B1EEE77A91
:107A4800A7EC017AEFD1BEF1140F01F00A840135D9
:107A5800C4F81451FEF772BC05F06EFF059B069042
:107A680093F800E0BEF1140F05BFDFF83880D4F8B2
:107A78001451D4F81451A8F80050FDF756B800BFB7
:107A8800503D0020D8160020C81600204040002095
:107A9800C05700202C580020565555554A3D002007
:107AA80048170020344D0020306E99BC2716983DA9
:107AB800A40DC93F843459BEDB0F4940D06D393A13
:107AC80000000000F0EEE76AB7EE005A35EE665A9D
:107AD8001FED0B4A5FED0B5A1FED0A6A1FED0C7A7A
:107AE80094ED6B0AF1EEC54AE6EE845AF5EEC07ADB
:107AF800A6EEA56AF1EE10FAA6EE867A48BF5FED0B
:107B0800127A27EE247A48BF37EEC77A27EE000AA2
:107B180028F0E0FCB0F5617F00F38D8607EE900A4F
:107B2800F8EEE76A5FED1B7A66EEA76A07EE905AF1
:107B3800BDEEE67AF8EEE77A17EE103A2033402BDE
:107B480041F281841FED220A28F0C4FC00B207EE3E
:107B5800900AB8EEE77AFFF7BEBAC249C24B896805
:107B68001B6899423FF696AA3B780C3B022B7EF69F
:107B7800A3A9BE4C3A702378002B3EF49DA900239C
:107B88002370FEF799B9BA4A02F1500503E00432AE
:107B9800954200F069821378262BF8D19678D3782D
:107BA8009E42F4D2FFF7EDBAB24DB34F95ED004ABD
:107BB80095ED057AD5ED014A95ED066AD5ED046A8D
:107BC80095ED035AD5ED025A67EE897A07EB8602DE
:107BD800A4EE277AA4EEA76A66EEC76AA5EE476AFE
:107BE800E5EEA76A20EE070A85ED056AC5ED066A87
:107BF80082ED007A29EE088A28F06CFC69EE288A62
:107C0800D5ED0E5AD5ED176A95ED091AD5ED121A6C
:107C180095ED0F5A95ED187A95ED0A2AD5ED132AA8
:107C280095ED0D6AD5ED167A95ED0C3AD5ED0B3A32
:107C380095ED154AD5ED144AE1EE085A002207EBF6
:107C48008601E8EEA16A00B2C4F80021A2EE085A43
:107C5800C4F80421C4F80821A8EEA27A26EE656AC1
:107C680067EEE67AA3EE655AA3EE886AA6EEC47AB2
:107C7800E8EEA47A85ED0E5AC1ED205A85ED0F6A1B
:107C8800C1ED406A85ED177AC5ED187AFEF710BB8D
:107C9800D4F89C51079B5D1BFEF710BABBF938203E
:107CA800CBF8201007EE902A0121F8EEE77ACBF8FE
:107CB8006020CBF87C100022012FCBED1C7ACBED95
:107CC8001B7ACBF8742001F09D82B7427CF491AF07
:107CD800BBF93A20CBF8642007EE902A0021012254
:107CE800F8EEE77ACBF82410CBF890200022012F89
:107CF800CBED217ACBED207ACBF8882001F0868273
:107D0800B7427CF4AAAFBBF93C20CBF8682007EE59
:107D1800902A00210122F8EEE77ACBF82810CBF858
:107D2800A4200022012FCBED267ACBED257ACBF8C3
:107D38009C207CF4C6AF9FED518A032D49D04CB1ED
:107D480007EE904AF8EEE77AF4EEC87AF1EE10FA08
:107D580001F1D0834A4A4B4C1168DBF86820A8F837
:107D6800060094F8200102EB560292FBF6F6002278
:107D7800CBF828608A620A63CA6228B1424A12684C
:107D880032F480637CF4A0AF404A126812F40032E7
:107D980041F030823E481146835C012B02F10C020F
:107DA80000F0778301311829F6D1FCF78DBF3949E6
:107DB8004B69002B3DF46DA83748384B008893FB7E
:107DC800F0F00B684FF0010E186081F811E0FDF734
:107DD80060B8B0EE480A28F07DFB00B2AFE720F0AB
:107DE800EFFA2F4A0292A2F10C0325210193009188
:107DF800A2F10A035021163A492018F033F9A8B91C
:107E0800284BAA7818604FF0FF31596007233B7060
:107E1800FFF73DB9DFF88C8020F0D2FA224AD8F873
:107E28000430126864339342C1F07C83AA78FFF768
:107E38002EB91E4B1B78D90701F16A831F200EF05B
:107E480083FA0028F2D00C233B70EFE71F2006923C
:107E58000EF07AFA069A00287FF419A901233B70DC
:107E6800FFF715B99C060020F43A00200F3B0020CC
:107E7800D4330020D43F0020683D002000000000DB
:107E88006C460020C81600207445002018370020D2
:107E9800183203082C4700204447002020A107007F
:107EA800421A0308983A00204C470020C04C002092
:107EB8001A200EF049FA00283FF4E6A89B4B1B88CD
:107EC800002B7FF4E1A89A4B4520D3F8008020F0DE
:107ED8003FFB0E2020F03CFB404617F019F8DDF878
:107EE8001C80404617F014F8924A934B12681A60A7
:107EF80040460A233B7017F0D5F8FFF7C5B8012AAA
:107F080001D1F9F721FC0D2313203B7010F034FE4A
:107F1800AA78FFF7BCB8894B89495B680968C833F8
:107F28008B4205D320F072FAAA7800283FF4AFA854
:107F3800032A93D1DFF84082D8F8000010F020F926
:107F4800804B1B780022022BC8F8002001F0118416
:107F5800AA7883E7012A01F0D4820E2313203B700C
:107F680010F00AFE62E720F02BFA17F07FFB0028DA
:107F78003FF45CAF20F04AFA00283FF457AF6D4A4F
:107F88006D4B12681A600A233B70AA78FFF77FB816
:107F980020F016FA6C4B002105208DE80300A3F1B0
:107FA80008020291532018F05DF800287FF43EAFD4
:107FB800624BAA78186008233B70FFF768B8604BDB
:107FC8005E491B684B60614800230B600321036016
:107FD8003970FFF75CB8DFED5E7A5E4B94ED687A36
:107FE800C3ED007AC3ED017AC3ED027A5A4BF0EE85
:107FF800674AF0EE673A1968FDF746B9574A584D8F
:10800800D2ED006A574A95ED006A1278C4ED646AA9
:1080180084ED656A002A00F01F8276EE665A94F9AC
:108028009821C4ED615A0132C4ED626A00F0898575
:10803800079BC4F89C31002537EE677AFCEEE77A97
:10804800494E84ED687A17EE902AA4F88C21FF2215
:1080580096ED005A84F89821FEF740B8434B1D78F6
:1080680005F00108FDF7AEBC3C4A3D4DD2ED007A63
:108078003C4A95ED007A1278C4ED647A84ED657A0D
:10808800002A00F0658377EE676A94F99821C4EDB9
:10809800616A0132C4ED627A00F0DB86079BC4F89E
:1080A8009C3100259FED2A7A2F4E84ED687AFF22B5
:1080B80096ED005A84F89821FEF710B82C49DFEDA8
:1080C8002D7A0968C4ED4C7A11F080530A9340F078
:1080D800A683DAF8001011F480030A9300F0CF8128
:1080E80000230A93B6EE007A67EE877AF4EEE57A13
:1080F800F1EE10FAC8BFF0EE675A40F39083C4ED72
:10810800685AFDF70BBB73EEE77AB7EE007AF4EE28
:10811800C77AF1EE10FAC4ED4C7A41F38F8084EE01
:10812800A77A8DED0E7AFDF7EEBA00BF2839002048
:10813800243900200C39002008390020983A002002
:108148004C470020EC3A0020F01B0308284C002084
:1081580000000000C03800207C4500203C39002089
:1081680060280020605A002074280020C04C00209D
:1081780018390020000000802C4C0020D14D0D9BA8
:108188009DED0E5A95ED006A002B00F01B8725EE39
:10819800866ACD48A5EE076AB0EE675AA6EE265A5B
:1081A800BDEEC56A16EE10EA16EE107AE645A8BFCF
:1081B80067467145C8BF0F4606EE107AB8EEC66A24
:1081C800012A80ED006A3DF401AC95ED046A9DED4D
:1081D8000F5A25EE866AA5EE076AB0EE675AA6EE34
:1081E800265ABDEEC56A16EE10EA16EE107AE64576
:1081F800A8BF67467145C8BF0F4606EE107AB8EEAD
:10820800C66A022A80ED016A3DF4E0AB95ED086A82
:108218009DED105A25EE866AA5EE076AB0EE675AFC
:10822800A6EE265ABDEEC56A16EE10EA16EE107ACC
:10823800E645A8BF67467145C8BF0F4606EE107AE7
:10824800B8EEC66A032A80ED026A3DF4BFAB95ED2D
:108258000C6A9DED115A25EE866AA5EE076AB0EE06
:10826800675AA6EE265ABDEEC56A16EE10EA16EE55
:10827800107AE645A8BF67467145C8BF0F4606EEA7
:10828800107AB8EEC66A042A80ED036A3DF49EAB04
:1082980095ED106A9DED125A25EE866AA5EE076ADD
:1082A800B0EE675AA6EE265ABDEEC56A16EE10EA7B
:1082B80016EE107AE645A8BF67467145C8BF0F4657
:1082C80006EE107AB8EEC66A052A80ED046A3DF417
:1082D8007DAB95ED146A9DED135A25EE866AA5EEE1
:1082E800076AB0EE675AA6EE265ABDEEC56A16EEC4
:1082F80010EA16EE107AE645A8BF67467145C8BF72
:108308000F4606EE107AB8EEC66A062A80ED056AB0
:108318003DF45CAB95ED186A9DED145A25EE866A1E
:10832800A5EE076AB0EE675AA6EE265ABDEEC56AF4
:1083380016EE10EA16EE107AE645A8BF67467145B4
:10834800C8BF0F4606EE107AB8EEC66A072A80ED57
:10835800066A3DF43BAB95ED1C6A9DED155A65EE3A
:10836800865AE5EE075AE6EEA57AFDEEE77A17EEAD
:10837800902A9445A8BF94468A42A8BF614607EE52
:10838800901AF8EEE77AC0ED077AFDF71FBBBEF149
:10839800010F7FF7D0AC07EE103AB8EEC77AC7EEF8
:1083A800876AB1EEE68AC8E4BEF1010F40F32E8772
:1083B80007EE103AB8EEC77AC7EE876AB1EEE68ADA
:1083C800032D13D04CB107EE904AF8EEE77AF4EE9D
:1083D800C87AF1EE10FA01F18D80DBF8642002EB27
:1083E800560292FBF6F2CBF8242089E4B0EE480A54
:1083F80028F070F800B2E5E7BEF1010F40F30287FC
:1084080007EE103AB8EEC77AC7EE876AB1EEE68A89
:10841800032D13D04CB107EE904AF8EEE77AF4EE4C
:10842800C87AF1EE10FA01F16580DBF8602002EB02
:10843800560292FBF6F2CBF8202046E4B0EE480A4A
:1084480028F048F800B2E5E7F7EE006AFDF78EBCC1
:10845800F7EE006AFDF704BD76EEC65AF0EE466AFE
:10846800DDE58222FDF7E8BFDFED187AFDF7B0BF42
:10847800174BD3F800E0BEF93270FEF75EBAB6EEDD
:10848800007AF4EEC75AF1EE10FA3FF72BAEFDF77B
:1084980045B9D4F824614A003EB1551800EB85056A
:1084A80076786D78B542BCF40FAC0A4400EB8200D4
:1084B8000022C4F82401A4F81022C4F81422FCF7FE
:1084C80003BC00BFDC270020E8380020000002437E
:1084D8007C45002095ED006A9DED0E4AE34825EEA7
:1084E800866AFDEEE43AA4EE076AB0EE674AA6EEA5
:1084F800264A13EE901AB4EEC45AF1EE10FAB0EE12
:10850800446A88BFB0EE646ABDEEC66A16EE10EA29
:1085180016EE107AE645A8BF67467145C8BF0F46F4
:1085280006EE107AB8EEC66A012A80ED006A3DF4BC
:1085380049AA95ED046A9DED0F4A25EE866AA4EED8
:10854800076AB0EE674AA6EE264AB4EEC45AF1EEC0
:1085580010FAB0EE446A88BFB0EE646ABDEEC66A2F
:1085680016EE10EA16EE107AE645A8BF67468E4565
:10857800B8BF0F4606EE107AB8EEC66A022A80ED3A
:10858800016A3DF41FAA95ED086A9DED104A25EE93
:10859800866AA4EE076AB0EE674AA6EE264AB4EEEB
:1085A800C45AF1EE10FAB0EE446A88BFB0EE646ABD
:1085B800BDEEC66A16EE10EA16EE107AE645A8BFBA
:1085C80067468E45B8BF0F4606EE107AB8EEC66A03
:1085D800032A80ED026A3DF4F5A995ED0C6A9DED3C
:1085E800114A25EE866AA4EE076AB0EE674AA6EE3F
:1085F800264AB4EEC45AF1EE10FAB0EE446A88BFC7
:10860800B0EE646ABDEEC66A16EE10EA16EE107A8F
:10861800E645A8BF67468E45B8BF0F4606EE107AF6
:10862800B8EEC66A042A80ED036A3DF4CBA995ED3D
:10863800106A9DED124A25EE866AA4EE076AB0EE2E
:10864800674AA6EE264AB4EEC45AF1EE10FAB0EE26
:10865800446A88BFB0EE646ABDEEC66A16EE10EAD8
:1086680016EE107AE645A8BF67468E45B8BF0F4696
:1086780006EE107AB8EEC66A052A80ED046A3DF463
:10868800A1A995ED146A9DED134A25EE866AA4EE1C
:10869800076AB0EE674AA6EE264AB4EEC45AF1EE6F
:1086A80010FAB0EE446A88BFB0EE646ABDEEC66ADE
:1086B80016EE10EA16EE107AE645A8BF67468E4514
:1086C800B8BF0F4606EE107AB8EEC66A062A80EDE5
:1086D800056A3DF477A995ED186A9DED144A25EED3
:1086E800866AA4EE076AB0EE674AA6EE264AB4EE9A
:1086F800C45AF1EE10FAB0EE446A88BFB0EE646A6C
:10870800BDEEC66A16EE10EA16EE107AE645A8BF68
:1087180067468E45B8BF0F4606EE107AB8EEC66AB1
:10872800072A80ED066A3DF44DA995ED1C6A9DED7A
:10873800154A65EE865AE7EE045AE6EEA57AB4EED7
:10874800E75AF1EE10FAC8BFF0EE647AFDF72AB9DD
:1087580077EEC76AF0EE477A97E4454A4FEA890709
:108768005FEA9C09384402EBC313274437D009F168
:1087780001094FEA091903EB090803F1100200F196
:10878800100607F1100112ED024A12ED035A12ED1C
:10879800016A12ED047A56ED024A56ED035A56ED77
:1087A800016A56ED047A64EE244A65EE255A66EEAF
:1087B800266A67EE277A1032904541ED024A41ED6C
:1087C800035A41ED016A41ED047A06F1100601F100
:1087D8001001D8D1A9F110094B4448444F441CF06A
:1087E800030C3EF489AFB3EC017AF0EC017A67EE42
:1087F800277ABCF1010CE7EC017AF4D1FEF77CBFD3
:10880800BEF834309FED1B7A07EE903AF8EEE77A1F
:10881800194B67EE877AC3ED007AFDF725B9B7EEF5
:10882800007A77EE677AF4EEE75AF1EE10FA88BF2D
:10883800F0EE675A63E407EE905ADFED106AF8EE3F
:10884800E77A66EEA65A9FED0E5A9FED0E6A9FEDE7
:108858000E7AA5EE856A26EEA55AA5EE867AE5EE8D
:10886800076A26EEA70AFFF76FB900BFE8380020AD
:10887800683D00206F12833A0000002084F9223FEF
:1088880092E741B99730083C15A82ABE95ED006AD1
:108898009DED0E4ACC4825EE866AFDEEE43AA4EE3C
:1088A800076AB0EE674AA6EE264A13EE907AB4EE4F
:1088B800C45AF1EE10FAB0EE446A88BFB0EE646AAA
:1088C800BDEEC66A16EE10EA16EE101AE645A8BF07
:1088D80061467745C8BF394606EE101AB8EEC66A33
:1088E800012A80ED006A3DF4E0AF95ED046A9DED44
:1088F8000F4A25EE866AA4EE076AB0EE674AA6EE2E
:10890800264AB4EEC45AF1EE10FAB0EE446A88BFB3
:10891800B0EE646ABDEEC66A16EE10EA16EE101ADC
:10892800E645A8BF6146BE45B8BF394606EE101AEF
:10893800B8EEC66A022A80ED016A3DF4B6AF95ED3D
:10894800086A9DED104A25EE866AA4EE076AB0EE25
:10895800674AA6EE264AB4EEC45AF1EE10FAB0EE13
:10896800446A88BFB0EE646ABDEEC66A16EE10EAC5
:1089780016EE101AE645A8BF6146BE45B8BF39468F
:1089880006EE101AB8EEC66A032A80ED026A3DF4B4
:108998008CAF95ED0C6A9DED114A25EE866AA4EE22
:1089A800076AB0EE674AA6EE264AB4EEC45AF1EE5C
:1089B80010FAB0EE446A88BFB0EE646ABDEEC66ACB
:1089C80016EE10EA16EE101AE645A8BF6146BE4537
:1089D800B8BF394606EE101AB8EEC66A042A80ED0A
:1089E800036A3DF462AF95ED106A9DED124A25EEDB
:1089F800866AA4EE076AB0EE674AA6EE264AB4EE87
:108A0800C45AF1EE10FAB0EE446A88BFB0EE646A58
:108A1800BDEEC66A16EE10EA16EE101AE645A8BFB5
:108A28006146BE45B8BF394606EE101AB8EEC66AAA
:108A3800052A80ED046A3DF438AF95ED146A9DED82
:108A4800134A25EE866AA4EE076AB0EE674AA6EED8
:108A5800264AB4EEC45AF1EE10FAB0EE446A88BF62
:108A6800B0EE646ABDEEC66A16EE10EA16EE101A8B
:108A7800E645A8BF6146BE45B8BF394606EE101A9E
:108A8800B8EEC66A062A80ED056A3DF40EAF95ED8C
:108A9800186A9DED144A25EE866AA4EE076AB0EEC0
:108AA800674AA6EE264AB4EEC45AF1EE10FAB0EEC2
:108AB800446A88BFB0EE646ABDEEC66A16EE10EA74
:108AC80016EE101AE645A8BF6146BE45B8BF39463E
:108AD80006EE101AB8EEC66A072A80ED066A3DF45B
:108AE800E4AE95ED1C6A9DED154A65EE865AE7EEF3
:108AF800045AE6EEA57AB4EEE75AF1EE10FAC8BFCA
:108B0800F0EE647AFDEEE77A17EE901A8C45A8BF6E
:108B18008C468F42D8BF674607EE907AF8EEE77A20
:108B2800C0ED077AFDF7BEBE28494A69002A3CF421
:108B380099AA0A6813604B74FCF794BA244DFDF7A0
:108B48000BB8D4F89C51079B5D1BFFF775BA214BF6
:108B58001B78DA0704D40DF09FFA002840F06885E6
:108B68001D4DD4F80C222B689A423EF69AAA3B78FF
:108B7800012B3DF4A1A9194C2278002A3DF49CA9A7
:108B88000B2B19D801229A4040F6030112EA01087A
:108B98007EF4F5AF12F4C06F0ED0093B012B0BD851
:108BA80045201FF0D5FCFF201FF0D2FC0C481FF019
:108BB80041FC40461FF0CCFC0A4B2A685A600B2344
:108BC8003B70FEF7DCBF00BFE83800202C470020D0
:108BD800584D0020C04C00204C4700200F3B00207F
:108BE800C0420308983A00200D9B002B00F07183C7
:108BF800E34D9DED0E4A95ED006A089B25EE866AC9
:108C0800A4EE076AB0EE674AA6EE264AB0EE446ABA
:108C180033B1B4EE445AF1EE10FAC8BFB0EE646A4C
:108C2800FDEEE44ABDEEC66A14EE907A16EE101A0E
:108C38008F4214EE90EA00F3F3846145A8BF6146C1
:108C480006EE101ACF48B8EEC66A012A80ED006A0F
:108C58003CF4BCAE95ED046ADDED0F4A089B25EEA9
:108C6800866AA4EE876AF0EE674AE6EE264AB0EE18
:108C7800646A002B00F0CA84B4EEE45AF1EE10FAEC
:108C880040F3C48439466145A8BF614606EE101A10
:108C9800B8EEC66A022A80ED016A3CF497AE95EDFB
:108CA800086ADDED104A089B25EE866AA4EE876AFD
:108CB800F0EE674AE6EE264AB0EE646A002B00F052
:108CC8009B84B4EEE45AF1EE10FA40F395843946E9
:108CD8006145A8BF614606EE101AB8EEC66A032AB7
:108CE80080ED026A3CF472AE95ED0C6ADDED114A36
:108CF800089B25EE866AA4EE876AF0EE674AE6EEE0
:108D0800264AB0EE646A002B00F06C84B4EEE45A94
:108D1800F1EE10FA40F3668439466145A8BF614612
:108D280006EE101AB8EEC66A042A80ED036A3CF40F
:108D38004DAE95ED106ADDED124A089B25EE866A68
:108D4800A4EE876AF0EE674AE6EE264AB0EE646A59
:108D5800002B00F03D84B4EEE45AF1EE10FA40F333
:108D6800378439466145A8BF614606EE101AB8EE49
:108D7800C66A052A80ED046A3CF428AE95ED146AAB
:108D8800DDED134A089B25EE866AA4EE876AF0EEAD
:108D9800674AE6EE264AB0EE646A002B00F00E84BD
:108DA800B4EEE45AF1EE10FA40F30884394661450E
:108DB800A8BF614606EE101AB8EEC66A062A80ED0C
:108DC800056A3CF403AE95ED186ADDED144A089B7C
:108DD80025EE866AA4EE876AF0EE674AE6EE264A32
:108DE800B0EE646A002B00F0E083B4EEE45AF1EED2
:108DF80010FA40F3DA8339466145A8BF614606EEAA
:108E0800101AB8EEC66A072A80ED066A3CF4DEAD91
:108E180095ED1C6ADDED154A089B65EE865AE4EE71
:108E2800875AE5EEA67A002B00F0B783F4EEC57AF0
:108E3800F1EE10FA40F1B1833A466245A8BF6246A6
:108E4800964607EE90EAF8EEE77AC0ED077AFCF767
:108E5800BDBDD4F89C51079B5D1BFFF723B907EEF6
:108E6800905ADFED496A9FED497A84F80452F8EE8A
:108E7800E77A67EEA67A77EE876ABDEEE66A16EEBF
:108E8800103A2033402B40F29782DFED416A414B84
:108E9800BDEEE77AC3ED016A17EE103A2033402B96
:108EA80000F260829FED3C7AF4EEC77AF1EE10FA98
:108EB80040F3CA83DFED395A9FED396A01E0F0EEDD
:108EC800477AF4EEC67AF1EE10FA37EEE57AF6DC78
:108ED800DFED347AB4EEE77AF1EE10FA40F1B183BF
:108EE800DFED2E5A9FED306A01E0B0EE677AB4EEFE
:108EF800C67AF1EE10FA77EE257AF6D49FED237A4A
:108F0800F4EEC77AF1EE10FA40F3E3829FED227A8D
:108F180077EE677A67EEA75A9FED245A9FED246A89
:108F28009FED247AA5EE856A27EEA55AA5EE867AE6
:108F3800E5EE077AC4ED827AFDF77ABD95ED000A71
:108F48000893069227F0C6FA1B49DFF870E0D1F8BB
:108F5800EC10DFF86CC0069AACF800008EFB013EFE
:108F6800C917C1EBAE1107EE901AF8EEE77A089B25
:108F7800FDEEE77A17EE901AACF80210FCF7F1BD97
:108F8800DC270020E838002035FA8E3CDB0FC93F8B
:108F98000000000000000020DB0F4940DB0FC94043
:108FA800E4CB1641DB0F49C0E4CB16C192E741B9C7
:108FB8009730083C15A82ABE20010020D34D621026
:108FC800344D002025EE866AA5EE076AB0EE675A92
:108FD800A6EE265ABDEEC56A16EE100A814200F3C7
:108FE8006C816045A8BF604606EE100A0A9BB8EE81
:108FF800C66A002B00F01084DC48012A80ED006A64
:109008003CF4E4AC95ED046A9DED0F5A25EE866AB2
:10901800A5EE076AB0EE675AA6EE265ABDEEC56AF7
:1090280016EE107AB94200F346816745A8BF674635
:1090380006EE107A0A9BB8EEC66A002B00F0A983E8
:10904800022A80ED016A3CF4C1AC95ED086A9DEDF9
:10905800105A25EE866AA5EE076AB0EE675AA6EEA4
:10906800265ABDEEC56A16EE107AB94200F32D8174
:109078006745A8BF674606EE107A0A9BB8EEC66A2F
:10908800002B00F0A483032A80ED026A3CF49EAC16
:1090980095ED0C6A9DED115A25EE866AA5EE076AD4
:1090A800B0EE675AA6EE265ABDEEC56A16EE107ADD
:1090B800B94200F308816745A8BF674606EE107AF3
:1090C8000A9BB8EEC66A002B00F07783042A80ED6D
:1090D800036A3CF47BAC95ED106A9DED125A25EEBF
:1090E800866AA5EE076AB0EE675AA6EE265ABDEE66
:1090F800C56A16EE107AB94200F3E3806745A8BF47
:10910800674606EE107A0A9BB8EEC66A002B00F096
:10911800B182052A80ED046A3CF458AC95ED146AD6
:109128009DED135A25EE866AA5EE076AB0EE675ADA
:10913800A6EE265ABDEEC56A16EE107AB94200F3BD
:10914800BE806745A8BF674606EE107A0A9BB8EE50
:10915800C66A002B00F02783062A80ED056A3CF4D6
:1091680035AC95ED186A9DED145A25EE866AA5EE84
:10917800076AB0EE675AA6EE265ABDEEC56A16EE25
:10918800107AB94200F3A3806745A8BF674606EE88
:10919800107A0A9BB8EEC66A002B00F07582072A7F
:1091A80080ED066A3CF412AC95ED1C6A9DED155AEB
:1091B80065EE865AE7EE055AE5EEA67AFDEEE77A01
:1091C80017EE902A914203DC6245A8BF6246114619
:1091D80007EE901A0A9BF8EEE77A002B7FF435AE7B
:1091E8000C9B002B7FF431AE0B9B9E45B8BFF0EE75
:1091F800647A2AE65E4A1278032A00F01582002271
:10920800FEF7C8BD9FED5B8AFFF702B99FED598A4B
:10921800FFF7D6B89FED580ADFF8708125EE800A6F
:1092280027F058F9D4F81451A8F80600FDF717B933
:10923800D4F89C51079B5D1BFDF7C0BF4F490968D7
:1092480011F080530A937EF44DAFFEF742BF4C48AD
:109258004C498046FEF73FBA079815F023FFFDF703
:1092680013BF04F069FB059BDFF8208193F800E049
:10927800069B3178D4F81451C01AA8F80400FEF7F8
:10928800E6BB04F059FB059BDFF8008193F800E08A
:10929800069BC01AA8F80200FEF74FBB04F04CFB6F
:1092A800059BDFF8E88093F800E0069BC01AA8F851
:1092B8000200FEF762BB0F46BAE6084694E60F4680
:1092C80042E70F461DE70F46F8E60F46D3E60F467E
:1092D8005DE70EA9BDEEE46A01EB820290462A48DA
:1092E800089A224D0A9B089416EE107A05E041452B
:1092F800A5EC016A00F1100031D090ED006AB1ECE4
:10930800014A25EE866AA7EE046AB0EE674AA6EE21
:10931800864AB0EE446A32B1B4EE445AF1EE10FA1D
:10932800C8BFB0EE646ABDEEC64A06EE107A14EE07
:10933800104AA74206DC14EE104A6445A8BF6446EA
:1093480006EE104AB8EEC66A002BD0D10C9C002C51
:10935800CDD10B9CA645B8BFB0EE646AC7E7089CA0
:10936800FCF734BBDFED037AE4E500BFE838002002
:10937800134F0020000000000000C84218390020E8
:10938800E83E0020C8160020DC270020344D0020CD
:1093980092E741B99730083C15A82ABEE4CB16419C
:1093A800DB0FC940E4CB16C1DB0FC93FDB0F4940D7
:1093B800DB0FC9BFDB0F49C0F4EEC77AF1EE10FA34
:1093C80040F355815FED0A5A1FED0C6A01E0F0EE9B
:1093D800476AF4EEC66AF1EE10FA36EEE57AF6DC84
:1093E8005FED0C6AB4EEE67AF1EE10FA40F12F81E7
:1093F8005FED155A1FED156A01E0B0EE667AB4EE1E
:10940800C67AF1EE10FA77EE256AF6D41FED1A7ACD
:10941800F4EEC76AF1EE10FA40F3B3801FED1D7A3F
:1094280077EE666A66EEA65A1FED275A1FED276A81
:109438001FED277AA5EE856A26EEA55AA5EE867A4F
:10944800E5EE076A23E51FED277AF4EEC76AF1EE29
:1094580010FA40F39B815FED2E5A1FED306A01E050
:10946800F0EE476AF4EEC66AF1EE10FA36EEE57AE7
:10947800F6DC5FED306AB4EEE67AF1EE10FA40F110
:1094880082815FED395A1FED396A01E0B0EE667AE4
:10949800B4EEC67AF1EE10FA77EE256AF6D41FED2F
:1094A8003E7AF4EEC76AF1EE10FA05DD1FED417A57
:1094B80077EE666AFFF7C5B91FED437AF4EEC76A1F
:1094C800F1EE10FA44BF1FED457A77EE666AFFF7B2
:1094D800B8B91FED497AF4EEC77AF1EE10FA44BF35
:1094E8001FED4C7A77EE677A14E5D14F07F18002C9
:1094F800FEF794BAA8F80600ABF8A860CC4CFBF7C6
:10950800EABBF7F79DFF00283EF490ACFEF725BDB7
:10951800802024F001FF08B10EF05EFE16F06CFE0C
:10952800FEF78CBC40201EF021FF00287EF47EACA4
:10953800D8F80030DFF844A3DFF844B34FF040090F
:109548000EE01FF005F8DBF80020D8F80030013AEB
:109558000133B9F10109CBF80020C8F8003079D0FF
:109568001AF803301846002BEBD100234FF0FF32D6
:10957800C8F800300423C8F804203B70AA78FDF727
:1095880086BD9FEDAC7AF4EEC76AF1EE10FA44BFDF
:109598009FEDA97A77EE666A44E7FDEEE77A17EE63
:1095A800902ABA42FFF64DAC47E4BDEEC66A16EE05
:1095B800101AB942BFF620AC394620E4BDEEC66A9F
:1095C80016EE101AB942BFF6F2AB3946FFF7F2BBF6
:1095D800BDEEC66A16EE101AB942BFF6C3AB3946DD
:1095E800FFF7C3BBBDEEC66A16EE101AB942BFF646
:1095F80094AB3946FFF794BBBDEEC66A16EE101A57
:10960800B942BFF665AB3946FFF765BBBDEEC66A22
:1096180016EE101AB942BFF636AB3946FFF736BB1D
:1096280014EE901AFFF70CBB0FF08AFAFBF74CBB4D
:10963800824B1B6803F59C530833C4F80C32FDF7C2
:1096480030BDF0EE477A59E4B0EE677A40E4F0EEC8
:10965800476ADBE61AF80330002B7EF4E7AB84E7B1
:1096680094F87831002B7BF4CBADFBF7B6BDB0EEA8
:10967800667AB5E60C9B002B7FF44BAD0B9B9E45A1
:10968800B8BFB0EE646A44E50C9B002B7FF487AD4D
:109698000B9B9E45B8BFB0EE646A80E5684A694B8B
:1096A80010681B689847684BD7ED006A93ED007AFD
:1096B800664BD3ED007A664B83ED020A654B67EE85
:1096C800277A2B4427EEAC7AD3ED007A624B67EE0B
:1096D800277AF0EE665AEDEEA75A93ED006AB1EEDE
:1096E800467AB4EEE57AF1EE10FA08DCF4EEC65AE2
:1096F800F1EE10FA8CBFB0EE467AB0EE657A574BB1
:109708001B78012B02D0192B7BF4E4ACDFED547AE3
:10971800F4EEE7DAF1EE10FACCBF01230023FBF7F1
:10972800E4BCDFED507AB4EEE7EAF1EE10FA27DC9C
:10973800DFED4D7AB4EEE7EAF1EE10FA20D44B4BA8
:10974800D3ED007AB1EE677AF4EEC7DAF1EE10FAEB
:1097580013D4F4EEE7DAF1EE10FA88BFF0EE67DA28
:10976800434B87ED00CA1B689342BBF6A1ABFBF7DE
:1097780005BC0FF03FF9FEF7EBBBF0EE47DAEFE779
:10978800DFED3CDAECE7F0EE476A88E6B0EE667AA1
:109798006FE60C9B002B7FF453AC0B9B9E45B8BF28
:1097A800B0EE646A4CE40C9B002B7FF4D5AC0B9BA9
:1097B8009E45B8BFB0EE646ACEE40C9B002B7FF4E4
:1097C80085AC0B9B9E45B8BFB0EE646A7EE40C9BEB
:1097D800002B7FF458AC0B9B9E45B8BFB0EE646A73
:1097E80051E4132B05D1B0EE480A26F073FE099B0D
:1097F8001880B0EE480ADBF808321F489847059BE6
:109808001B78132BB0EE408A7CF4E1AE26F062FEA2
:10981800099B5880FCF7DBBE0C9B002B7FF4ECAB5C
:109828000B9B9E45B8BFB0EE646AFFF7E5BB00BF6F
:10983800C8160020DB0FC9BFDB0F49C04C4700200A
:10984800482700205C270020000000209C260020DC
:10985800B43800206C270020D42700200C420020B8
:109868000000964200C0F84400C0F8C4D027002089
:10987800B427002000000000C0570020DC190308AE
:10988800284C00202DE9F04F2DED068BA04BA14A66
:109898001C7897B000F59C41203181460B911160EE
:1098A800002C00F0E2869C4A1268904240F28380C5
:1098B8009A4A069216689A499A4A0591013C1C7080
:1098C800994B049206F480560893002E40F081804C
:1098D800964B1B78022B01F02481042B01F0928116
:1098E800012B01F04681924B9945089B9B7800F229
:1098F8008D85002B40F08E858E4B0793069B1E6846
:1099080016F4805740F07F86DFF860A2049BB3F915
:109918000610059B5D8BA942B4BF00250125864B27
:109928001B6813F080535ED0079A127812F0010278
:109938005FD00598408C884241F3D182002D5ED1DA
:109948007E4C94F88C10002959D17D487D490068D7
:1099580090F82D0000240C604C608C607A49002837
:109968004ED10870002A4FD0F0064DD5774A1278AC
:10997800D10649D4002F47D1002B45D1720243D4D8
:10998800734B1B78002B02F0FC81724B9B78002DE7
:1099980042F08E823BB1704A704B12681B689B1A6A
:1099A800002BC2F27A821020644C0FF0E5F80123F4
:1099B80084F88D3028E0594B06931E68594B584A55
:1099C800049306F48056584B05920893002E3FF4F2
:1099D8007FAF00215848F7F76BFC00287FF478AF79
:1099E8000DF01EFA74E774029ED4079A127802F0FA
:1099F8000102524C002184F88C10002DA5D0524948
:109A080001200870002AAFD1554B1A78002A40F07F
:109A1800BD800599049C488BB4F90070898BB4F912
:109A28000240B842B4BF8026002646F04003B9423F
:109A3800D8BF33469B0843F08006A042B8BF3346E0
:109A4800049F43F04006A142C8BF33469B08B7F9BC
:109A58000440B7F9066043F08007A042B8BF3B4610
:109A680043F04007A142C8BF3B469B0843F080072C
:109A7800324C8642C8BF3B4643F0400794F88EE01C
:109A88008E42B8BF3B469E4501F03584A4F890202D
:109A980084F892202E4984F88E300E78002E01F03A
:109AA8005D835F2B01F0D0836F2B01F0E883079B68
:109AB8001B78DE076AD494F89210002966D1B4F9AD
:109AC8009030322B62DD94F88E200120572A84F8DA
:109AD80092004DD0069B1B685D0741F174825A2A9B
:109AE80041F0718294F89430002B42F0418194F84F
:109AF800963083F0010384F89630002B42F0E4811D
:109B08000C200FF039F8174B174D099341E000BFAF
:109B18006C33002044320020683300203C58002079
:109B280098480020D2690020184F0020D23C00201D
:109B3800404B4C00C04C002018390020E41800208D
:109B48007C450020C0380020401800202039002023
:109B58008B140020E83A00204C470020A828002059
:109B6800FF54002080450020784500202434002040
:109B7800884B894A19684FF47A73B3FBF1F3C3EB46
:109B8800431103EB8103DB00A2F8A830834B844D1B
:109B98000993069B1B685F0700F1A8860DF1500921
:109BA800804E0A950022C9F804203446149240F6E3
:109BB800330B4FF0190840F28337049D02E0043458
:109BC800544522D0A178E378994218FB0170F6D267
:109BD80094F801E00EF1040E18FB037135F91E30FC
:109BE8005B45A8BF5B46B3F5617FB8BF4FF46173AF
:109BF8009842E4DA9942E2DB21782729DFD84846FF
:109C08000434F7F745FB5445DCD1674A0A9D1378BD
:109C1800664A99E8030082E80300002B40F03F867B
:109C2800634B1A78002A00F0B98501215F48F7F7DD
:109C38003FFB002840F0DE82089BDB78002B40F0D9
:109C4800D9825C4B0A932B881FB227F001071FFAB1
:109C580087F84345A5F8008000F0E287564F4FF09B
:109C680002090E204FF0140A4FF0FF0B87F80090FE
:109C780087F801A087F802B00EF07EFF49464B48EE
:109C8800B5F80080F7F714FB002841F0AC8228F003
:109C980002039BB243452B800BD0474B0220142173
:109CA800FF2218700E2059709A700EF065FFB5F8F3
:109CB8000080424B424A197850680B9318F0030F02
:109CC80008BF81F00201C1F340010C9207F0B0FC1B
:109CD80024213648F7F7ECFA30B9079A13785F076A
:109CE80044BF23F0040313700A9B1B6813F00A0F88
:109CF80011D006212D48F7F7DBFA002801F0C680BD
:109D08002B88580641F1378207212848F7F7D0FAFF
:109D1800002840F0E1870C212448F7F7C9FA2A887F
:109D2800002800F0478342F480739A422B8009D0C0
:109D3800214B022214211A700E20FF2259709A70AA
:109D48000EF01AFF1F4B1B78082B00F03F830E2BD9
:109D580000F03C83069BD3F8008018F4806F6BD02A
:109D6800194B1B79002B00F0308214210F48F7F7AC
:109D78009FFA002840F02E821AF000F901200EF018
:109D880003FE002855D0DFF844A000274FF0CC0B85
:109D9800A14620E02C580020B45500208045002022
:109DA80078450020D4330020605A0020183900205C
:109DB8005554002024450020643800201447002012
:109DC800184700200C3B0020484D0020DC6600208E
:109DD800DFB2022F2CD80BFB07F87B1C5AF808407F
:109DE800002CF5D1032290F9023002940192C27836
:109DF800E24951F8222000921846224623460121C2
:109E08000EF002FA034607EB470000EB00100A9336
:109E180053B121460AEB8000CC2227F016FB0A9B9F
:109E28004AF808300137FFB21DF04AFA0028D0D1AD
:109E38004C46069BD3F80080079B93F800A0D04BB4
:109E48001AF0010A00F0388201221A70099B04995D
:109E58001B68B1F906105A89CA4801279142077050
:109E680080F21082C84B4FF07E521A60059BC74F94
:109E7800B3F81890049B97F90420B3F900303878A8
:109E880097F801C0002AA3EB090714BF01224FF07D
:109E9800FF32002FB8BF7F42B7F5FA7FA8BF4FF453
:109EA800FA77B84280F2EB813F1A07EE907AF8EE23
:109EB800E77AB74F4B45C7ED007A03DAF1EE677AD8
:109EC800C7ED007A049BB3F902E0AEEB0903002B5F
:109ED800B8BF5B42B3F5FA7FA8BF4FF4FA73984254
:109EE80080F2CA811B1A07EE903AF8EEE77AF1453C
:109EF800C7ED017A03DDF1EE677AC7ED017A049BBD
:109F0800B3F90400A0EB0903002BB8BF5B42B3F51B
:109F1800FA7FA8BF4FF4FA736345CCBFA3EB0C03D9
:109F2800002302FB03F207EE902AF8EEE77A484591
:109F3800C7ED027ABCBFF1EE677AC7ED027A18F472
:109F4800805800F07681B1F5FA6F924BA8BF4FF4B4
:109F5800FA61B1F57A7F1A78B8BF4FF47A71A1F532
:109F68007A71002A41F00F818B4ADFF844E282FBC4
:109F78000130CB17C3EB6013581C6FF0630C3EF92C
:109F880010003EF913E00CFB0313A0EB0E0003FBDB
:109F980000F382FB0312DB17C3EB62139E440FFA34
:109FA8008EFE07EE90EAB8EEE78A87ED038AB8F1ED
:109FB800000F40F09C832B885A0640F1FB807749BC
:109FC800774A91ED018AD2ED019A92ED026A91EDFC
:109FD800034A92ED030A91ED029A92ED007AD1EDCF
:109FE800005AD7ED011A97ED002A6E4A6E4938EEED
:109FF800445A79EEC63A77EE007A65EE233A75EE62
:10A00800C96A75EE890A37EE401A66EEA76AB0EE9D
:10A01800633AA0EE813A13F00303B0EE665A78EE85
:10A02800044A79EE867AA0EE815AF0EE638AA4EEAD
:10A03800A73AD4EEA78AA4EEE75A33EE263AF0EE12
:10A04800687AF0EE674AF6EE008A35EE88AAE0EE06
:10A05800C14A28EEC33A35EE635A77EE293A77EECD
:10A06800E67AAAEE233A25EE285A76EE403A34EEFE
:10A0780049AAE0EE817A74EEA64AAAEE235A34EE93
:10A08800094A37EE697A64EEA84A63EE036AE4EE99
:10A09800074A75EEC85A36EE006A67EEA87AB0EE3F
:10A0A800667A95EE057AE5EE056AE5EE867AB1EE12
:10A0B800648AF0EE665AF0EE476AB1EE674AE8EE57
:10A0C800246A63EE270A67EEA43AE4EE275AB1EE53
:10A0D800450AB0EE609AB0EE631AA4EE277A23EE32
:10A0E800244AE7EEA76AA5EE249AA0EE031AE8EE42
:10A0F800245AB0EE448A31EEA16AE0EE240AA5EEB5
:10A10800278A66EEA16A72EE028AE5EE033A61EEEC
:10A11800211A26EE096AA4EEA47AA0EE274A0CBFFB
:10A12800D7ED022ADFED212A82ED005AA2EE256A38
:10A13800E8EEA06AE2EE081A73EEA33A27EE227A56
:10A1480034EE044AF0EE005AE3EEA26AA4EE226A64
:10A15800A1EEA57AC7ED016AC1ED366A81ED356ACF
:10A1680087ED006A81ED377A82ED013AC2ED027A15
:10A17800C2ED034AF3B987ED027A1BE09C39030864
:10A18800C14C002078180020F4170020C03A0020A5
:10A19800584D0020C41D00201F85EB51CC00002025
:10A1A80084000020BC000020E4180020000000000B
:10A1B800C86A0020BAF1000F40F01B8124F0F8FCB7
:10A1C80017B0BDEC068BBDE8F08F079B1B78D9074D
:10A1D8007FF5D2AD4FF40F7024F09EF800283FF4BD
:10A1E80028AE0DF0F9FF4FF40F7024F03FF8002867
:10A1F800F7D11EE69A4B0A931B689B077FF523ADA0
:10A20800B5F8008018F0010F7FF441AD48F0010364
:10A2180098452B803FF43BAD924B022214211A70D3
:10A228000E20FF2259709A700EF0A6FCB5F8008037
:10A238002DE5059B5A8B9142C0F29884B1F5FA6FCF
:10A24800D4BFC2EB0101C2F5FA614FF47A7303FB84
:10A2580001F185480378C2F5FA62B1FBF2F1002BEF
:10A268003FF482AE4378814A01FB03F182FB01236C
:10A27800C917C1EB631177E6DFED7D7A37E6DFEDCD
:10A288007C7A16E6B1F5FA6F80F24484187A8B1A54
:10A2980003FB00F3C2F5FA6293FBF2F3C3F1640324
:10A2A80007EE903AF8EEE77A9FED727A724B67EE16
:10A2B800877AC3ED007AD9E51B780693002B7FF4E3
:10A2C800C5AD6E4A1268002A3FF4C0AD6C4A0792C9
:10A2D80012F8030CDFF8E0B11146D71E0CF00AF8AB
:10A2E8009BF80090079A002800F01486069BB9F1A5
:10A2F800000F53D107F1080178790BF0FBFF002814
:10A3080041F019855F49B87A0BF0F4FF002800F096
:10A318001486B9F1020F41F00A855B49F87B0BF00E
:10A32800E9FF002841F0FF845849387D0BF0E2FF2F
:10A33800002800F01486B9F1040F41F0F084544964
:10A34800787E0BF0D7FF002841F0E5845149B87FAB
:10A358000BF0D0FF002800F01486B9F1060F41F089
:10A36800D6844D4997F823000BF0C4FF002841F02C
:10A37800CA844A4997F828000BF0BCFF002800F06F
:10A388001486B9F1080F41F0BA84454997F82D00B1
:10A398000BF0B0FF00283FF459AD09231A4602EB31
:10A3A800820217443F4A7878B9788BF800301070E9
:10A3B80051704BE522F480739BB29A422B807FF454
:10A3C800B7AC394B1B78082B7FF4C1AC2A8822F034
:10A3D80040039BB29A422B803FF4BCAC214B022233
:10A3E80014211A700E20FF2259709A700EF0C4FBC7
:10A3F800B0E40B9B19780C9B01F00101186807F079
:10A4080017F917B0BDEC068BBDE8F08F13B9089AA1
:10A4180001239370254B089A1D7892F821400793E1
:10A428001B200BF091FF012C05F00108814600F07C
:10A43800238705F00205089A1D4E92F82030DFF8B0
:10A448007CA01C4F09959346052B00F29287DFE804
:10A4580013F0BF00B5003700FD00FF00F20000BF99
:10A468002445002064380020C41D00201F85EB51BE
:10A47800000000000AD7233CF4170020C44C002039
:10A488000E380020183800201D38002022380020FF
:10A49800273800202C38002031380020363800209A
:10A4A8003B380020C84C00200C3B0020C04C00204A
:10A4B8007C28002074450020080000208B14002010
:10A4C800012C04BF05238BF82030B8F1000F12D0FF
:10A4D800059B3088B3F918100022134661F30F0268
:10A4E80060F31F4261F30F03049861F31F43036095
:10A4F8000323426009939E4DDBF814102A689142A9
:10A5080080F01C8647F230510322CBF81C108BF8E0
:10A518002020022008F086FB0CF082FC2968DBF87A
:10A528001C200A440421CBF818208BF82010012C99
:10A5380040F095872A68DBF81810914280F0198757
:10A548009AF8000020B90BF0FFFE002840F01187B0
:10A558003A6822F002023A602A687388642101FB93
:10A5680003234FF480600022CBF810308BF82020B2
:10A578008BF8032008F026FB9BF8203064E70BF0EB
:10A58800E9FE012807D17A4D72882B68642101FB06
:10A598000233CBF81030B9F1000F02D0B379002B99
:10A5A8004BD1012C00F0E586714DDBF810102A68BC
:10A5B8009142C0F0498701238BF82030012C3AD012
:10A5C800F379012B46D00BF053FE9BF820303BE784
:10A5D800B8F1000FD3D1099D4FF48060B9F1000F95
:10A5E80000F03E8308F006FB089A00231361002D53
:10A5F8003FF484A928460EF0BFFA069B1E6816F49D
:10A6080080573FF481A91D215A48F6F751FE0028CA
:10A618007FF47AA9584B03F1500A03E004339A45B2
:10A6280000F0D2861A78262AF8D19978DA789142F9
:10A63800F4D2FFF76BB94E4D8EE70BF019FE0322EB
:10A648004FF47A738BF82020CBF81C30484D60E724
:10A65800474D6CE70BF00CFE032240F6B8338BF83D
:10A668002020CBF81C30424D53E7444F3B78002B59
:10A6780001F07D82424BDFF81881DFF818B1DFF86E
:10A6880018A1059345465E46049099460EE019F8D0
:10A6980004109847032C28DC88B93B782AF8020F65
:10A6A80001349C4205F1040580F25A81072CE1B27D
:10A6B8003046DBF80430EADD984700B2EDE738F8B9
:10A6C80024206B88801A4FF47A719B1A01FB00F0E2
:10A6D80040F6CA0290FBF3F00844904240F2EE23A1
:10A6E800A8BF10469842B8BF184600B2D5E71D214A
:10A6F8002048F6F7DDFD28B100F015BE0436B44257
:10A708003FF459AC31782629F8D1B278F3789A42D7
:10A71800F4D2089BDB78002B7FF44DAC1548F6F794
:10A72800C7FDDFED187A002801F0388238EE678A15
:10A73800154A1649FDEEC87ACDED047ABDF91030F8
:10A748001B0382FB0302DB17C3EBA212C9F57A7362
:10A758001BB203FB02F343F30F334B4407EE903A6B
:10A76800F8EEE77A0123C7ED037A0B7023E400BF04
:10A778004C47002018390020D4330020983400209A
:10A788009848002000007A44D34D62106C180020CD
:10A79800AC340020A0540020E2180020DFF8B49167
:10A7A800DFF8B4A1644F0A9209F15A084FF0010B7F
:10A7B800494619F8010C0BF09DFD00B399F8040007
:10A7C80099F8023099F803E000EB400107EB8101AA
:10A7D800013BD1F8A02003EB4303534493420ED02E
:10A7E80097F8CC20C1F8A0300BFA00F022EA00005C
:10A7F8000A9B81F89CE0C1F8A43087F8CC0009F1E5
:10A808000609C145D4D14D4B4D4A1B780A93099B83
:10A81800DFF848A112681B680B93AAF19C094FF056
:10A82800000B9046DAF8043083B31F7877B3DAF870
:10A838000820A8EB0202002A0CDB99F8CC200121A1
:10A8480001FA0BF122EA010208F5FA7189F8CC2025
:10A85800CAF808100A9ACAB19AF80020597804323E
:10A86800D2B2002940F0418305990498098B30F948
:10A87800122001F1C800824240F3B88599F8CC1043
:10A888009A7841FA0BF3D80740F142860BF1010B95
:10A89800BBF1040F0AF10C0AC4D1FFF7C6B9294B62
:10A8A80003E004339C423FF4BBA919782329F8D16B
:10A8B8009878DA789042F4D22348F6F7F9FC002821
:10A8C8003FF4AEA9214B1B6813F4003341F0FB8120
:10A8D80000221F4B1046995C142902F10C0201F06A
:10A8E800828001301828F6D1FFF79AB9124C94F8F3
:10A8F80096305BB1079B1B78DE0707D5049BB3F93D
:10A908000620059B5B8B9A4200F3F48511210E48C3
:10A91800F6F7CEFC002800F0D08294F89A302BB9D4
:10A9280094F8943013B93223A4F89830012384F8AA
:10A938009A30FFF733B900BFE4180020094F002010
:10A948004C470020D4330020183900201837002045
:10A958001832030825370020101C0308801900202E
:10A96800DDF81090C04A0692C049126842F2010A06
:10A97800A1FB091B12EA0A0A4FEA9B1B00F09A8204
:10A98800BB4DBC48BC4CBD492E7800782670087079
:10A998001EB1BA490E7886F00106B94C0F2184F829
:10A9A8002410002B00F0F283059DB64BB5F826C0A5
:10A9B800B5F824E0059D109318462D8B0078B24B0E
:10A9C800129594F825500995B04D0495A3FB0053B2
:10A9D8005B0803EB4303C31ADBB20F90CDF834C016
:10A9E80002F480520C9304F128000BF59673CDF80D
:10A9F800449097F80080DDF82490DFF8D4C20994D9
:10AA0800A24C0E91139200210A930896CDF81CE0EF
:10AA1800089B002B00F03483099B079D33F9112014
:10AA28001FFA82FEAE454FEA410303D30D9DAE45A2
:10AA380040F26B835CF82120934580F02B83E25E23
:10AA4800BAF1000F40F0408301314145E25200F174
:10AA58000600DDDB0E9A099C8D4B84F824200F2A12
:10AA680049460CBF01220022DDF8449084F82510E5
:10AA78001A7000F09283874B7E49804ADFF854B2FF
:10AA880008931C46042001230B70137008F0CAF8C1
:10AA9800DBF80030A1686268E3605B1A934284BF08
:10AAA800002384F82130069B3C781E68002C01F0B6
:10AAB8006280059A784DB2F824E0178B734916F432
:10AAC8008056284640F0A28332460EE0437803EBD6
:10AAD800830303EB830303F2EE239BB20132A2420A
:10AAE80021F8023B00F102000ED015F81230002BBD
:10AAF80000F00F83022BE9D001320B8821F8023BCA
:10AB0800A24200F10200F0D1109A137801331370B9
:10AB1800FEF7DBBE1B7AC3F1640307EE903AFFF73A
:10AB2800C1BB059A0499537DD27D013B31F913309D
:10AB38001AB1C3F53B6308331BB2A3F57A7307EE6A
:10AB4800903A9FED567A564AF8EEE77A40F2FF318E
:10AB580067EE877AFCEEE77ACDED077ABDF81C3010
:10AB68008B4228BF0B461380FEF7BDBE4146FFF758
:10AB780070BB434CD4F88830A9EB0303002BFEF6D6
:10AB8800B2AE484A484B527C059933F812308A7D58
:10AB9800DFED466A9FED466AC97D9BB207EE102A33
:10ABA80007EE903AB8EEC77AF8EEE77A27EE267AFB
:10ABB80067EE867A0B9AC4F88820C7EE876A40F257
:10ABC800FF32FCEEE67ACDED077ABDF81C309342F1
:10ABD80028BF134609B1D31A9BB23648364D0178BF
:10ABE800364C35F81160226825F81130921B134451
:10ABF80001312B4D236001F00F021B0902702B80DD
:10AC0800FEF771BE02F098FE2D4B2E4A1B68C31A40
:10AC180093427EF768AE224B00221A80FEF763BE8D
:10AC280002212948F6F744FB00283FF430A82F807A
:10AC380018F0020F7FF43DA848F0020343452B802B
:10AC48003FF437A8214B022214211A700E20FF224C
:10AC580059709A700DF090FFB5F80080FFF729B889
:10AC680007F0B0FFC0E400BF3C580020D34D62108D
:10AC78002032002008010020094F0020090100208F
:10AC8800E418002089330020ABAAAAAAD2690020C0
:10AC98001E550020184F0020E03400206F12833F1B
:10ACA800104F0020C4460020E44600200000C8429F
:10ACB80000008044D33C0020D83C0020D43C002035
:10ACC800B816002060E31600183900206438002008
:10ACD8008C3300204C470020CE4AB2F90030002BBC
:10ACE800B8BF5B42B3F5E17FBFF615A8B2F90230F1
:10ACF800002BB8BF5B42B3F5E17FBFF60CA8C64B8B
:10AD080093ED096AD3ED076A93ED057AD3ED037ADB
:10AD180076EE866A77EE877A76EEA66AB7EE007ADE
:10AD280037EE666A77EEA77AB0EEC66AF0EEE75AB3
:10AD3800B4EEE56AF1EE10FAB4BFB0EE655AB0EEC3
:10AD4800465AB5EE405AF1EE10FA40F0A4839FED52
:10AD5800B37AB4EEE56AF1EE10FA44BF9FEDB06A3B
:10AD680036EE477AB7EE006AF4EEC66AF1EE10FAEC
:10AD7800C8BFDFEDAC6AF5EEC07AC8BF36EEC77A59
:10AD8800F1EE10FA48BFB1EE477AF6EE007A27EEF8
:10AD9800677ADFEDA37A77EE276ABDEEE66A16EEEC
:10ADA800103A2033402B40F25B86DFED9F6A9F4AC2
:10ADB800DFED9D7AC2ED006AFDEEC76AC2ED017A49
:10ADC80016EE903A2033402BC2ED027A49D8DFEDD7
:10ADD800957AB4EEE77AF1EE10FA40F3B2879FED78
:10ADE800946ADFED946A01E0B0EE677AB4EEE67A31
:10ADF800F1EE10FA77EE467AF6DC9FED8F7AF4EEF4
:10AE0800C77AF1EE10FA40F1AA879FED896ADFED63
:10AE18008B6A01E0F0EE477AF4EEE67AF1EE10FA8A
:10AE280037EE867AF6D4DFED7E7AB4EEE77AF1EE85
:10AE380010FA40F38686DFED7B7A37EEC77A27EE85
:10AE4800076ADFED7F5ADFED7F6ADFED7F7AE6EE96
:10AE5800256A67EE065AE6EE267AA5EEA77AF0EEA0
:10AE6800477A7A4BC2ED037A1A6812F4003240F03E
:10AE78005986774B1046995C0A2902F10C0200F0BA
:10AE88003B8501301828F6D1FEF745BF2A8822F005
:10AE980040039BB29A422B803EF436AF6D4B0222A0
:10AEA80014211A700E20FF2259709A700DF064FE5A
:10AEB800FEF72ABF68490E786AE594F89430002BAB
:10AEC8003EF46CAE079B1B7813F001037EF466AE6C
:10AED800012284F8943084F89520FEF75FBE5F4C19
:10AEE800012184F88C10FEF78ABD012900F0228523
:10AEF80099F8CC20012303FA0BF30BF1010B134350
:10AF0800BBF1040F89F8CC300AF10C0A7FF48AAC43
:10AF1800FEF78BBE511D78790BF0ECF900283FF451
:10AF2800F1A9B9F1010F40F0068707F10D01B87AD0
:10AF38000BF0E0F9002840F0FA864949F87B0BF05D
:10AF4800D9F900283FF4F0A9B9F1030F40F0EB86D6
:10AF58004449387D0BF0CEF9002840F0E08642499C
:10AF6800787E0BF0C7F900283FF4F0A9B9F1050F76
:10AF780040F0D1863D49B87F0BF0BCF9002840F07D
:10AF8800C6863B4997F823000BF0B4F900283FF434
:10AF9800F0A9B9F1070F40F0B686364997F82800AE
:10AFA8000BF0A8F9002840F0AA86334997F82D003D
:10AFB8000BF0A0F900283EF449AFB9F1090F3EF4AF
:10AFC80045AFFFF7EAB95D2A00F0A8855B2A00F0D3
:10AFD800A4825E2A00F03B86562A00F04886972A0B
:10AFE80000F07D86A72A00F02886244D2B889B0731
:10AFF80040F0F585A2F1B703072B00F2C082DFE825
:10B0080013F0B202BE02BE02BE02A602BE029A023D
:10B018009A0200BF2845002094000020A7DFA8342A
:10B02800DB0FC93FDB0F494000000000CC000020C7
:10B03800DB0FC940E4CB1641DB0F49C0E4CB16C196
:10B0480092E741B99730083C15A82ABE1837002066
:10B058001832030864380020094F0020E418002043
:10B068001D38002022380020273800202C380020E6
:10B0780031380020363800203B3800207845002041
:10B08800079B002B3FD05CF8212093454FEA4103F2
:10B09800FFF4D5ACBA4ABA4DD25C05EB030E002AD0
:10B0A80000F09480022A47D19EF8012002EB820228
:10B0B80002EB820202F2EE2292B2032933DD12B2CF
:10B0C800BAF1000F3FF4C0AC0C9D20F81520B9F17F
:10B0D800000F03D10F9D022D7FF6B6ACB0F8029099
:10B0E8000288B0F804E04A449644A64A0FFA8EFE55
:10B0F80082FB0E52A44DA2EBEE7225F803E012B2C9
:10B108004FF00109A0E41A464B000A9D4CF8215063
:10B1180096E4D3B2022B04D9032B7FF4EDAC73462B
:10B12800DCE43B46DAE4012505FA01FE0E9D25EA3A
:10B138000E0512B20E9583E4E25ABEE7934A1278DE
:10B14800002A7FF4DFA9B8F1000F3FF4DBA9012C36
:10B1580040F00F819BF82030FFF776B931468C48D4
:10B16800F6F7A6F8002800F0A28084F893600CF0A7
:10B1780085FAFEF79CBC43F0400293422A807FF494
:10B188008DAEFEF7C1BD5B78FFF76DB8814B824A83
:10B19800109201221A70814B04931B217C48F6F708
:10B1A80087F800287FF467AC7D4BDFF818B2089366
:10B1B8001946DBF80030CA688B609B1AC82B00F26E
:10B1C800DE84069B1E6806F480569DE4CAB2022AF5
:10B1D80040F2AD83032AAFD1129A139D079E002D2A
:10B1E80008BF324669E728F0010292B242452A8038
:10B1F8003FF41EAD0E2087F8009087F801A087F86D
:10B2080002B00DF0B9FCB5F8008011E500220FE09E
:10B21800437803EB830303EB830303F2EE239BB230
:10B228000132A24221F8023B00F102003FF46CAC6B
:10B2380015F812301BB1022BEAD00B88F0E7D3B215
:10B24800032BFAD83B46EBE7B2F5FA7FFEF69EAC45
:10B2580094F89230002B7EF499AC079B1B7801215F
:10B268000B4084F8921000F0A2830BF0D9FD4D4BEF
:10B278004D4D0993FEF78DBC0025FFF7DCB8B2F5FC
:10B28800FA7FFEF683AC94F89230002B7EF47EAC05
:10B29800079A12780121D70784F8921000F14A849E
:10B2A8000CF0ECF93F4B404D0993FEF772BC079B3D
:10B2B8003E4A1B781060DB077EF5FDAB3C4B1B78E4
:10B2C800002B3EF463AC089BDB78002B7EF45EAC6D
:10B2D80094F893300133DBB2032B84F893307EF675
:10B2E80055AC344B5B7813B9002D7EF44FAC0BF0A2
:10B2F80097FDFEF7DCBB304A30491068B4F990205E
:10B30800C66981FB06018911F617701A00F5FF401E
:10B318007F3082423EF7BEAB891B0A4412B2A4F8C2
:10B328009020FEF7B7BB089BDB78002B7FF4EAA9D7
:10B33800DFED237A214938EE678AC9F5FA63FDEE15
:10B34800C87A1BB2CDED047ABDF91020120381FB37
:10B358000201D217C2EBA11203FB02F343F30F332E
:10B368004B4407EE903AB8EEE78A87ED038AFFF779
:10B37800C9B9099D002D3EF4C1AAFFF73BB900BF2A
:10B38800E034002056555555541900203018002037
:10B39800183900201E55002089330020D26900206A
:10B3A800184F00208045002078450020AC28002058
:10B3B800094F0020E83A00206C460020D34D621067
:10B3C80000007A444C470020BC4A059BD588049A63
:10B3D8001B8BB2F906105A1B914240F388802B440C
:10B3E8009942B4BF00250125FEF799BAC8398A42A7
:10B3F80042DA99F8CC109A7841FA0BF3D9073FF55D
:10B4080045AA524201200C920DF09CFC7B1E0C9A1E
:10B41800162B00F25081DFE813F0F7010B02DE0172
:10B4280030021F024402C901B4019F018A0175015B
:10B438004E01300240014402C901B4012C01180137
:10B4480004015902EE00DA000AF012FF032140F667
:10B45800B8328BF82010CBF81C20FFF75AB8AB464F
:10B468000899DBF80020CB69099D13448B61002DF6
:10B478003EF444AAFFF7BEB899F8CC30012202FA8C
:10B488000BF223EA020308F5FA7289F8CC30CAF8FD
:10B498000820FFF7FBB9B4EEE56AF1EE10FA8CBFAD
:10B4A800B0EE654AB0EE464AC4EE054A9FED842ADE
:10B4B8009FED845ADFED841ADFED842A9FED843AEC
:10B4C800DFED843A9FED844AA4EE825AE4EEE12A45
:10B4D800A4EE857AA4EEA23AB0EE475AB0EE637AAB
:10B4E800A4EE837AA4EE874A84EE057A31E4012536
:10B4F800FEF715BA00217948F5F7DAFE00287FF43F
:10B5080005AA322384F89600A4F89830FFF7FEB90C
:10B51800002A0CBF0120022075E7714B012202208E
:10B528007049714C0B60714B2270714D09930DF08D
:10B5380009FCFEF72EBB6D4A6B4B099211466D4A0A
:10B548000A6002225A7023F04FF9FEF722BB674ABD
:10B55800654B09921146684A0A6000225A7023F026
:10B5680043F9FEF716BB614A5F4B09921146634ADD
:10B578000A6001225A7023F037F9FEF70ABB792ACC
:10B5880000F07F847A2A00F073849E2A00F03D84BC
:10B598009D2A00F03284AE2A00F02784AD2A00F0FC
:10B5A8001C84EF2A00F01684FD2A00F01084FB2A80
:10B5B80000F0FD83FE2A00F06D84F72A00F0758400
:10B5C8007B2A00F0EE83494B0993FEF7E2BAD9F8DB
:10B5D800D0004B4B90F836109B7811446429A8BFD3
:10B5E800642121EAE17180F83610002B40F097843D
:10B5F80009F084FF7CE4D9F8D000414B90F837106B
:10B608009B781144FE29A8BFFE2121EAE17180F848
:10B618003710002BECD016200AF0E0FED9F8D00045
:10B62800E6E7D9F8D000364B81781144C829A8BF7D
:10B63800C82121EAE17181709B78002BD8D01420B1
:10B648000AF0CCFED9F8D000D2E7D9F8D0002C4BBC
:10B6580041781144C829A8BFC82121EAE171417085
:10B668009B78002BC4D013200AF0B8FED9F8D0007C
:10B67800BEE7D9F8D000224B01781144C829A8BFE9
:10B68800C82121EAE17101709B78002BB0D012200B
:10B698000AF0A4FED9F8D000AAE7194B0B989B78BA
:10B6A800417911446429A8BF642121EAE1714171FB
:10B6B800002B40F02384D9F8D00099E764280020B3
:10B6C80099FB243F69A2163E39094E3DE3B59E3EDB
:10B6D80088FA163E45FE7F3FA7DFA83418390020B8
:10B6E800422F00207C450020705400208045002017
:10B6F80078450020945400207C5400208854002071
:10B7080014300020D9F8D000C44B017A9B7811443A
:10B71800C829A8BFC82121EAE1710172002B3FF4B2
:10B7280067AF0B200AF05AFED9F8D00060E7D9F8C5
:10B73800D000BA4BC1799B781144C829A8BFC82149
:10B7480021EAE171C171002B3FF452AF0A200AF0DF
:10B7580045FED9F8D0004BE7D9F8D000AF4B817936
:10B768009B781144C829A8BFC82121EAE1718171D9
:10B77800002B3FF43DAF09200AF030FED9F8D00085
:10B7880036E7D9F8D000A54B417993F802E0114487
:10B79800C829A8BFC82121EAE1714171BEF1000F93
:10B7A80040F09A83112F7FF43FAF21E7D9F8D000FA
:10B7B8009A4B017993F802E01144C829A8BFC8211F
:10B7C80021EAE1710171BEF1000F40F09E83102F54
:10B7D8007FF43EAF0CE70B99904B0F790C9317440D
:10B7E800642FA8BF642727EAE7770F7122F0FCFFD0
:10B7F8000C9B9B78002B3FF45EAF032039460AF080
:10B80800EDFDD9F8D000F3E60B98844B017811448C
:10B81800FA29A8BFFA2121EAE17101709B78002B6F
:10B828003FF449AF01200AF0D9FDD9F8D000DFE68E
:10B838000B987A4B817811446429A8BF642121EAC6
:10B84800E17181709B78002B3FF435AF02200AF03C
:10B85800C5FDD9F8D000CBE60B98704BC1799B7821
:10B86800114481F30801C171002B3FF424AF052076
:10B878000AF0B4FDD9F8D000BAE60B98674B817985
:10B8880093F802E011446429A8BF642121EAE17118
:10B898008171BEF1000F40F029830D2F7FF4FEAEB9
:10B8A80009E7D9F8D0005D4BC17893F802E011445C
:10B8B800C829A8BFC82121EAE171C170BEF1000FF3
:10B8C80040F032830F2F7FF4D7AE91E60B98534B9D
:10B8D80041781144B1F5967FA8BF4FF4967121EADB
:10B8E800E17141709B78002B3FF4E5AE15200AF01A
:10B8F80075FDD9F8D0007BE64949D1F800E042004F
:10B90800BEF1000F08D0171803EB87079EF801E077
:10B918007F787745BEF4FFA91044424F424A03EBB3
:10B92800800300200B6038801060FEF7F4B9129A8B
:10B93800FFF7C3BB04999B7831F91220B2F5617FF8
:10B948004FF4966191FBF3F3C0F2088140F633019E
:10B958009142A8BF11460C2FA1F5617191FBF3F13B
:10B9680000F09A81182F7FF4C3AAC9B2C8290B46E0
:10B97800A8BFC823D9F8D020D77DD8B2B8423FF4A1
:10B98800B7AADF1B254BD07548BF0737FF109B7838
:10B998000137FFB23BB9002F3FF4AAAA38460DF091
:10B9A800D1F9FFF7A5BA18200AF018FDF3E71F49E7
:10B9B800096811F4003140F069811D4B08465D5C4F
:10B9C8000F2D01F10C0100F0938001301828F6D1F9
:10B9D8000023FA3A84F89230164BA4F89020164DBA
:10B9E8000993FEF7D6B80E49D1F800E04200BEF13F
:10B9F800000F08D0171803EB87079EF801E07F783F
:10BA08007745BEF40DA90244064F074803EB8203AD
:10BA180000220B603A800260FEF702B91430002061
:10BA2800EC170020D8180020DC1800201837002058
:10BA3800183203088045002078450020E4CB1641E1
:10BA4800DB0F49C0DB0FC940E4CB16C1DB0FC93F90
:10BA5800DB0F494092E741B99730083C15A82ABE48
:10BA6800B4EEE77AF1EE10FA40F372815FED0B5A0B
:10BA78001FED0E6A01E0F0EE676AF4EEC66AF1EEB9
:10BA880010FA76EEE57AF6DC5FED136AF4EEE67A04
:10BA9800F1EE10FA40F159815FED165A1FED166A62
:10BAA80001E0F0EE667AF4EEC67AF1EE10FA77EE7F
:10BAB800A56AF6D45FED1B7AF4EEE76AF1EE10FAA8
:10BAC80040F3C9805FED1E7A77EEE66A66EEA65A05
:10BAD8001FED205A1FED206A5FED207AA5EE856ADA
:10BAE80026EEA55AE5EE867AE5EE276AFFF75FB9F6
:10BAF800CA490F6845003FB12E1803EB86067F78C8
:10BB08007678BE42BFF464AF0544C54EC54803EB22
:10BB1800850300250B603580056059E7C24B00227C
:10BB28000120FDE4C14B1B78032B00F0E4800022C8
:10BB3800FFF79FB9BE4ABF4D1360BF4B0993FEF78D
:10BB480028B8DFEDBE7AB4EEE77AF1EE10FA44BF1A
:10BB5800DFEDBB7A37EEC77AFFF771B90C2F00F02B
:10BB6800BB80182F7FF4C4A900210B4602E7B54A11
:10BB78000592FEF7F7BE06F48056FEF7C5BFB24A37
:10BB8800069B1E68136823F004031360089A0123B8
:10BB980006F4805682F82130FEF7B6BF38EE678A81
:10BBA800AA4BAB491870FDEEC87AC9F5FA63CDED1A
:10BBB800047ABDF91020120381FB0201D217C2EBEF
:10BBC800A1121BB203FB02F343F30F334B4407EEFE
:10BBD800903AF8EEE77AC7ED037AFEF7ECB900235E
:10BBE800BB2A149300F08480B72A00F0B480BE2AE0
:10BBF80000F0A580BD2A7FF4C2AC4FF6FE71954ACD
:10BC08008D48D6890990908933440144D381918124
:10BC180010F08AFDF4F7BAFC10F06EFD00F080FD1C
:10BC280001200DF08FF8B4F890300022FA3BA4F808
:10BC3800903084F89220FDF7ACBF874A7D4D137889
:10BC480043F0040313707C4B0993FDF7A2BF834BA9
:10BC58000222032064E4DFED797AF4EEE76AF1EE7C
:10BC680010FA44BFDFED767A77EEE66A2EE710F039
:10BC78005BFDF4F78BFC10F03FFD00F051FD012057
:10BC88000DF060F894F88E20FFF7A9B96749097894
:10BC9800032968D0194690E6CFB2714B0D915B78B5
:10BCA800BB423FF425A96F4B0C93384607F00AFCBA
:10BCB8000C9B0D999B781BB1C9B20C200AF08EFB26
:10BCC8000137FFB267E6594B1B78032B7EF400AEB1
:10BCD8000CF036FFFDF7A4BF00273946DDE7624BBD
:10BCE800544D4FF4C8721A80534B0993FDF751BF56
:10BCF8001946022383E70CF023FFFEF70CB808234C
:10BD08001A46FEF74CBB07231A46FEF748BB062324
:10BD18001A46FEF744BB05231A46FEF740BB042328
:10BD28001A46FEF73CBB03231A46FEF738BB02232C
:10BD38001A46FEF734BB01231A46FEF730BB022130
:10BD48005DE7F0EE477AFFF758B8F0EE676AB1E6BC
:10BD5800F0EE667A98E619464FF6FE734FE7B0EEB6
:10BD6800677AFFF760B80CF0EBFEB4F990202FE685
:10BD7800314B84F8941084F895002E4D0993FEF702
:10BD8800B6BD002D3DF40FAE384C94F88D30002B25
:10BD98003DF43AAE0CF0D4FE002384F88D30FDF764
:10BDA80033BE4FF4FA61022007F0B2FA0BE4002127
:10BDB800022007F0ADFAB4F890301F4A0992963B7A
:10BDC8000022A4F8903084F89220FDF7E2BE00210A
:10BDD8000120EEE700210846EBE7FF2100201DF0D7
:10BDE800E3FA94F88E20FFF7DCBB012100201DF058
:10BDF800DBFA94F88E20FFF7D1BB0021FF201DF05D
:10BE0800D3FA94F88E20FFF7C6BB002101201DF05D
:10BE1800CBFA94F88E20FFF7BBBB00BFEC170020CD
:10BE2800D8180020DC180020F42E0020134F002022
:10BE3800AC2800207845002080450020DB0FC9BFD2
:10BE4800DB0F49C098480020744500206C1800207A
:10BE5800D34D6210C83A002020390020902F0020CE
:10BE68007054002014300020E26A0020E4180020FA
:10BE7800324A334B0993137A43F001031372FDF7E7
:10BE880088BE2E4A2E4B0993137A23F001031372AE
:10BE9800FDF77FBE002103208BE72A4C0AF0C0FF84
:10BEA800002384F88D30FDF7AFBD0021042080E722
:10BEB800002B3FF469AF2449244A09684FF47A708B
:10BEC80000FB031313605FE70B200CF055FE1C4BBF
:10BED8001F4D0993FDF75DBE11200D930C920AF0DA
:10BEE8007DFAD9F8D0000D9B0C9A5BE40D200D93D8
:10BEF8000C920AF073FA0D9B0C9ACEE40E200AF00D
:10BF08006DFAD9F8D000FFF773BB10200D930C928F
:10BF18000AF064FAD9F8D0000D9B0C9A57E4172060
:10BF28000AF05CFAFFF7C7BB0F200D930C920AF0DA
:10BF380055FAD9F8D0000D9B0C9AC3E4045500209B
:10BF480080450020E41800204C470020A828002045
:10BF58007845002038B50B4C23688BB15A68821A93
:10BF6800002A054604DA0CE05A68AA1A002A07DBF8
:10BF78009A68226018461A6890472368002BF3D104
:10BF880038BD38BD703300200B4B002210B402724C
:10BF980003F1B404012102E0072A09DC9979890731
:10BFA80002D51979815401329C4203F11403F3D16B
:10BFB8005DF8044B704700BFDC3A03081F23037089
:10BFC800704700BF022101222223017202704370D0
:10BFD800704700BF2C22022302704370704700BFD5
:10BFE8002DE9F0478C4B1B78DB07074644D58B4B74
:10BFF8008B4D1C788B4E012C59D01CD3022C07D1A9
:10C0080089498A4A09881288914201D901241C70F9
:10C01800EB7AE3B12B89D3B1854B1B78BBB107F021
:10C0280073FA002800F09B802B7B83422CBF0121F0
:10C03800002131700CE07C497E4A098810886A7BAF
:10C04800801A8842E2DAEB7A0024002BE2D13178B8
:10C058002A79632A06D8022C774E00F0BA80337802
:10C06800002B5DD1754AAB7A8C4238BF0C461470F0
:10C07800002B4CD1BDE8F0876B4B694D19885B8864
:10C08800E878CB1A83EAE3728142A2EBE3721DD30C
:10C098002B788B421AD3614B1C78E01E012861D99A
:10C0A8006749097802294FD0012C5E4EA5D15F4A15
:10C0B8005D491288687B0988121A914239DD5D4A08
:10C0C80012888A42A4D200241C70A1E7B1EB400F69
:10C0D800E1DC524B1C78E11E012940F29480022ACF
:10C0E800DEDC57494F4E0878DFF84481DFF844C159
:10C0F800DFF838E100210324022834701C7088F826
:10C108000010ACF80010AEF8001081D11FE0012C2F
:10C1180071D0022C0BD10720BDE8F0470CF02CBDE4
:10C128007068381A474B984258DD72709AE7BDE834
:10C13800F08702241C706BE7022AD2DD4049097897
:10C1480002294FF0040464D13949364E09783E4833
:10C15800022ACCBF00220122C28081804BE7022143
:10C16800317075E7022A9BDC95F800C091FBFCFC56
:10C178000CF1010CBCF1080FDFF8B4A0304EA87820
:10C1880095F801E096F800802A4CDFF8A090254E3B
:10C19800A8BF4FF0080C8AF800C01FFA8CFA10FBF1
:10C1A8000AF01EFB0AFE80B2DFF88CA02080A9F8F6
:10C1B80000E000244FF0640EB8F1020F34701C70D8
:10C1C800CAF804408AF801E07FF439AF0FFA8CF11D
:10C1D800BDE73078A0B9012377603370C2F16402FB
:10C1E8001A4B00FB02F083FB0023C017A0EBA350FF
:10C1F8006430707036E70820BDE8F0470CF0BCBC2E
:10C208007368F81A8EE7032C96D10D49097802292C
:10C218009AD0044EFCE600BFC04C0020BC1D002094
:10C2280014450020CC1D0020404D0020C01D0020DA
:10C23800564D0020BE1D0020C41D0020134F0020B5
:10C24800304D00207F969800344D00206BCA5F6BFC
:10C258002DE9F0470569C3681D4028D00F460646FA
:10C268004FF000484FF00009B5FA85F328FA03F2B9
:10C27800D2431B3B32611540042B16D8DFE803F08C
:10C288003129211903007B6A002B32D003F1FF3AD0
:10C298001FFA8AFAC7F824903C6A34B1236820460A
:10C2A800514698476468002CF8D1002DDCD1BDE8D0
:10C2B800F0873868716B036889B29847002DD3D12D
:10C2C800F5E77868B16B036889B29847002DCBD140
:10C2D800EDE7B868F16B036889B29847002DC3D1C0
:10C2E800E5E7F868316C036889B29847002DBBD13F
:10C2F800DDE7F36A1FFA83FACEE700BF08B501212C
:10C30800022005F0C9F9094B1B7803F00503052B3A
:10C3180008D00021012005F0BFF90021084605F0EA
:10C32800BBF9FEE709F02EFBF3E700BF74250020F8
:10C33800022828BF022010B4084C094B207000EBDB
:10C348008002C0EBC20207495DF8044B013003EBE1
:10C358004203C0B20B600CF0F5BC00BF7054002063
:10C36800F42E00207C45002008B510F0DDF9F4F724
:10C378000DF9BDE8084010F0BFB900BF2DE9F04F36
:10C38800013085B0C3B203938E4D8F4F8F4C904EC2
:10C398000A2302933220DFF8409219F0F5FB4FF49C
:10C3A800FA7A4FF0100C4FF47A70D9F80430C3F3CE
:10C3B8000803002B40F0C880EFF31183002B40F0F6
:10C3C800C3802968A26800BF2B689942F9D1D7F8C1
:10C3D80000E000FB0EF39B1AB3FBFEF300FB0131F8
:10C3E8004FF0010E0191D9F80430C3F30803002B74
:10C3F80040F08E80EFF31183002B40F089802B688A
:10C40800A16800BF2A689342F9D1D7F800B000FBB1
:10C418000BF2521AB2FBFBF200FB0323019A9B1AA0
:10C42800B3F57A7FDFD3BAF1010ABED1039B002BA3
:10C4380040F0C4804FF47A7ADFF89C9150464FF070
:10C44800100CD9F80430C3F30803002B40F099808E
:10C45800EFF31183002B40F094802968A26800BF95
:10C468002B689942F9D1D7F800E000FB0EF39B1A2C
:10C47800B3FBFEF300FB01314FF0010E0191D9F837
:10C488000430C3F308033BBBEFF3118323BB2B68D2
:10C49800A16800BF2A689342F9D1D7F800B000FB21
:10C4A8000BF2521AB2FBFBF200FB0323019A9B1A10
:10C4B800B3F57A7FE3D3BAF1010AC2D1029B013BFB
:10C4C80002937FF467AF4349434B4448444A0860AA
:10C4D800DA6005B0BDE8F08FEFF311888CF31288AD
:10C4E800A1682368DB0344BFC6F800E0A1682B6895
:10C4F80032685FFA88F888F31188D7F800801A4400
:10C5080000FB08F35B1AB3FBF8F300FB0233CDE73B
:10C51800EFF311888CF31288A1682368DB0344BF0A
:10C52800C6F800E0A1682B6832685FFA88F888F3DB
:10C538001188D7F800801A4400FB08F35B1AB3FB94
:10C54800F8F300FB023369E7EFF311828CF31288EA
:10C55800D4F808E02368D90303D501233360D4F85D
:10C5680008E02B683168D2B282F311883A6819441E
:10C5780000FB02F3A3EB0E03B3FBF2F300FB013164
:10C588002EE7EFF311828CF31288D4F808E02368C1
:10C59800D90303D501233360D4F808E02B68316848
:10C5A800D2B282F311883A68194400FB02F3A3EB74
:10C5B8000E03B3FBF2F300FB01315DE7184619F0F7
:10C5C80053F937E74C4700205047002010E000E0BF
:10C5D80048470020FC9F002000ED00E0EFBEADDEE4
:10C5E8000400FA0538B5434B5A899989914224BF0A
:10C5F80000225A81198ADA89914224BF0022DA81FD
:10C60800DA788AB3072A2FD03B493C4D91F853007A
:10C61800012400210A282C709C70D9713DD00C2867
:10C6280065D0DFED377A8ABB364C9FED370AA278A2
:10C63800002918BFF0EE407A062A04D8334901EBE6
:10C64800820191ED000A217959B3013A032A4DD8A4
:10C65800F7EE007A87EE800A23F03CFF23889842A1
:10C6680028BF1846208038BDD97921B19878042888
:10C67800B8BF04209870204890F853000A280CD0BE
:10C688000C28CED1DFED227A002ACDD0072ACBD0D4
:10C698000A282CD1DFED1F7AC6E70A20DFED1E7AC3
:10C6A800C1E79B78154A07EE103A1178B8EEC77AB9
:10C6B80027EE277A07EE901AF8EEE77A67EE877A80
:10C6C800B4EEE70AF1EE10FA10DDC0EE077AFDEEDF
:10C6D800E77A17EE903A102BA8BF1023012BB8BFAA
:10C6E8000123DBB28B4238BF0B46137038BDDFED38
:10C6F8000B7A99E7A0550020B4550020BC3A0020D9
:10C708006F1203393C5A00206F120338581C030873
:10C718000AD7A3390F506E3A5304E9386F12833A97
:10C728002DE9F047AA4FAB4E0FF0FEFFBE421ED2D6
:10C73800DFF81C83DFF81C934446258862197DB115
:10C748004A450DD2052D0BD933886188C3F30B03F5
:10C75800994200F0E280144625886219002DEFD135
:10C7680071683046143605F0F6F9BE42E4D39A4AA9
:10C778001378A3F1170102290FD9984911F833004A
:10C78800002840F0F680D8000144497829B194493E
:10C7980011F83330002B00F01481924B5A78022A9A
:10C7A80040F2E180002290495A701A788F48022A94
:10C7B800016000F2D48002EB82018D4BC2EBC10212
:10C7C80003EB4203998C5A8C8A4C9142236001D323
:10C7D80000225A84884B9A78042A00F0E98032B9FA
:10C7E8001A88B2F5F07F84BF4FF4F0721A80834D37
:10C7F800FFF7F8FE2B68824A1A40002A00F0E4800E
:10C80800D80700F1D080590400F1C8801A0700F158
:10C81800C0809B0400F1B6801AF0AEFA10B97948CE
:10C828000BF024FB802005F0CDF94FF4007005F0E3
:10C83800C9F94FF4802005F0C5F94FF4001005F050
:10C84800C1F94FF0007005F0BDF94FF0806005F0B8
:10C85800B9F94FF0006005F0B5F921F0C5FF0021E6
:10C868003022694824F0F1FD206808F0F1FC674B9C
:10C87800276803F1500102E0043399426DD01A7819
:10C88800002AF9D19C78D8788442F5D26049614B66
:10C898000D79614961480A70614E624C0460C82292
:10C8A800642111FB0521002259609A60DA601A613F
:10C8B8005A619A61DA6183F8202083F82120376071
:10C8C80015F05CF9584B9FED595A1B88584A9FED53
:10C8D800596A5079584906EE903AF8EEE66A138894
:10C8E800C5EE265A07EE103A53881279C1ED005A60
:10C8F80007EE903AB8EEC77A504BF8EEE77A18721E
:10C908005A7227EE067A67EE867ABDE8F04783ED1D
:10C91800017AC3ED007A0FF0EFBE63799B077FF4CD
:10C928001AAF716894F804A0304605F014F93388FA
:10C93800BAEB133F04D01436BE42FFF4FDAE16E73F
:10C9480073887068AA1FC3F30B039A4204F10601A7
:10C95800A8BF1A4623F07EFCEDE7012296E70022E5
:10C968001A70234B2EE7204902EB420201EB8201A9
:10C978001BE7D8000C186468002C7FF405AF172457
:10C98800147001E72E4805F01DF9402005F01AF94A
:10C9980042E72C4805F016F92B683AE72A4805F0D3
:10C9A80011F92B6832E7294805F00CF92B682AE7BA
:10C9B8009A8AB2F57A7FBFF41AAF4FF47A729A82E4
:10C9C80015E718231370E8E643F008032B6017E710
:10C9D80020750308C07003080C3B0020443F03087F
:10C9E800C4370308705400207C5400208045002080
:10C9F800F42E00207C4500203C5A002064300020A2
:10CA080009600002C448002080190020D4330020A7
:10CA18007C280020184F00208B140020C419002007
:10CA2800B4190020CE3A002070180020C0C9FB4875
:10CA3800A416002017B7D1387418002080260020CB
:10CA4800094000020160000209200002086000029B
:10CA580002F003080000040808B50FF065FEF3F7BC
:10CA680095FD0FF049FEFFF75BFE0120BDE8084089
:10CA78000CF068B92DE9F047B54C82B063682046E0
:10CA88009847002800F0BF80B24B1B780122042B86
:10CA980084F83C2000F0BA80B4F91610B4F91820D4
:10CAA800B4F91A3021636263A363AB4B1B88002B74
:10CAB80069D0AA4DD4ED0C7AD5ED004A95ED050A5A
:10CAC80095ED015A95ED067AD5ED035A95ED026A72
:10CAD800F8EEE76AD5ED047AA4EEA60AA5EE267A62
:10CAE80067EEC07AA5EEC07AE6EE267A85ED057A7D
:10CAF800C5ED067A23F0EEFCD4ED0D6AD5ED094AB2
:10CB080095ED0E0A95ED0A5A95ED0F7AD5ED0D7A49
:10CB1800D5ED0C5A95ED0B6A2063F8EEE66AA4EEA3
:10CB2800A60AA5EE267A67EEC07AA5EEC07AE6EEEA
:10CB3800267A85ED0E7AC5ED0F7A23F0CBFCD4ED7D
:10CB48000E6AD5ED124A95ED170A95ED135A95ED33
:10CB5800187AD5ED167AD5ED155A95ED146A6063F5
:10CB6800F8EEE66AA6EEA40AA6EE857A67EEC07A23
:10CB7800A0EE657AE6EE867A85ED177AC5ED187A25
:10CB880023F0A8FCA063764FA17F764814F078FFC5
:10CB98003B88002B7CD1744E3568744B1B685B074F
:10CBA80042D4B5F90070216B636BA06B704A714E6B
:10CBB80092ED026AD2ED006AD2ED015AC91B2163D7
:10CBC800B5F90270DB1B6363B5F904703568C01BE7
:10CBD80007EE900AB8EEE75A07EE901AB8EEE77A31
:10CBE80007EE903AF8EEE77A36EE056A36EE877A7F
:10CBF80077EEA57A0135A06382ED026A82ED007AAC
:10CC0800C2ED017A356002B0BDE8F0875A4BB4F93D
:10CC18001600B4F91810B4F91A2018802063598046
:10CC280061639A80A26340E7544F3B88322B7ED0E1
:10CC3800002B5BD152480378002BB2D0DFF848E1D3
:10CC4800F169326A8EFB01730027C9170770C1EBBF
:10CC580023118EFB0203D217C2EB2312736A2980B9
:10CC68006A80A08A47498EFB03E2DB17C3EB2213D5
:10CC78001B1AAB80CF600FF057FDF3F787FC0FF05E
:10CC88003BFDFFF74DFD01200CF05CF8356888E7A7
:10CC9800354E226B3568B3F5C87F4FF00003236328
:10CCA8002B80398818BF7068B7F8008008BF00204B
:10CCB800B1F5C87F18BFB368616B02440B4400200C
:10CCC800B8F5C87F60637260B36068803AD0D4F802
:10CCD80038E0F168A0637144B8F1010FA880F160F1
:10CCE80054D008F1FF38A7F8008056E7F169226BA5
:10CCF800002323632B80B7F800E00A44BEF1320F0B
:10CD0800616B63636B80F261A26B6BD0706A019098
:10CD1800306AA3630144019831620244BEF1010FF5
:10CD2800AB80726263D00EF1FF333B8082E7154B14
:10CD38002988D8686A88AB883182B0617282B382E8
:10CD48000021D4E7A36BF360A063A880C9E700BF04
:10CD580030450020304D00207C40002080400020DD
:10CD6800E26A002060450020C41900203C580020D9
:10CD78007426002070260020344D00207C190020E5
:10CD880079190020C83A00201F85EB51DFF80CC143
:10CD9800DFF8F8E0C8328CFB02A9C833D217C2EB1F
:10CDA800E9128CFB03A9DB17C3EBE913C8316B80CD
:10CDB8002A808CFB013CA28ACB17C3EBEC139B1A8D
:10CDC800AB80CEF80C000FF0AFFCF3F7DFFB0FF0F1
:10CDD80093FCFFF7A5FC40460BF0B4FFB7F80080C2
:10CDE80035687EE7A36331627262AB809BE7234AB2
:10CDF800234812682349037012F4003281F800E0D6
:10CE080032D113462049C85C0B2803F10C030ED01D
:10CE18000132182AF7D1338A2B80728A1B4B6A8019
:10CE2800B18AB269A980B7F800E0DA607BE71848F0
:10CE3800D0F800C05300BCF1000F09D003EB020E7C
:10CE480001EB8E0E9CF801C09EF801E0E645E2D2A7
:10CE58001344DFF84CE00F4A01EB83010023016023
:10CE6800AEF800301360D6E70B4A1278032A01D0D7
:10CE78001A46C7E70BF064FE3568CCE71837002080
:10CE88007E1900207819002018320308C83A0020BB
:10CE9800EC170020DC180020134F00201F85EB51F1
:10CEA800D818002038B50C4C0C4DAC4206D261683D
:10CEB8002046143404F04FFEAC42F8D3084A094B1C
:10CEC800094C1460002209491A705A700848086011
:10CED800BDE838401DF0A2BBC070030820750308E8
:10CEE8007C45002070540020F42E0020804500204E
:10CEF8007C54002008B5FFF7D5FF0FF015FCF3F7B9
:10CF080045FBBDE808400FF0F7BB00BFF0B50C29A2
:10CF18002BD8DFE801F06F2A2A2A4C2A2A2A2B2A42
:10CF28002A2A0700046AB2F80CE097881668674D49
:10CF380024F480540462036A4468C16923F40053EA
:10CF480043EA0E3321F4E641A84243EA073341EAB3
:10CF5800062100F0B58005F50065A84200F0B08014
:10CF680092684460C16102640362F0BD046A9689F4
:10CF78009588D2F800E0554F24F480740462036A5F
:10CF88004468C16923F4007343EA062321F073015E
:10CF9800B84243EA052341EA0E017ED04C4DA8422F
:10CFA8007BD092684460C161C2630362F0BD046AC9
:10CFB80096899588D2F800E0444F24F01004046262
:10CFC800036A4468816923F0200321F0807143EAF1
:10CFD800061321F4E641B84243EA051341EA0E215B
:10CFE80048D03B4DA84245D0926844608161826335
:10CFF8000362F0BD046A9389B2F804E01768334EFF
:10D0080024F001040462056A4468816943EA0E0356
:10D0180021F4803125F002059BB221F07301B04262
:10D0280043EA050341EA070114D0294DA84211D06B
:10D0380005F54065A8420DD005F58065A84209D0E0
:10D0480005F58065A84205D0926844608161426315
:10D058000362F0BDD689158A578A23F00803334343
:10D068003D43D68824F4407423F00403ADB233431F
:10D078002C43E9E7D589178AD68823F0800343EA49
:10D08800051324F44064558A23F0400344EA8704D6
:10D0980043EA061344EA8504A6E7D589178AD688A1
:10D0A80023F4006343EA052324F44054558A23F407
:10D0B800806344EA071443EA062344EA051470E748
:10D0C800158A24F4804444EA851449E7002C014079
:10D0D800003401402DE9F04FF022002183B0784858
:10D0E800784CDFF80492784D784E794FDFF8FC8160
:10D0F80024F0ABF977487849DFF8F4E1DFF8F4C1B8
:10D1080000221359834200F0C180B3F1804F00F030
:10D11800C980AB4200F0C880B34200F0C780BB4270
:10D1280000F0C680734500F0C580634500F0C480F8
:10D13800434500F0C380DFF8C0A153457ED00AF50F
:10D14800806A534508BF092379D01432C82AD8D138
:10D158005C4C624D624E604F04F1C80802E0143422
:10D16800A04568D0A379002BF9D023794FEA131989
:10D1780009F1FF39B9F1050F03F00F03EFD835F8BE
:10D18800190040FA03F2D207E9D54FF0010A0AFA6A
:10D1980003F3013B184022F0EFFD16F8093051491E
:10D1A800184411EBC002DAD051F83000DFF84CE136
:10D1B800217A00F138439B0A1EF8033003F01F0E52
:10D1C8005B09022B0AFA0EFA62D0032B65D0012BF9
:10D1D80003D17B694AEA03037B6193880093B3FA1E
:10D1E80083F3C3F11F039BB2DA0800EB820203F05A
:10D1F8000703D2F820E09B004FF00F0C0CFA03FC59
:10D208002EEA0C0EC2F820E0D2F820E001FA03F36F
:10D2180043EA0E03136269460023022214348DF890
:10D2280004208DF805308DF806308DF807301BF096
:10D2380015FEA04596D103B0BDE8F08F082309EB91
:10D24800C3034FF0010B93F820A00AF01F034FEA25
:10D258005A1ABAF1020F0BFA03F30BD0BAF1030F03
:10D268000ED0DA457FF471AFD1F814A043EA0A036F
:10D278004B616AE7D1F818A043EA0A038B6164E7B7
:10D28800D1F81CA043EA0A03CB615EE70023D6E786
:10D29800BB694AEA0303BB619FE7FB694AEA0303E8
:10D2A800FB619AE70123CAE70223C8E70323C6E71D
:10D2B8000423C4E70523C2E70623C0E70723BEE724
:10D2C800A8470020DC3A030800040040000800409A
:10D2D80000100040002C014000100240A43B03084D
:10D2E800B03B0308CC490020581C0308004001400B
:10D2F800001400400034014000440140D43A0308BF
:10D3080001490248FEF7A4BF7048002000480140C8
:10D3180001490248FEF79CBF204800200040014018
:10D3280001490248FEF794BFF84700200004004076
:10D3380002494FF08040FEF78BBF00BFD047002066
:10D3480010B5064C06482146FEF782FF04F1A001FD
:10D358000448BDE81040FEF77BBF00BFA847002087
:10D36800002C01400044014001490248FEF770BF0B
:10D37800A8470020002C01402DE9F04104684E4DDB
:10D38800A30AAB427AD00AD94C4DAB425FD00135E3
:10D39800AB4277D0023DAB425DD0BDE8F081B3F53A
:10D3A800801F67D04A3DAB4259D14FF0700E02261C
:10D3B80047794FEA970C002968D0B0006346851971
:10D3C8000227D4F80C809F400CEB4503BFB23C4DBC
:10D3D80003F1040C47EA080745F8231045F82C2008
:10D3E800E760EFF31181502282F31288821905EB6E
:10D3F800C2021369002B34D013620433821905EB7F
:10D40800C202576917B11F6053690433821905EBCB
:10D41800C202976917B11F6093690433821905EB3B
:10D42800C202D76917B11F60D36904330027CAB293
:10D438001F6082F31188304405EBC000036A9BB972
:10D44800E3684FF6FE721340E360BDE8F0814FF0E9
:10D45800C00E0426ACE74FF0980E0326A8E7BDE8F7
:10D46800F08105EB0E03C9E7E36843F00103E360CD
:10D47800BDE8F0814FF0480E012699E74FF0200EE5
:10D48800002695E74FF0E80E052691E7BF0802232E
:10D4980006FA03F0BB40DB43E768094D9BB23B400B
:10D4A80087190CEB470CE3600CF1040345F82C10CA
:10D4B80045F8232095E700BF4B00100051001000ED
:10D4C800A847002030B503685C4D18885C4CB4FB55
:10D4D800F2F20139013AAB4294B283B089B282B216
:10D4E80066D05848834263D0B3F1804F60D0A0F52E
:10D4F800983083425CD000F58060834258D052480F
:10D5080083425BD000F5806083427DD022F4407274
:10D5180000F58C3092B283421A80D9621C850ED0F5
:10D52800484A93420BD002F54062934207D002F575
:10D538008062934203D002F58062934201D10022B7
:10D548001A8601225A611A883C4992B242F00102B5
:10D558008B421A8062D0B3F1804F61D03B4A93422C
:10D5680060D002F5806293425ED002F50062934279
:10D578005CD002F5806293425AD002F59032934211
:10D5880058D002F54062934256D002F58062934229
:10D598001ED002F58062934208BF092219D002A862
:10D5A8004FF0012340F8043D1BF022FC03B030BDCE
:10D5B800254822F07002834292B2A3D101201A803A
:10D5C800D9621C8558611A8892B202431A80C5E74D
:10D5D80008221F4B03EBC20301A893F821408DF8E2
:10D5E8000440012300228DF805308DF807308DF8AE
:10D5F80006201BF0FDFB1B2CD8D1164B019301A86C
:10D608001BF0F6FB03B030BD01201A80D9621C85DF
:10D6180058611A8892B202431A809CE70022D8E720
:10D628000122D6E70222D4E70322D2E70422D0E778
:10D638000522CEE70622CCE70722CAE7002C0140E4
:10D6480000A24A04003401400010004000040040D9
:10D65800581C030819010001204B98422DD0B0F145
:10D66800804F2CD0A3F5943398422AD003F58063D9
:10D67800984228D003F50063984226D003F58063CA
:10D68800984224D003F59033984222D003F54063A2
:10D69800984220D003F58063984207D003F5806351
:10D6A800984208BF092202D00020704708220C4B7C
:10D6B80003EBC20393F8200070470022F7E701222A
:10D6C800F5E70222F3E70322F1E70422EFE7052258
:10D6D800EDE70622EBE70722E9E700BF002C01404F
:10D6E800581C03082DE9F04F013085B0C3B20393ED
:10D6F8000B4602918B4C8C4E002B00F09A80322006
:10D708008A4D8B4FDFF82C9218F03EFA4FF4FA7AD4
:10D718004FF0100C4FF47A70D9F80430C3F30803B3
:10D72800002B40F0DE80EFF31183002B40F0D9800E
:10D738002968A26800BF2B689942F9D1D7F800E0A0
:10D7480000FB0EF39B1AB3FBFEF300FB01314FF015
:10D75800010E0191D9F80430C3F30803002B40F0FF
:10D768008780EFF31183002B40F082802B68A1683B
:10D7780000BF2A689342F9D1D7F800B000FB0BF23A
:10D78800521AB2FBFBF200FB0323019A9B1AB3F572
:10D798007A7FDFD3BAF1010ABED1039B002B40F098
:10D7A800BD804FF47A7ADFF88C9150464FF0100C18
:10D7B800D9F80430C3F30803002B75D1EFF31183B4
:10D7C800002B71D12968A26800BF2B689942F9D152
:10D7D800D7F800E000FB0EF39B1AB3FBFEF300FB47
:10D7E80001314FF0010E0191D9F80430C3F3080359
:10D7F80013BBEFF31183FBB92B68A16800BF2A683C
:10D808009342F9D1D7F800B000FB0BF2521AB2FBE1
:10D81800FBF200FB0323019A9B1AB3F57A7FE3D34B
:10D82800BAF1010AC4D1029B013B0293002B7FF499
:10D8380066AF05B0BDE8F08FEFF311888CF312885E
:10D84800A1682368DB0344BFC6F800E0A1682B6821
:10D8580032685FFA88F888F31188D7F800801A448C
:10D8680000FB08F35B1AB3FBF8F300FB0233D2E7C3
:10D87800EFF311888CF31288A1682368DB0344BF97
:10D88800C6F800E0A1682B6832685FFA88F888F368
:10D898001188D7F800801A4400FB08F35B1AB3FB21
:10D8A800F8F300FB023370E7EFF311828CF3128870
:10D8B800D4F808E02368D90303D501233360D4F8EA
:10D8C80008E02B683168D2B282F311883A681944AB
:10D8D80000FB02F3A3EB0E03B3FBF2F300FB0131F1
:10D8E8007FE7EFF311828CF31288D4F808E02368FD
:10D8F800D90303D501233360D4F808E02B683168D5
:10D90800D2B282F311883A68194400FB02F3A3EB00
:10D918000E03B3FBF2F300FB013118E7184617F0CA
:10D92800A3FF3EE710E000E0484700204C470020F6
:10D938005047002000ED00E0204B5B68C3F308036C
:10D9480030B4BBB9EFF31183A3B91D4B1D4C186854
:10D95800A16800BF1A689042F9D11B4B1C684FF4AC
:10D968007A7202FB04F3591AB1FBF4F130BC02FBE2
:10D9780000107047EFF31182102383F312881149C6
:10D988008C680B6813F4803F104B02D0012018609C
:10D998008C680B49D2B20D68186882F311880A4B5B
:10D9A80019684FF47A72284402FB01F31B1B30BC40
:10D9B800B3FBF1F302FB0030704700BF00ED00E05D
:10D9C8004C47002010E000E0504700204847002066
:10D9D8002DE9F84F8046FFF7AFFF254E2549DFF8C0
:10D9E800A0E0254A254D844610274FF47A7401207B
:10D9F800DEF80430C3F30803D3B9EFF31183BBB9DE
:10DA08000B68D2F808A000BFD1F800904B45F7D1B9
:10DA1800D6F800B004FB0BF9A9EB0A09B9FBFBF92E
:10DA280004FB0393A3EB0C034345E1D3BDE8F88F54
:10DA3800EFF3118A87F31288D2F808B01368DB0372
:10DA480044BF2860D2F808B00B68D5F800905FFA98
:10DA58008AFA8AF31188D6F800A0994404FB0AF3DD
:10DA6800A3EB0B03B3FBFAF304FB0933DAE700BFBC
:10DA7800504700204C47002010E000E048470020B5
:10DA880000ED00E02DE9F04FDFF830C1474A484982
:10DA9800484E494D8046102718F1FF38C0F0848061
:10DAA800DCF80430C3F30803002B5CD1EFF31183D7
:10DAB800002B58D10B68946800BF08688342F9D1DD
:10DAC800D6F800904FF47A7000FB09FEAEEB040E16
:10DAD800BEFBF9FE00FB03EEDCF80430C3F30803D9
:10DAE8004FF47A740120FBB9EFF31183E3B90B68A3
:10DAF800D2F808A000BFD1F800904B45F7D1D6F86E
:10DB080000B004FB0BF9A9EB0A09B9FBFBF904FB0C
:10DB18000393A3EB0E03B3F57A7FBDD2DCF8043090
:10DB2800C3F30803002BDFD0EFF3118A87F31288C1
:10DB3800D2F808B01368DB0344BF2860D2F808B0F5
:10DB48000B68D5F800905FFA8AFA8AF31188D6F83C
:10DB580000A0994404FB0AF3A3EB0B03B3FBFAF30D
:10DB680004FB0933D5E7EFF3118487F31288D2F861
:10DB780008901368D80303D501232B60D2F80890C6
:10DB88000B682868E4B284F31188D6F800A04FF433
:10DB98007A7400EB030E04FB0AF3A3EB0903B3FB4F
:10DBA800FAF304FB0E3E97E7BDE8F08F10E000E0C3
:10DBB8004C470020504700204847002000ED00E077
:10DBC80030B4EFF31183102282F312880649074C10
:10DBD8000A680748013200250A602560DBB202683E
:10DBE80083F3118830BC70474C4700204847002019
:10DBF80010E000E02DE9F04FC04B1E788BB0002EEE
:10DC080040F0BC80BE4BBF4C1D78DFF818A3DFF88E
:10DC18001893DFF8188305F00105A4F10A0B54F8EE
:10DC28000A3CBBB1CC2707FB06B7184602F006FD35
:10DC380080B154F80A0C02F0F9FC14F8023C8BB9D4
:10DC4800242831D0F5B154F80A3C184602F0F6FC05
:10DC58000028EED10136032E04F1CC04DFD10BB03D
:10DC6800BDE8F08F012B23D0022B2BD0032B37D00C
:10DC7800042B67D0052B40D0062B4FD054F80A2C24
:10DC88001346D2E754F80A3C23281A4600F0898143
:10DC98009D4991F832108142C7D19C4BCAF8009037
:10DCA800C3F80C801346C0E7012304F8023CCAE716
:10DCB8004D2854F80A2C0CBF0223002304F8023C18
:10DCC8001346B2E700233C2804F8023C45D03E281E
:10DCD800D4D10122032304F8012C04F8023CB2E752
:10DCE800C02814D80022042304F8050C04F8040CF6
:10DCF80004F8062C04F8023CA5E714F8063C14F8CE
:10DD0800052C9A422FD814F8043C834203D00023F0
:10DD180004F8023C97E7062304F8023C14F801ECE7
:10DD2800BEF1000F00F08281BEF1010F00F0C68144
:10DD380001360023032E04F8023C04F1CC047FF4DE
:10DD48006EAF8CE714F8043C04F8030C5840052324
:10DD580004F8040C04F8023C75E7032204F8013CBB
:10DD680004F8022C6FE714F8042CF9184240013328
:10DD780004F8042C04F8063C887264E7644B1868BD
:10DD880000283FF46CAF03F01DFEDFF8A4A1614D3D
:10DD9800DFF8A091DAF8000002F050FC00283FF408
:10DDA8005EAFDAF8000002F041FC09281BD03F28DA
:10DDB80019D02B68002B67D1042800F0A9810C2802
:10DDC80000F0E8807F28E5D0A0F12002D2B25E2AD8
:10DDD800E0D80BB92028DDD05A1C09F803002A60C6
:10DDE80014F028F9D6E72C68002C5BD14A4FA346DB
:10DDF80007F59878BBF1000F08BFBB4608374745C1
:10DE0800F8D1BBF1000F00F07881083FDBF8000083
:10DE18003A68065D135D9E42204402EB040140F01F
:10DE28006A81661E4E4422460BB9FD2A5DD906F862
:10DE3800013F01322A6010F8013F11F801EF9E45B9
:10DE4800F2D00AB15F4512D0344814F0FBF85F45B0
:10DE580008D35BF8080B14F0F5F8092014F0EAF879
:10DE6800BB45F6D92E4814F0EDF82A6800249442F0
:10DE780090D2661E4E4416F8010F14F0DBF82B689A
:10DE880001349C42F7D385E70C2800F083800A28E8
:10DE980052D00D2850D07F2800F0FD80FF2B3FF690
:10DEA80079AF91E71C4E002706F59878BB4602E04B
:10DEB800083646450DD0224631684846F2F764FEDA
:10DEC8000028F5D1B346002FF2D13746083646452B
:10DED800F1D13B465F469B46002B97D1002F3FF47C
:10DEE80059AF0E4814F0AEF8B3E7511C202009F8DA
:10DEF8000200296009F801300A46A3E755540020BA
:10DF0800C04C0020E6660020C448002000ED00E078
:10DF1800CC2D0020D42E0020DC240308A0430308C5
:10DF2800A8430308FC9F0020EFBEADDE0400FA05FD
:10DF380060380020D22D002014F005F923217C48F8
:10DF480023F09AFA002800F0E180A0EB090028608D
:10DF580088B1431E19F80310202940F0E78009EB27
:10DF6800030204E012F8011D202948D10346581E77
:10DF7800002BF7D12B604FF480720021484623F024
:10DF880064FA6C4B1B78002B3FF469AE6A4814F0B6
:10DF980059F8FFE6694814F055F8674814F052F844
:10DFA800F8E667496748C978674ADFF8CCE19362C1
:10DFB800003118BF012101706449D1624021136307
:10DFC80082F8341082F83550614962480B602C326F
:10DFD800CEF80020574A0123137014F045FB564829
:10DFE80014F030F84FF4006004F01CFE5A4B93F81C
:10DFF8003230232B00F0928014F8023C3CE62B6070
:10E00800564C002204F5987809F8032002E00834F9
:10E01800444577D0216848460BF082FE0028F6D0A8
:10E0280044456FD2636898470023A3E74C4BADF88B
:10E0380022E00FCB0DF1280C02AF87E80F004CF857
:10E0480024ED14F8051C14F8033C069404EB010EA7
:10E05800624639464FF0010C06A8CDF81CE0ADF831
:10E0680020308DF824C0F4F789FFE8B9019F002318
:10E0780004F8023C002F3FF4EDAD54F80A0C09F007
:10E08800E1FF013654F80A0CB847032E04F1CC041A
:10E098007FF4C5ADE3E5013B002232482B6009F867
:10E0A800032013F0CFFF75E6029A2F4B03923946EF
:10E0B800A4F10A00029309F03EFFD7E714F8053CE3
:10E0C80014F8032C0694234407936E2A4FF0000398
:10E0D80008930993ADF820207FF42AAE06A8F2F73A
:10E0E800D5FD06A8F2F7C6FD06A8F2F7C3FD06A8F7
:10E0F800F2F7C0FD1CE62246A3E61C48083F13F0D1
:10E10800A1FFA6E61A4813F09DFF8DE728681FE7D0
:10E1180007480BF029FA0BB0BDE8F08F154A14F840
:10E12800023CC2F80C80CAF80090A5E5034667E7F0
:10E13800D22D002055540020A8430308B0430308FB
:10E1480070540020441E0020C4190020FD0101085D
:10E1580060380020DC430308C4480020DC2403089E
:10E16800C41C0308D8430308F46A0020A04303082A
:10E17800BC43030800ED00E0CC2D00202DE9F04F52
:10E188002DED028B95B0054615F0F8FEB14B1C78C5
:10E1980024B115B0BDEC028BBDE8F08FDFF820B3D9
:10E1A800DBF800305805F4D5AB4F3A68002A00F088
:10E1B8001B81AA4ED6F8283103F5F43348339D4223
:10E1C800C0F01281A64996F82C310968C6F8285182
:10E1D8000133DBB2890786F82C3101F11881580721
:10E1E80001F05680282B9F4B039301F0A6815E20F7
:10E1F80090479D4B1B78002B6BD0984E9B4AD6F8C6
:10E208003031EB1A934200F2C787DFF8B8A29AF8C8
:10E218000090B9F1000F33D1DFF86082D8F8000020
:10E2280002F00CFAC0B201280ED90228904F41F032
:10E238008C823B78002B41F0BE83D6F83831EB1A3C
:10E24800B3F57A6F81F066848A480268002A40D064
:10E258009AF80030BBB9884BD8F800001B689B7847
:10E268001E3B012B4FF0020141F2B283043015F03E
:10E27800CFFD012200238AF8002086F8443126E0E9
:10E288007C4802682AB3D6F8403140F6B731EB1A19
:10E298008B421ED996F83C31002B01F04D82013B90
:10E2A800DBB286F83C31002B01F01B8112F8011B10
:10E2B80096F84471026096F845317048CA190133DE
:10E2C800006886F8442186F8453102F0BBF9C6F8A3
:10E2D80040516B4A039B12781B68012A03F1010322
:10E2E8000C9300F0A686674B1B786BB1664F3B68B2
:10E2F80053B1039B594ED3F80090D6F85831A9EB87
:10E308000303632B00F23886DFF8BC8198F800908D
:10E31800B9F1020F01F0C180554F97F87430032B03
:10E3280000F08087594B1B7873B1594C23685BB157
:10E338004A4EFFF701FBD6F86431049044F61F6299
:10E34800C31A934200F2D280524B1B78002B4ED155
:10E35800514B1B7843B1414ED6F8B43203F5004314
:10E36800E8339D4280F0DF864C4B1B78002B3FF44E
:10E3780010AF3A4E4A4C4B4D06F2BD27206802F0CA
:10E388005DF900283FF405AF206802F04FF92B78BB
:10E3980080465A1E33B120682A7002F04FF90028CF
:10E3A800F2D1F6E603223946781E23F034F896F8BF
:10E3B800BC3296F8BD2286F8BF8283F47F4383F08F
:10E3C800FF039B1A1FFA88F89BB2B8EB132FD5D11D
:10E3D80096F8BE22DBB29A42D0D1781E1BF0B0F874
:10E3E8002B7818442870C9E71E4B039301E72E4C7D
:10E3F8002278002A40F014862C4F3C78002C65D1F6
:10E408002B4E3078002841F06182144E294CD6F802
:10E41800AC122278284B93FBF2F30B449D4297D31E
:10E4280096F8B032254AC6F8AC52D75CFB0701F122
:10E438008F83B90701F1D8837A0701F1248396F80D
:10E44800B0322178013393FBF1F201FB123386F8E5
:10E45800B0327DE755540020984500203C1A002032
:10E46800244500204C4700202A4600203F0D030089
:10E478000C000020904500208C4500208845002095
:10E488002B46002038460020745E002040460020BD
:10E498004446002068460020694600204A4600207D
:10E4A80050460020544600201C4600209D4F002066
:10E4B8009C4F0020A44F0020A0860100A04F002000
:10E4C8003C580020944500205E330020054E306EF5
:10E4D800002841F06A808146034B87F80090C3F812
:10E4E800AC5235E7AC4F00203C1A002096F86A3150
:10E4F800002B41F00780DC4B1A6802F00803002B60
:10E5080048F603414AF60B404BF60F4349F60747D6
:10E5180004BF03460F4612F0040F4FF0190118BF4D
:10E528001F46920686F86A1103D547F4804747F0DC
:10E53800200704F0DBFFC7F30909002841F07584C0
:10E54800CA4B9B79002B41F06984984664204FF0B0
:10E55800FF3A4FF0000C0C970D97ADF83CC0CDF882
:10E5680042C0CDF846C0CDF84AC0CDF83890ADF8D5
:10E578003E80ADF840A08DF84E000CAF0FCFDFF80D
:10E5880004E386F805C0AEE80F0097E80F00AEE890
:10E5980007002EF8023B71464FF0010C1B0CFE27BA
:10E5A8001F20C82201F81E39B770B27186F807C05B
:10E5B800F07096F87A01307180F0F10383EA031362
:10E5C800DAB2130983F0E70343EA022383EAC203BA
:10E5D8001BB283EA0312D2B2C3F3072383EA1213EE
:10E5E80043EA022383EAC2031BB283F0C80282EA29
:10E5F8000212D2B2C3F3072383EA121343EA0223B7
:10E6080083EAC2031BB283EA0C0787EA0717FFB243
:10E61800C3F3072282EA171242EA072200EB0C032F
:10E6280082EAC7070EEB0C0086F87A31378011F8BA
:10E63800013B7B4083EA0313DBB21A0982EA172203
:10E6480042EA032282EAC3031BB29FB281423780A7
:10E65800EDD183F07C0383EA0313DBB24FEA131E88
:10E668008EEA172E8EEA032E8EEAC30E0FFA8EFE5E
:10E678001FFA8EF9DFF810C2A6F800905FFA8EFE36
:10E688004FEA192986F8289086F827E00CF5D17802
:10E6980006F1220ADCF80000DCF80410DCF8082097
:10E6A800DCF80C3047460FC70CF1100CD445B846BF
:10E6B800F0D1DCF8000038606D4F9CF8043088F821
:10E6C800043007F1270886F8C9E186F8CA9117F8D7
:10E6D800011F206801F0B6FFB845F8D196F86B31F4
:10E6E800002B40F014876349039A097812680A20BE
:10E6F80086F86B01002901F0D6805F4F0129388820
:10E70800089041F2F8830229B7F802E001F0A783E4
:10E71800B8880790032901F0E483F8880690042953
:10E7280001F09D840529388901F094840629B7F8F9
:10E738000A9001F08B840729B7F80C8001F08384D4
:10E74800FB89059396F87A110C920B4683F03002F8
:10E7580082EA0212D2B217094849099387F07A0768
:10E7680047EA02270988337187EAC202444FC1EB9E
:10E77800012187FB013A089B4FF0000C63F30F0C53
:10E78800079B6EF31F4C4FF0000E63F30F0E069BB2
:10E79800CDF834C012B28A440027C91763F31F4E5C
:10E7A800C1EB6A2A059BCDF838E082EA021160F3D2
:10E7B8000F070020C9B268F30F00C2F3072269F3FC
:10E7C8001F4782EA111263F31F404FF000090F97A9
:10E7D8008DF845A010908DF8449042EA01220DF181
:10E7E800300C82EAC107BCE80F003FB287F0C808C6
:10E7F80088EA0818DFF88CE086F805905FFA88F850
:10E80800C7F30727AEE80F0087EA181747EA082377
:10E818009CE8030083EAC8031BB283F023024EF886
:10E82800040B82EA0212D2B2C3F30723099F83EAD8
:10E838001213704643EA022383EAC20207F1010C6D
:10E8480020F814194FF023081621FE27C82386F84C
:10E858007AC1328086F807800EF1020EB770F17027
:10E86800B371114612E000BF244500201445002072
:10E87800DF1B0020A0540020D2690020104F002088
:10E8880003082080441A00203E1A002010F8013B9B
:10E898004B4083EA0313DBB21A0982EA112242EAE7
:10E8A800032282EAC3031BB299B270453180EDD1CD
:10E8B80083F0F40383EA0313DBB24FEA131E8EEAF4
:10E8C800112E8EEA032E8EEAC30E0FFA8EFE1FFA61
:10E8D8008EF8E64FA6F800804FEA182C5FFA8EFEF5
:10E8E80086F81EE086F81FC07968BA683868FB6841
:10E8F80007F5D178A8E80F0038697969BA6906F28E
:10E90800A317A8E8070006F2C11886F8C1C186F85F
:10E91800C0E117F8011F206801F094FEB845F8D14E
:10E9280096F87271002F40F0E885D14B96F87AE19D
:10E93800B3F90010B3F90220B3F904309FEDCD6AA2
:10E94800777107EE103A039B1B680C938EF06A03ED
:10E9580083EA031306EE901AD9B20B0983F0D503A4
:10E9680043EA012383EAC1031BB283EA031152423B
:10E97800C9B207EE902AC3F3072383EA111343EAC7
:10E988000123F8EEE77AF8EEE66AB8EEC77A83EA8A
:10E99800C1031BB267EE867A66EE866A27EE067AB0
:10E9A800002083F0C808CDED0E7ACDED0D6A8DED0F
:10E9B8000F7A10901190129088EA081C0DF1300916
:10E9C8005FFA8CFCC3F30728B9E80F0088EA1C1823
:10E9D80048EA0C2888EACC08DFF8A8C20FFA88F8B9
:10E9E800ACE80F0088F01E0799E8070087EA0717C8
:10E9F800FFB2C8F3072383EA171343EA07238CE817
:10EA0800070083EAC7071C20C8214FF005094FF00B
:10EA18001E08FE230EF10102F07086F8729186F846
:10EA28000780B3700CF10C00B171ACF1100186F8DD
:10EA380004E0378086F87A2111F8013B7B4083EAAD
:10EA48000313DBB21A0982EA172242EA032282EA96
:10EA5800C3031BB29FB281423780EDD183F02703F5
:10EA680083EA0313DBB24FEA131E8EEA172E8EEAEF
:10EA7800032E8EEAC30E0FFA8EFE1FFA8EF9DFF808
:10EA8800ECC1A6F800905FFA8EFE4FEA192986F8C5
:10EA9800259086F824E00CF5D17806F1220ADCF8F6
:10EAA8000000DCF80410DCF80820DCF80C304746DD
:10EAB8000FC70CF1100CD445B846F0D16E4FBCF816
:10EAC8000030A8F8003007F1240886F8C6E186F877
:10EAD800C79117F8011F206801F0B4FDB845F8D1B7
:10EAE80096F873310393002B40F0038596F87AA1CA
:10EAF8005F4B624AB3F90410B2F90620604FDFF8A1
:10EB080088C1DFF880E186F804A08AF0220080EA54
:10EB18000010C0B2030983F0590343EA002383EAD3
:10EB2800C0031BB2B2F5FA6F83EA0310C0B2A8BFE4
:10EB38004FF4FA62C3F30723B2F57A7F83EA10131E
:10EB480043EA0023B8BF4FF47A7283EAC000A2F503
:10EB58007A72642303FB02F28CFB029CD31787FBB7
:10EB68000172C9174FF0000807B2C3EBAC13C1EB31
:10EB7800A2010DF13009CDF83080CDF83480CDF800
:10EB88003880CDF83C8087F0C80CADF84230ADF83D
:10EB98004010C846B8E80F008CEA0C1C5FFA8CFCE1
:10EBA800C7F3072787EA1C1747EA0C2787EACC0729
:10EBB800AEE80F003FB287F04A0383EA0313DBB2E3
:10EBC800C7F3072181EA131141EA0321724681EA5A
:10EBD800C303D8F800C09DF80C1071710AF1010741
:10EBE80005204A214FF0FE0886F87A7142F810C9CC
:10EBF80014274FF0C80C86F8730133800EF1040E09
:10EC0800F17186F80280F77086F806C0184612F887
:10EC1800011B414081EA0111C9B20B0983EA1023A3
:10EC280043EA012383EAC10109B288B27245308000
:10EC3800EDD181F0140181EA0111C9B24FEA111E28
:10EC48008EEA102E8EEA012E8EEAC10E0FFA8EFE83
:10EC58001FFA8EFC4FEA1C2A044B044886F81DA0B4
:10EC68005FFA8EFE86F81CE010E000BF3E1A002016
:10EC78002845002088C3E43ADF1B0020D269002021
:10EC880067666666441A0020D34D6210DA4F5968E9
:10EC98009A680068DB68A6F800C007F5D17CACE884
:10ECA8000F0038697969B7F81880ACE8030006F2F4
:10ECB800A317ACF8008086F8BFA1B84686F8BEE175
:10ECC80006F2BF1A18F8011F206801F0BBFCC24504
:10ECD800F8D1CA4BCA4A1B781278013B12F00100DE
:10ECE800DBB214BFC0214021172B03D8C54A1344F7
:10ECF8001B7B0393C44B1A8893071ABF002341F068
:10ED08001001012312F4027F18BF022312F0100F22
:10ED180018BF062312F0200F18BF1023002840F058
:10ED2800EA864FF0030C96F87AA10C938AF0460312
:10ED380083EA0313DAB2130983F0920343EA022346
:10ED480083EAC2031BB283EA0310C0B2C3F30722EB
:10ED580082EA101242EA002282EAC00212B282F06B
:10ED6800C80E8EEA0E1E00235FFA8EFE9DF80C80F8
:10ED78008DF834800320C2F307228DF837C082EA69
:10ED88001E128DF835308DF836108DF8380042EAAD
:10ED98000E2C99E807008CEACE0E0FFA8EFEDFF8EB
:10EDA8007482F3718EEA0E1CA8E803005FFA8CFCEB
:10EDB800CEF3072E8EEA1C1E4EEA0C2181EACC0CFB
:10EDC80096F808E088F800200FFA8CFC8EEA0C0E02
:10EDD8008EEA0E1E5FFA8EFECCF3072282EA1E121E
:10EDE80042EA0E22707AB17A96F80BC0737182EA01
:10EDF800CE0E0FFA8EFE80EA0E0080EA0012D2B222
:10EE0800CEF3072080EA121040EA022080EAC2000E
:10EE180000B2414081EA0111C9B2C0F3072282EA77
:10EE2800111242EA012282EAC10212B28CEA020CF1
:10EE38008CEA0C1C5FFA8CFCC2F3072282EA1C12D3
:10EE480042EA0C2296F80CE0707BB17B96F81090A1
:10EE580086F804A082EACC0212B28EEA020E8EEA8A
:10EE68000E1E5FFA8EFEC2F3072282EA1E1242EAE3
:10EE78000E2282EACE0212B2504080EA0010C0B2DE
:10EE8800C2F3072282EA101242EA002282EAC00292
:10EE980012B2514081EA0111C9B2C2F3072282EAD3
:10EEA800111242EA012282EAC102F17B13B281EA1D
:10EEB800030282EA0212D2B2C3F3072383EA1213CF
:10EEC80043EA022383EAC2031BB289EA030282EA05
:10EED8000212D2B2C3F3072383EA121343EA0223CE
:10EEE80083EAC2031BB283F0320282EA0212D2B270
:10EEF800C3F3072383EA121343EA022383EAC20314
:10EF08001BB29AB24FF0FE0C0AF10101DBB232805B
:10EF18004FF0090EC82086F802C04FEA122CA8F15B
:10EF28000E0286F803E0B07186F87A1186F812C0EE
:10EF38000393737458F80E0C5168926838F802AC51
:10EF48009DF80C3008F5CA7EAEE8070008F5D278BF
:10EF58008EF80290AEF800A086F8B4C186F8B331F6
:10EF680017F8011F206801F06DFBB845F8D1049B24
:10EF7800C6F86431FFF7E8B9DFF89CA0DFF89C8099
:10EF8800412014F099FCBAF9023088FB0320DB1702
:10EF9800C3EBA00080B214F075FCBAF9003088FB0E
:10EFA8000320DB17C3EBA00080B214F06BFCBAF9A6
:10EFB800043088FB0320DB17C3EBA00080B214F0F9
:10EFC80061FC124B3868197801F03CFB96F85C310B
:10EFD80013F0010800F0BF830D4AC6F858910133B9
:10EFE800DBB2A2FB0312D20802EB8202A3EB4203BC
:10EFF80086F85C31FFF788B93E1A00200C3B0020E8
:10F00800C04C0020D41C030878450020C46A0020A6
:10F01800CDCCCCCC441A0020284500206766666613
:10F028008B4B8C49186801F0D9FA00232370FFF73D
:10F03800E3B9894F386800283FF455A94FF0000A12
:10F048002346DFF84882854E049554469A4601F0D7
:10F05800F5FAF8B1F4B94FF001092546386801F01E
:10F06800E5FA83B27E2B00F02D8298F80120002A61
:10F078004BD196F84811C1B11B2B86F8482100F0F6
:10F08800FB810D2B47D0386888F8019001F0D6FA3B
:10F098000028E3D15346A24650460CAA7049049D65
:10F0A8001C4614F021FCFFF71EB97D2B00F0F183FC
:10F0B80096F84C2122B180F02003DBB286F84C117F
:10F0C80096F84721062A10D8B6F84A113868194424
:10F0D800A6F84A11B118013281F8503186F8472153
:10F0E80001F0ACFA0028B9D1D4E7B6F84A2188F87B
:10F0F800019013449BB21A0A52FA83F3FF2BA6F825
:10F108004A31386802D1574CA1E7386801F096FABD
:10F118000028A3D1BEE73868A6F84A2101F08EFA84
:10F1280000289BD1B6E796F8B832C6F8B452012B3E
:10F1380040F2068396F8B9224B49981801EB8001F2
:10F14800013202F001024F6A86F8B922BFB1474C7A
:10F158000D940DF15009123CA52349F8204D802249
:10F1680086F8103115232946484686F8112186F875
:10F178001231B847002840F0698296F8B8323C4A04
:10F18800013382FB0312A2EBE37202EB42029B1AE9
:10F1980086F8B832FFF7E8B8364A374B92F80BE0F2
:10F1A800039A1B881168D6F834213448891A4FF419
:10F1B8007A72DFB202FB0EF21B0A8777077591425B
:10F1C8004FF00007C37743758770077180F0A582F9
:10F1D8002B4B2C491A689B68C6F8305181FB02E713
:10F1E800D21781FB03E1C2EBA702DB17C3EBA10334
:10F1F80011124FEA232C4FF0F40E027701274177C2
:10F2080080F8203030217522782380F821C080F8DA
:10F218001AE0C77680F8221080F8232080F824307E
:10F22800FEF7F3BF184B0493186801F0FBF90028A8
:10F238003FF478A8049B0121186801F0EFF9022235
:10F24800002387F8742088F80030FFF76BB800BFF8
:10F25800984F0020DC450020844500203C1A0020FF
:10F26800821B00208C1B0020D41C0308611B00207B
:10F2780056555555484D0020404D00206C4F0020F4
:10F288005443002067666666703400200C00002036
:10F298005E2090473B6802209847C74BC74AB3F99E
:10F2A8004C3082FB03124FEAE378C8EBA2080FFA4E
:10F2B80088F85FFA88F014F0FFFDC8F3072014F00F
:10F2C800FBFD3B685E2098473B6803209847BC4B92
:10F2D8001B78D90740F1208107F03CF8B94B9FED26
:10F2E800BA7AD3ED037A67EE877AFCEEE77ACDED4A
:10F2F800037ABDF80C30002800F06383D8B24FEAD7
:10F30800132814F0D9FD404614F0D6FDAF4B1B78F6
:10F31800042B77D0DFF8E4A2B6F82E119AF8002073
:10F32800DFF8DC9291FBF2F302FB13139BB2B9F8FE
:10F338000010A6F82E314FEA03181FFA88F8642344
:10F3480003FB01235200B3FBF2F348EA0328C3F39B
:10F3580003225E203B681FFA88F848EA02089847AB
:10F368003B68062098475FFA88F014F0A5FD4FEA3D
:10F37800182014F0A1FD9649B6F82E214B7AB9F859
:10F3880000900132012BA6F82E2100F08B854A7BD4
:10F3980009EB89031FFA83F9002A40F0B6833B681A
:10F3A8005E2098473B683A2098478A4BA3FB093868
:10F3B8004FEA58181FFA88FA5FFA8AF014F07CFDB1
:10F3C8004FEA1A2014F078FD3B685E2098473B68A6
:10F3D8003B209847642303FB18939BB27748053377
:10F3E80080FB0320DB17C3EBA000C0B214F064FD60
:10F3F800002014F061FDDFF8F48198F80630002B46
:10F4080040F0108396F82C313A68FEF7EBBEDFF82F
:10F41800F4819FED718A4FF0240A5E209047504690
:10F428003B6898476D4BF8EC016A9B8A07EE103AE7
:10F43800F8EEE66AB8EEC77A0AF1010AC6EE877AEC
:10F448005FFA8AFA67EE887AFDEEE77ACDED037AFD
:10F45800BDF90C905FFA89F014F02EFDC9F307206E
:10F4680014F02AFDBAF1270F01D03A68D5E796F8CB
:10F478002C313A68FEF7B3BE386801F0DFF800288F
:10F488007FF401AE386886F8469188F8019001F05B
:10F49800D5F800287FF4E2ADFCE5FEF74DFA504BB5
:10F4A8001B68A0EB030A40F6B8339A4500F2E681E0
:10F4B8004C4A13793A2B00F0F783002388F8003080
:10F4C800FEF730BF386886F8465186F8475186F807
:10F4D800489188F8015001F0B1F800287FF4BEADDA
:10F4E800D8E596F8441196F845313F484A1CFEF78E
:10F4F800E6BE013B86F8733139E5013F86F8727143
:10F50800FFF7EEBA013B86F86A31FFF7E7B8013B2F
:10F5180086F86B31FFF704BA344A354BB2F80880E5
:10F52800A3FB08384FEA98085FFA88F014F0C4FC87
:10F538004FEA182014F0C0FCE8E64FF0000A5E20FD
:10F54800D3F8008086F82CA190473B68DFF8B89084
:10F5580017209847504614F0AFFC264BA3FB08230E
:10F568009B0BA9FB03125209C2EB0212A3EB820305
:10F57800D8B214F0A1FC3B685E2098473B6818207D
:10F5880098471D4BA3FB08239B09A9FB03125209AB
:10F59800C2EB0212A3EB8203D8B214F08DFC5046E2
:10F5A80014F08AFC3A68FEF722BE0024DFF85C807B
:10F5B800A1464FF0500A2EE0B455002067666666F3
:10F5C800C04C0020584D0020CDCC4C3E134F00209D
:10F5D800484D00201F85EB5100007A44304500203B
:10F5E800643300204C330020884500201445002057
:10F5F800CDCCCCCC73B2E745D34D6210564D00202C
:10F60800404D00206045002089888888393F0208DD
:10F61800DBB283F3118816F804B0601C59463044F5
:10F6280014F044F8002840F048810BF101031C4411
:10F63800EFF311838AF31288326E9442E8DB0022DA
:10F64800DBB2326683F31188FEF746BF0C9DA542F4
:10F658004FF000014FD941F2210014F8013B81EA33
:10F6680003235A0013F4004F80EA020192B289B2D0
:10F6780008BF11464A0080EA020311F4004F99B20C
:10F6880093B218BF0B46590080EA010213F4004FE9
:10F6980089B293B208BF0B465A0013F4004F80EAB0
:10F6A800020192B289B208BF11464A0080EA0203F9
:10F6B80011F4004F99B293B218BF0B465A0013F4D5
:10F6C800004F80EA020192B289B208BF11464B008E
:10F6D80011F4004F80EA03029BB292B208BF1A46A7
:10F6E800510080EA010312F4004F9BB289B218BF9F
:10F6F8001946AC42B1D14846F1F7FEFAB6490C9C1E
:10F70800B648641A152CA8BF1524224620F0A2FD7D
:10F71800B34A96F8B832147031E5B24B039A1B78A5
:10F728001268C6F83421013B012B3FF651AD102277
:10F738000223827003714BE514F0A0FBFEF7C7BDEE
:10F74800A94A02EB8302576A00E514F087FB0123FC
:10F758003B70FEF779BDA54B1B88DA0515D4D80692
:10F7680000F17A83990600F1AD835A0600F1B0835F
:10F77800180700F1B083D90700F1B08313F0020F26
:10F788000CBF4FF004084FF00C08994B994A1B78AE
:10F79800D27803F001030AB143F002035320049323
:10F7A80014F08AF8944A128802EB820202EB820271
:10F7B800900080B214F066F8002014F063F88F4AC5
:10F7C8008F4912883868C2EBC212520081FB02319D
:10F7D80011444FEAE27ACAEB612A5FFA8AFA514683
:10F7E80000F030FF874B38681A78049B48EA030812
:10F7F800844B8AEA020A002183F800A000F022FF65
:10F808004146386800F01EFF7E4B7E4A1B783868F8
:10F8180088EA0303DBB21946137000F013FF96F869
:10F828005C31002B7FF4D8AB4F2014F045F81EF064
:10F83800CFFD1EF0CDFD1EF0CBFD0121386800F094
:10F8480001FF714A6F4B92F800801B786D4A386847
:10F8580008F0010883F001034146137000F0F2FE3E
:10F86800684B684A1B78386888EA0303194613709E
:10F8780000F0E8FE96F85C31FFF7AEBB634AB2F8D9
:10F888005E3100210133A2F85E3188F80010FEF7DE
:10F8980049BD386886F84C9100F0D0FE00287FF406
:10F8A800DDABFFF7F7BB8846894608460691079106
:10F8B8008E4608910591FEF745BF41463A2013F060
:10F8C80051FE40EA09095FFA89F9AEE65049514B01
:10F8D8000093A1F13F07504B504A0B9101F8404C5F
:10F8E8000CA84F490A97F1F7DFFA0A9F7B1C0A9385
:10F8F8003C700A9B2922591C0A911A700A9BEA2219
:10F90800591C0A911A700A9BC822591C0A910CA802
:10F918001A701FF037FD00F101080CA942460A9839
:10F9280020F098FC0A9A02EB080301330A9302F8C4
:10F9380008400A9B5A1C0A921C700A9B5A1C0A927D
:10F948001C700A9B5A1C0A921C700A9B5A1C0A9229
:10F958001C700A9B5A1C0A921C700A9B5A1C0A9219
:10F968001C700A9B5A1C0A921C700A9B5A1C0A9209
:10F978001C700A9B5A1C0A921C700A9B5A1C0A92F9
:10F988001C700A9B5A1C0A921C700A9B5A1C0A92E9
:10F998001C700A9B0122991814A80A911A7050F831
:10F9A800283DDB1B3B7014F0A9FA184B3470C3F8E0
:10F9B800AC52FEF7CDBCC6F8385187F80090FEF778
:10F9C80043BCDBF80020D2067FF598AC804698E46B
:10F9D80000F024FEFEF74DBC4C1B00202C3C002000
:10F9E800413C0020134F0020D41C03087845002018
:10F9F800C04C0020184F0020404D0020104F002020
:10FA080003082080C46A0020203900203C1A002006
:10FA1800DC4500207654002000440308084403080D
:10FA2800144403083B68DFF87492DFF86CA25E2088
:10FA380098473B6828209847D9F800308AFB032A62
:10FA4800DB17C3EBAA0A5FFA8AF014F035FACAF397
:10FA5800072014F031FA3B685E2098473B68042081
:10FA68009847B8F80830002B40F00182D9F80830E0
:10FA780083F310085FFA88F014F01EFAC8F3072021
:10FA880014F01AFABEE47A4B7A4A0D93A3F14008AF
:10FA98001268002103F8401C212388F80230D300A3
:10FAA80040F1F48174490327744B1B88580500F111
:10FAB800EA81DA0700F1098203F00203704A002B99
:10FAC8001CBF03271146DFF8D8913A46484620F074
:10FAD800C1FB07EB090314A80133A9F1020140F89F
:10FAE800203D00225B1A07F8092088F8013014F03D
:10FAF80005FAFEF7A4BC634AD278002A0CBF4FF07F
:10FB0800040C4FF0050CFFF70EB99AF8003099FB7A
:10FB1800F3F944E40123D8F800003B7000F086FDB7
:10FB28000746D8F8000000F081FD79067EF48CAB1A
:10FB38008E287EF489AB9AF80030002B7EF4A0ABB7
:10FB4800514B524A1A602D2386F83C31FEF783BB8D
:10FB5800DFF850919FED4E8AB9F90230444A0D9270
:10FB680007EE903AF8EEE77A0DF1500867EE887ADA
:10FB7800A2F14003FDEEE77AA2F13D0148F8201D0D
:10FB880002F8400C0822CDED037A5A701E229A70B2
:10FB9800BDF80C104046F1F789F8B9F9003007EEC6
:10FBA800903AF8EEE77A404667EE887AFDEEE77A13
:10FBB800CDED037ABDF80C10F1F778F8B9F90430F7
:10FBC80007EE903AF8EEE77A404667EE887AFDEE5F
:10FBD800E77ACDED037ABDF80C10F1F767F84046E7
:10FBE80014F08CF9FEF725BC214A2A4B0D920DF131
:10FBF8005008A2F13D0048F8200D1988DFF89C90C4
:10FC0800A2F1400300204FF00A0E02F8400C08222F
:10FC180083F801E040469A70F1F748F8D9F80030C7
:10FC28001D49DA1781FB0313C2EBA30399B24046BF
:10FC3800F1F73CF803F068FCD9F808900C9B4FEA00
:10FC48001942591C0C911A700C9B4FEA1922591C25
:10FC58000C911A700C9B5A1C0C9283F800900C9B08
:10FC68005A1C0C921870404614F048F9FEF7E4BB91
:10FC7800DC45002018390020EC43030878450020B3
:10FC8800FC430308184F0020904500206C4F0020CB
:10FC980058A08B41404D002067666666544300209B
:10FCA8009F450020284500209178049210460DF0C9
:10FCB80045FD049A00287FF400AC9349934F944B78
:10FCC800944E09880592944AF961F863B6F85E1172
:10FCD80018689B68C7F86CA0F862FB641068F9653F
:10FCE800049200F05BFA824600287EF416AB049B6F
:10FCF8004946186800F092FC059A96F86031D27867
:10FD08000692642B4FF0040287F8742040F01681A5
:10FD180096F86131072B08BF86F861A196F8613122
:10FD2800089307EB0319D9F80410059108461FF04A
:10FD380029FBD9F8081007915FFA80F908461FF0E7
:10FD480021FB5FFA80FA089B74480599059009EB36
:10FD58000A020832C27123F00F0282726F4A03F05E
:10FD68000F0353736D4B0AEBC900987318464A4644
:10FD78000F3020F06FFA6A4B079909F1090018440F
:10FD8800524620F067FA0598C37903F10109CBB10F
:10FD9800013B5FFA83FC0CF1080CDFF89CE184441A
:10FDA8000023073010F8012B5A409300D10883EA4A
:10FDB800420301F0180153404EFA01F253408445C2
:10FDC800DBB2EFD1564A069809F8023020F024FA3F
:10FDD80096F861310022013386F8613186F8602196
:10FDE800059BDDF814909B785BB1049B19F804100F
:10FDF800186800F027FC013499F80230E4B2A342F5
:10FE0800F3D896F860310322013386F8603187F819
:10FE1800742088F80020049BFFF706BA3C4B804604
:10FE2800B3F900A06420FEF794BB374B3D4A1B880A
:10FE3800927903EB830303EB83034FEA83081FFAEA
:10FE480088F8002A54D14FF0FF330FFA83FA03F0F1
:10FE58005BFB40B2FEF77DBB4FF0340895E4984653
:10FE680099461846069307930593FEF76BBC03F073
:10FE78004BFB14F021F8002014F01EF896F82C31F2
:10FE88003A68FEF7AFB9032727491CE6DBF80030CC
:10FE9800264A274903F48003002B16BF114604277E
:10FEA800032701E63B685E2098473B68392098475E
:10FEB8005FFA89F014F000F84FEA192013F0FCFFFC
:10FEC800FFF799BA4FF024085FE41A490427FAE5C6
:10FED8004FF0100859E44FF0200856E44FF0080896
:10FEE80053E498469946184606930593FEF72ABCAC
:10FEF800074B1B68A9E79846994618460693079347
:10FF08009E460593FEF71EBC404D00200C000020C5
:10FF1800544300203C1A0020703400204C5E00201E
:10FF2800525E002014450020F0430308EC43030808
:10FF3800E4430308F44303080007090E97F8759093
:10FF48004B494C4A059219F00F0F04BF09F10109FA
:10FF58005FFA89F9B9F1070F28BF4FF001094FEA95
:10FF6800091A07EB0A035FFA8AFC187C0023095C6C
:10FF7800937202F10D0307EB0A024CEA0000012913
:10FF88001870D26803F1010E0CD90239C9B2881C65
:10FF98001844734603F8012B83424FEA1222F9D121
:10FFA80001318E44BA4422F0600309F101099AF83C
:10FFB80011205FFA89F91343B9F1080F8EF8003060
:10FFC8000EF1010351D04FEA091A07EB0A012A4A38
:10FFD800087C2749095C9A1A02EB010E0CF1100CF7
:10FFE800BEF1130F5FFA8CFCC5DDD2B2931DDBB2F4
:08FFF8000598DFF88CE043F0EE
:020000040801F1
:100000004001C17103F1010CCBB105325FFA82FAF4
:100010000AF1080A824400230EF1010010F8011BC6
:1000200059408B0083EA4103CA084B40154902F04E
:10003000180241FA02F253408245DBB2EED1069833
:100040000CF80E3087F8759020F0EAF8CCE60593AE
:10005000FEF77CBB98460593FEF778BB9846994619
:100060000593FEF773BB9846994618460593FEF72D
:100070006DBB034A9A1ABCE7D41C03084C5E0020EF
:10008000595E00200007090E525E0020436A826913
:10009000D154436A0169826B01338B4228BF00232C
:1000A0004362002A2FD0EFF31181502383F312888B
:1000B000836B1A68D2072CD470B45E686EB9456A37
:1000C000826A954217D084691444DC600ED9AA1A5A
:1000D0005A608562002280F854201A6842F00102BA
:1000E000C9B21A6081F3118870BC70470469A21A02
:1000F0005A608662EEE7012380F85430C9B281F37A
:10010000118870BC7047026D136843F08003136060
:100110007047C9B281F31188704700BF426B10B4B9
:1001200062B1436CC2684469D11A013B615C5DF8FD
:10013000044B08BF13464364C8B27047016A436961
:10014000C4685B5C0131A14228BF114601625DF8C1
:10015000044BD8B2704700BF836B13B190F85400C2
:100160007047836A406A181AB0FA80F040097047F5
:10017000416A836A99420AD3CB1A816B026961B1E1
:100180004968501E0B4483420AD2C01A7047026964
:100190001144CB1A816B0029F2D1501EC01A70474E
:1001A00000207047436B43B1426C5B6893422FBFA2
:1001B000981AC0689B1AC0187047C269036A9A42AD
:1001C0002FBFD01AC0688018C01A70470A4B30B5CC
:1001D00003F1140493F900205D78072AC8BF143A8C
:1001E000811804330D7313F8025C855413F8012C45
:1001F0000A76A342EED130BD081D030803682DE93D
:10020000F041DF691FB13B46BDE8F0411847002AC5
:10021000164611DD04460D460E4400E023689B6837
:10022000204698470028F9D0236815F8011B1B6861
:1002300020469847AE42F1D1BDE8F0810023232249
:10024000027043708370C3707047152303701623C8
:10025000C370172383712D2343702E2303712F2323
:10026000C371704730B50446006D61710368A268C0
:1002700023F00103036087B0A379009213F0040216
:100280003DD04FF4805213F00203019244D1029307
:100290004FF480630022039311F00103059237D1DC
:1002A000049308238D07694648BF049319F024F886
:1002B0006079236DA17900F00202002A15BF4FF486
:1002C00040324FF480324FF40034002410F0010F1C
:1002D000586808BF2246CC074CBF024320EA0202FE
:1002E0005A609A6809074CBF42F0080222F00802DF
:1002F0009A601A6842F001021A6007B030BD13F02C
:10030000020301920BD04FF4005513460295C1E74A
:10031000042304930C23C5E74FF40053B7E702937B
:10032000B8E700BF10B50446006DA160036823F074
:1003300001030360A37986B013F00402009141D059
:100340004FF4805213F00203019244D102934FF410
:10035000806362790393D1074FF000030493059300
:1003600045BF0423049308230C236946920748BF22
:10037000049318F0C1FF6079236DA17900F00202A7
:10038000002A15BF4FF440324FF480324FF400344E
:10039000002410F0010F586808BF2246CC074CBF5C
:1003A000024320EA02025A609A6809074CBF42F0F1
:1003B000080222F008029A601A6842F001021A60EC
:1003C00006B010BD13F00203019207D04FF40051A4
:1003D00013460291BDE74FF40053B7E70293B8E725
:1003E00000232622036002702722827001224360CC
:1003F00002718371704700BF1D4B70B59C68236DFF
:10040000626BDD69C2B1A36B2BB12B0702D5236DE3
:1004100008221A6270BD2A06F7D5A26A616A8A426A
:1004200020D0511CA069A162825C2069266D8142A6
:100430003285EAD3A362E8E7A906E4D5E26A22B1ED
:10044000988C216B80B29047DDE7E1699B8C6069F5
:10045000DBB24E1CE6614354E169E368994228BF70
:10046000E261D0E7226D136823F080031360CCE7CC
:10047000782500201D4B70B55C68236D626BDD69CB
:10048000C2B1A36B2BB12B0702D5236D08221A62D0
:1004900070BD2A06F7D5A26A616A8A4220D0511C33
:1004A000A069A162825C2069266D81423285EAD30F
:1004B000A362E8E7A906E4D5E26A22B1988C216B31
:1004C00080B29047DDE7E1699B8C6069DBB24E1C2E
:1004D000E6614354E169E368994228BFE261D0E7ED
:1004E000226D136823F080031360CCE77825002089
:1004F0001D4B70B51C68236D626BDD69C2B1A36BC7
:100500002BB12B0702D5236D08221A6270BD2A0673
:10051000F7D5A26A616A8A4220D0511CA069A16203
:10052000825C2069266D81423285EAD3A362E8E7C6
:10053000A906E4D5E26A22B1988C216B80B290477B
:10054000DDE7E1699B8C6069DBB24E1CE6614354D8
:10055000E169E368994228BFE261D0E7226D136840
:1005600023F080031360CCE77825002070B4EFF30C
:100570001186502383F31288836B1A68D20720D424
:100580005D686DB9446A826A944217D081691144EA
:10059000D9600ED9A21A5A608462002280F85420D1
:1005A0001A6842F00102F1B21A6081F3118870BC3E
:1005B000704701698A1A5A608562EEE7012380F864
:1005C0005430F1B281F3118870BC704703685B6AE4
:1005D00003B11847704700BF03681B6A03B118478F
:1005E000704700BF03682DE9F041DF691FB13B464A
:1005F000BDE8F0411847002A164611DD04460D46B5
:100600000E4400E023689B68204698470028F9D0F4
:10061000236815F8011B1B6820469847AE42F1D1AC
:10062000BDE8F08103689B69184700BF03685B69F8
:10063000184700BF0368DB68184700BF03689B6862
:10064000184700BF03685B68184700BF03681B6852
:10065000184700BF054B53F8203033B11A689B8808
:10066000918A0B4218BF1B04936170471847002002
:1006700003682DE9F04F03F13845644EAD0A0124BB
:10068000755D05F01F066D09022D04FA06F400F0F1
:10069000A280032D00F0A480012D52D08088B0FAF2
:1006A00080F4C4F11F04A4B2E50803EB850504F04F
:1006B00007042E6AA4000F27A74026EA07062E6229
:1006C0002E6A01F0030702FA04F47A1E3443012A69
:1006D000C1F3810CC1F300182C62C1F3411135D96B
:1006E000C60700F19780850700F1A380440700F159
:1006F000B180020700F1BF80C60600F1CD808506FB
:1007000000F1DB80440600F1E980020600F1F78089
:10071000C60500F10581850500F11381440500F14E
:100720002181020500F12F81C60400F13D8185047D
:1007300000F14B81440400F15981020455D4BDE815
:10074000F08F334D6E6934436C61A7E70024224675
:100750004FF0010E4FF0030904E00132102A04F1BA
:100760000204ECD00EFA02F636EA0005F5D1D3F811
:1007700008A009FA04F5ED430AEA050AC3F808A03F
:10078000D3F808B00CFA04FA4AEA0B0AC3F808A036
:10079000B3F804A01FFA8AFA2AEA06069E80B3F884
:1007A00004A008FA02F646EA0A06B6B29E801E685F
:1007B0002E401E60D3F800A007FA04F646EA0A06A7
:1007C0001E60D3F80CA001FA04F605EA0A0A46EA0C
:1007D0000A05DD60C1E70E4DAE693443AC615DE7EB
:1007E0000B4DEE693443EC6158E71A6822F0404241
:1007F0001A601A6842EA87771F60DA6822F040427E
:1008000042EA8171D960BDE8F08F00BFD43A030895
:10081000001002401A6822F003021A601A683A4374
:100820001A60DA6822F003020A438507DA607FF56E
:100830005DAF1A6822F00C021A601A6842EA870259
:100840001A60DA6822F00C0242EA81024407DA6098
:100850007FF54FAF1A6822F030021A601A6842EA38
:1008600007121A60DA6822F0300242EA0112DA60F6
:1008700002077FF541AF1A6822F0C0021A601A68B9
:1008800042EA87121A60DA6822F0C00242EA811254
:10089000C606DA607FF533AF1A6822F440721A6038
:1008A0001A6842EA07221A60DA6822F4407242EAC1
:1008B00001228506DA607FF525AF1A6822F44062CE
:1008C0001A601A6842EA87221A60DA6822F44062E3
:1008D00042EA81224406DA607FF517AF1A6822F4F3
:1008E00040521A601A6842EA07321A60DA6822F443
:1008F000405242EA0132DA6002067FF509AF1A6817
:1009000022F440421A601A6842EA87321A60DA68B2
:1009100022F4404242EA8132C605DA607FF5FBAE3E
:100920001A6822F440321A601A6842EA07421A60D2
:10093000DA6822F4403242EA01428505DA607FF546
:10094000EDAE1A6822F440221A601A6842EA874221
:100950001A60DA6822F4402242EA81424405DA60F1
:100960007FF5DFAE1A6822F440121A601A6842EA74
:1009700007521A60DA6822F4401242EA0152DA6041
:1009800002057FF5D1AE1A6822F440021A601A6897
:1009900042EA87521A60DA6822F4400242EA81523F
:1009A000C604DA607FF5C3AE1A6822F040721A609E
:1009B0001A6842EA07621A60DA6822F0407242EA74
:1009C00001628504DA607FF5B5AE1A6822F04062F4
:1009D0001A601A6842EA87621A60DA6822F0406296
:1009E00042EA81624404DA607FF5A7AE1A6822F019
:1009F00040521A601A6842EA07721A60DA6822F0F6
:100A0000405242EA0172DA6097E600BF036803F1E0
:100A100038422DE9F04F920A584DAA5C02F01F05AA
:100A200052090124022A04FA05F400F08C80032AFA
:100A300000F08E80012A3CD001F003077A1E012AC3
:100A4000C1F3810CC1F300188088C1F3411135D97D
:100A5000C60700F19780850700F1A380440700F1E5
:100A6000B180020700F1BF80C60600F1CD80850687
:100A700000F1DB80440600F1E980020600F1F78016
:100A8000C60500F10581850500F11381440500F1DB
:100A90002181020500F12F81C60400F13D8185040A
:100AA00000F14B81440400F15981020455D4BDE8A2
:100AB000F08F334A55692C435461BDE70024224628
:100AC0004FF0010E4FF0030904E00132102A04F147
:100AD0000204ECD00EFA02F636EA0005F5D1D3F89E
:100AE00008A009FA04F5ED430AEA050AC3F808A0CC
:100AF000D3F808B00CFA04FA4AEA0B0AC3F808A0C3
:100B0000B3F804A01FFA8AFA2AEA06069E80B3F810
:100B100004A008FA02F646EA0A06B6B29E801E68EB
:100B20002E401E60D3F800A007FA04F646EA0A0633
:100B30001E60D3F80CA001FA04F605EA0A0A46EA98
:100B40000A05DD60C1E70E4A95692C43946173E79D
:100B50000B4AD5692C43D4616EE71A6822F04042F3
:100B60001A601A6842EA87771F60DA6822F040420A
:100B700042EA8171D960BDE8F08F00BFD43A030822
:100B8000001002401A6822F003021A601A683A4301
:100B90001A60DA6822F003020A438507DA607FF5FB
:100BA0005DAF1A6822F00C021A601A6842EA8702E6
:100BB0001A60DA6822F00C0242EA81024407DA6025
:100BC0007FF54FAF1A6822F030021A601A6842EAC5
:100BD00007121A60DA6822F0300242EA0112DA6083
:100BE00002077FF541AF1A6822F0C0021A601A6846
:100BF00042EA87121A60DA6822F0C00242EA8112E1
:100C0000C606DA607FF533AF1A6822F440721A60C4
:100C10001A6842EA07221A60DA6822F4407242EA4D
:100C200001228506DA607FF525AF1A6822F440625A
:100C30001A601A6842EA87221A60DA6822F440626F
:100C400042EA81224406DA607FF517AF1A6822F47F
:100C500040521A601A6842EA07321A60DA6822F4CF
:100C6000405242EA0132DA6002067FF509AF1A68A3
:100C700022F440421A601A6842EA87321A60DA683F
:100C800022F4404242EA8132C605DA607FF5FBAECB
:100C90001A6822F440321A601A6842EA07421A605F
:100CA000DA6822F4403242EA01428505DA607FF5D3
:100CB000EDAE1A6822F440221A601A6842EA8742AE
:100CC0001A60DA6822F4402242EA81424405DA607E
:100CD0007FF5DFAE1A6822F440121A601A6842EA01
:100CE00007521A60DA6822F4401242EA0152DA60CE
:100CF00002057FF5D1AE1A6822F440021A601A6824
:100D000042EA87521A60DA6822F4400242EA8152CB
:100D1000C604DA607FF5C3AE1A6822F040721A602A
:100D20001A6842EA07621A60DA6822F0407242EA00
:100D300001628504DA607FF5B5AE1A6822F0406280
:100D40001A601A6842EA87621A60DA6822F0406222
:100D500042EA81624404DA607FF5A7AE1A6822F0A5
:100D600040521A601A6842EA07721A60DA6822F082
:100D7000405242EA0172DA6097E600BF10B50409FA
:100D8000013C052C17D80D4B33F8142000F00F0050
:100D900042FA00F313F001030DD0012303FA00F02F
:100DA000013810401EF0ECFF054A064B125D10445E
:100DB00003EBC00010BD002010BD00BFA43B030822
:100DC000B03B0308CC4900202DE9F04F4A484B4B7B
:100DD0004B4C4FF090414FF0010A4FF002094FF099
:100DE00004084FF0080C4FF0100E202740268025F5
:100DF00030F8022B12F0010F03D01960A3F804A001
:100E0000083312F0020F03D01960A3F804900833DE
:100E100012F0040F03D01960A3F80480083312F015
:100E2000080F03D01960A3F804C0083312F0100FA4
:100E300003D01960A3F804E0083312F0200F02D0A9
:100E400019609F80083312F0400F02D019609E8015
:100E5000083312F0800F02D019609D80083312F41D
:100E6000807F05D04FF4807B1960A3F804B008336D
:100E700012F4007F05D04FF4007B1960A3F804B092
:100E8000083312F4806F05D04FF4806B1960A3F81B
:100E900004B0083312F4006F05D04FF4006B1960F2
:100EA000A3F804B0083312F4805F05D04FF4805BE0
:100EB0001960A3F804B0083312F4005F05D04FF4B2
:100EC000005B1960A3F804B0083312F4804F05D01A
:100ED0004FF4804B1960A3F804B00833D20B04D050
:100EE0004FF4004219609A80083301F58061A142F5
:100EF0007FF47EAFBDE8F08FA43B0308CC4900200F
:100F000000180048002867D003682DE9F04F03F16E
:100F100038445C4EA40A0125345D04F01F066409C0
:100F2000022C05FA06F558D0032C00F0A580012C00
:100F300058D08088B0FA80F4C4F11F04A4B2E50848
:100F400003EB850504F007042E6AA4000F27A740D1
:100F500026EA07062E622E6A01F00307A2407C1ED5
:100F60003243012CC1F3810CC1F300182A62C1F392
:100F700041113CD9C60700F18980850700F19580B1
:100F8000440700F1A380020700F1B180C60600F11A
:100F9000BF80850600F1CD80440600F1DB800206AB
:100FA00000F1E980C60500F1F780850500F10581B3
:100FB000440500F11381020500F12181C60400F10E
:100FC0002F81850400F13D81440400F14B8102042E
:100FD00000F15981BDE8F08F70472B4CA66935436D
:100FE000A561A6E7284C666935436561A1E7002441
:100FF00022464FF0010E4FF0030904E00132102A9F
:1010000004F10204E6D00EFA02F636EA0005F5D144
:10101000D3F808A009FA04F5ED430AEA050AC3F873
:1010200008A0D3F808B00CFA04FA4AEA0B0AC3F88D
:1010300008A0B3F804A01FFA8AFA2AEA06069E80DE
:10104000B3F804A008FA02F646EA0A06B6B29E8091
:101050001E682E401E60D3F800A007FA04F646EA88
:101060000A061E60D3F80CA001FA04F605EA0A0A83
:1010700046EA0A05DD60C1E7034CE6693543E561F0
:1010800057E700BFD43A0308001002401A6822F064
:1010900003021A601A683A431A60DA6822F00302FF
:1010A0000A438507DA607FF56BAF1A6822F00C02FD
:1010B0001A601A6842EA87021A60DA6822F00C02A3
:1010C00042EA81024407DA607FF55DAF1A6822F0D8
:1010D00030021A601A6842EA07121A60DA6822F0CF
:1010E000300242EA0112DA6002077FF54FAF1A6858
:1010F00022F0C0021A601A6842EA87121A60DA689F
:1011000022F0C00242EA8112C606DA607FF541AFE2
:101110001A6822F440721A601A6842EA07221A60BA
:10112000DA6822F4407242EA01228506DA607FF52D
:1011300033AF1A6822F440621A601A6842EA8722C2
:101140001A60DA6822F4406242EA81224406DA60D8
:101150007FF525AF1A6822F440521A601A6842EAF5
:1011600007321A60DA6822F4405242EA0132DA6049
:1011700002067FF517AF1A6822F440421A601A6817
:1011800042EA87321A60DA6822F4404242EA813247
:10119000C605DA607FF509AF1A6822F440321A609A
:1011A0001A6842EA07421A60DA6822F4403242EAD8
:1011B00001428505DA607FF5FBAE1A6822F4402211
:1011C0001A601A6842EA87421A60DA6822F44022FA
:1011D00042EA81424405DA607FF5EDAE1A6822F4F6
:1011E00040121A601A6842EA07521A60DA6822F45A
:1011F000401242EA0152DA6002057FF5DFAE1A685A
:1012000022F440021A601A6842EA87521A60DA68C9
:1012100022F4400242EA8152C604DA607FF5D1AE80
:101220001A6822F040721A601A6842EA07621A606D
:10123000DA6822F0407242EA01628504DA607FF5E2
:10124000C3AE1A6822F040621A601A6842EA8762E6
:101250001A60DA6822F0406242EA81624404DA608D
:101260007FF5B5AE1A6822F040521A601A6842EA59
:1012700007721A60DA6822F0405242EA0172DA60BC
:1012800002047FF5A7AE1A6822F040421A601A687D
:1012900042EA87771F60DA6822F0404242EA8171B1
:1012A000D960BDE8F08F00BF002852D0036803F179
:1012B00038422DE9F04F920A504DAA5C02F01F050A
:1012C00052090124022A04FA05F443D0032A00F04B
:1012D0009080012A43D001F003077A1E012AC1F34E
:1012E000810CC1F300188088C1F341113CD9C607B5
:1012F00000F18880850700F19480440700F1A28006
:10130000020700F1B080C60600F1BE80850600F13C
:10131000CC80440600F1DA80020600F1E880C605C0
:1013200000F1F680850500F10481440500F1128189
:10133000020500F12081C60400F12E81850400F130
:101340003C81440400F14A81020400F15881BDE867
:10135000F08F70472A4A95692C439461BBE7284A6D
:1013600055692C435461B6E7002422464FF0010E24
:101370004FF0030904E00132102A04F10204E6D020
:101380000EFA02F636EA0005F5D1D3F808A009FAFC
:1013900004F5ED430AEA050AC3F808A0D3F808B03B
:1013A0000CFA04FA4AEA0B0AC3F808A0B3F804A03E
:1013B0001FFA8AFA2AEA06069E80B3F804A008FA01
:1013C00002F646EA0A06B6B29E801E682E401E60ED
:1013D000D3F800A007FA04F646EA0A061E60D3F81E
:1013E0000CA001FA04F605EA0A0A46EA0A05DD60DD
:1013F000C1E7034AD5692C43D4616CE7D43A0308AA
:10140000001002401A6822F003021A601A683A4378
:101410001A60DA6822F003020A438507DA607FF572
:101420006CAF1A6822F00C021A601A6842EA87024E
:101430001A60DA6822F00C0242EA81024407DA609C
:101440007FF55EAF1A6822F030021A601A6842EA2D
:1014500007121A60DA6822F0300242EA0112DA60FA
:1014600002077FF550AF1A6822F0C0021A601A68AE
:1014700042EA87121A60DA6822F0C00242EA811258
:10148000C606DA607FF542AF1A6822F440721A602D
:101490001A6842EA07221A60DA6822F4407242EAC5
:1014A00001228506DA607FF534AF1A6822F44062C3
:1014B0001A601A6842EA87221A60DA6822F44062E7
:1014C00042EA81224406DA607FF526AF1A6822F4E8
:1014D00040521A601A6842EA07321A60DA6822F447
:1014E000405242EA0132DA6002067FF518AF1A680C
:1014F00022F440421A601A6842EA87321A60DA68B7
:1015000022F4404242EA8132C605DA607FF50AAF32
:101510001A6822F440321A601A6842EA07421A60D6
:10152000DA6822F4403242EA01428505DA607FF54A
:10153000FCAE1A6822F440221A601A6842EA874216
:101540001A60DA6822F4402242EA81424405DA60F5
:101550007FF5EEAE1A6822F440121A601A6842EA69
:1015600007521A60DA6822F4401242EA0152DA6045
:1015700002057FF5E0AE1A6822F440021A601A688C
:1015800042EA87521A60DA6822F4400242EA815243
:10159000C604DA607FF5D2AE1A6822F040721A6093
:1015A0001A6842EA07621A60DA6822F0407242EA78
:1015B00001628504DA607FF5C4AE1A6822F04062E9
:1015C0001A601A6842EA87621A60DA6822F040629A
:1015D00042EA81624404DA607FF5B6AE1A6822F00E
:1015E00040521A601A6842EA07721A60DA6822F0FA
:1015F000405242EA0172DA6002047FF5A8AE1A682E
:1016000022F040421A601A6842EA87771F60DA685F
:1016100022F0404242EA8171D960BDE8F08F00BFFC
:1016200010B1036882881A85704700BF10B1036843
:1016300082889A61704700BF38B1002983880268A8
:1016400014BF002110218B40936170470E4B1B8803
:1016500001463BB90D4B0E4A1B7810680BB981F05F
:101660000101E9E70B4B5A691AB118B91A68106001
:1016700058747047084A18681188084A92FBF1F2BA
:10168000012102605974704724470020264700203A
:10169000284700202C4700204447002020A10700B5
:1016A00010B40A4B0A4A1C7801238340234052F8A5
:1016B000200029B9B3FA83F149095DF8044BBBE76F
:1016C000191C18BF01215DF8044BB5E71447002031
:1016D0001847002030B1036882881B8A1A4214BF61
:1016E00001200020704700BF2DE9F0410B4E346807
:1016F00073691C400FD0DFF828800127B4FA84F307
:10170000C3F11F0307FA03F558F82300036898474D
:10171000AC437561F2D1BDE8F08100BF0004014027
:10172000FC1C00202DE9F0410B4E346873691C400D
:101730000FD0DFF828800127B4FA84F3C3F11F0328
:1017400007FA03F558F8230003689847AC4375611E
:10175000F2D1BDE8F08100BF00040140FC1C002074
:101760002DE9F0410B4E346873691C400FD0DFF84F
:1017700028800127B4FA84F3C3F11F0307FA03F5A5
:1017800058F8230003689847AC437561F2D1BDE86F
:10179000F08100BF00040140FC1C00202DE9F04155
:1017A0000B4E346873691C400FD0DFF82880012786
:1017B000B4FA84F3C3F11F0307FA03F558F82300C2
:1017C00003689847AC437561F2D1BDE8F08100BF72
:1017D00000040140FC1C00202DE9F0410B4E346850
:1017E00073691C400FD0DFF828800127B4FA84F316
:1017F000C3F11F0307FA03F558F82300036898475D
:10180000AC437561F2D1BDE8F08100BF0004014036
:10181000FC1C00202DE9F0410B4E346873691C401C
:101820000FD0DFF828800127B4FA84F3C3F11F0337
:1018300007FA03F558F8230003689847AC4375612D
:10184000F2D1BDE8F08100BF00040140FC1C002083
:101850002DE9F0410B4E346873691C400FD0DFF85E
:1018600028800127B4FA84F3C3F11F0307FA03F5B4
:1018700058F8230003689847AC437561F2D1BDE87E
:10188000F08100BF00040140FC1C0020084A93695D
:1018900010B5084C43F0010393612046402200211B
:1018A0001FF0D7FD4FF0FF332364C4F8433010BD61
:1018B00000100240FC1C002003685B6A184700BF50
:1018C0002DE9F041044618460D46164698461DF08F
:1018D0005DFD2768E6722844A07229467D6943466B
:1018E00032462046AC46BDE8F0416047036810B57B
:1018F00004461B689847236820469B689847A37B4B
:101900000133A37310BD00BF10B5036804469B6884
:101910009847FF2301226373227310BD08B5FFF7B8
:101920002DFA38B12D2282710022C2712021BDE82A
:101930000840B9E408BD00BF0B4B984206D0A3F5A0
:10194000784398420DD04FF0FF3070470022074B8C
:1019500003EB02135A89013292B25A81588980B23C
:1019600070470122F3E700BF0030014074470020B8
:10197000F0B50D460178012983B00446164618D00B
:10198000022902D0002003B0F0BD80681F46FFF797
:1019900047FE45F080016068EFF7C4FC3B463246E5
:1019A00000216068EFF720FDA068FFF73FFE0120EF
:1019B000E9E790F90400421CE4D00228E2DC6179F6
:1019C00000962A46F0F750FBDDE700BF427A02B9E5
:1019D000704710B504460368406804F10A0198474F
:1019E0000023637210BD00BF437A5A1C0344D2B275
:1019F00042729972037A934200D802B9704710B5C7
:101A000004460368406804F10A01984700236372A2
:101A100010BD00BF98B10B4B012210B402FA01F1C6
:101A200003F1750402E00333A34209D01A7882421D
:101A3000F9D15A780A42F6D001205DF8044B70477C
:101A40000020FAE71C1D030830B40A4D002305F1FD
:101A5000140401E0272B09D003EB43020133A15CFE
:101A60008142F7D12A4430BC907D7047002030BCC1
:101A7000704700BF081D03082DE9F34105690646BC
:101A80000F467DBBD0F80080C8F30A0323B30023C0
:101A9000D6F80080019315F001FC042819D1224CDE
:101AA000236943F001032361BBB2A8F8003015F0AD
:101AB000F5FB04282ED108F102030193019B3F0C92
:101AC0001F8015F0EBFB2369042823F00103236139
:101AD00025D06FF0010505E015F0E0FB042805D0E6
:101AE0004FF0FF35284602B0BDE8F0810E4C236967
:101AF00043F002032361C4F81480236943F04003D8
:101B0000236115F0CBFB2369042823F00203236132
:101B1000BDD0E5E7236923F001032361D9E73368EA
:101B200004333360DEE700BF00200240F8B504460E
:101B30000D468E180027B54201D12069F8BDE36833
:101B4000591CE160234415F8012B1A720429F2D1C3
:101B5000A1682046FFF790FFE7602061EBE770B5D2
:101B6000448806460D46C4F30B042246002128464D
:101B70001FF06FFC33690A4A934209D3094A934222
:101B800006D2224628461946BDE870401EF066BBC4
:101B900023B121462846BDE87040184770BD00BFFC
:101BA000207503080C760308064B07498B4202D3C5
:101BB0000023184670471A88C2F30B029042F8D0EF
:101BC0001433F3E7C070030820750308024A136852
:101BD00023EA0000106070476430002008B503F06D
:101BE00043FE024B024ADA60FEE700BF00ED00E070
:101BF0000400FA05024A034B1278197809F0EEB98D
